:020000040800F2
:100000000020001091FC020835B5020811300008EC
:1000100031B502082DB5020829B50208000000001C
:1000200000000000000000000000000025B50208EC
:1000300021B50208000000001DB50208592800087B
:10004000F9FC0208F9FC0208F9FC0208F9FC0208B4
:10005000F9FC0208F9FC0208E13100080D33000840
:10006000D13200089532000859320008F54A0008DC
:10007000E54A0008D54A0008C54A0008B54A000804
:10008000A14A00088D4A0008F9FC0208F9FC0208A0
:1000900045B90208F9FC0208F9FC02081D32000803
:1000A000351D0008751D0008251D00089D1D000850
:1000B000651D0008551D0008451D0008F9FC0208D3
:1000C000F9FC0208F9FC0208F9FC0208F9FC020834
:1000D000F9FC020885290008092900088D28000874
:1000E000A5310008F9FC02080DB50208F9FC020868
:1000F000F9FC0208F9FC0208F9FC0208F9FC020804
:10010000000000000000000000000000F9FC0208F0
:10011000F9FC0208F9FC0208F9FC0208F9FC0208E3
:10012000794A0008654A0008514A00083D4A00081B
:10013000294A0008F9FC0208000000000000000045
:10014000F9FC0208F9FC0208F9FC020800000000B2
:10015000000000000000000000000000000000009F
:100160000000000000000000F9FC0208F9FC020891
:10017000F9FC020800000000000000000000000080
:0801800000000000F9FC020878
:1001880003680A7A591C01601A70704738B50B4C1D
:1001980023688BB15A68821A002A054604DA0CE0F3
:1001A8005A68AA1A002A07DB9A68226018461A6851
:1001B80090472368002BF3D138BD38BD9431002017
:1001C8000B4B002210B4027203F1DC04012102E09F
:1001D800072A09DC9979890702D5197981540132EE
:1001E8009C4203F11403F3D15DF8044B704700BF40
:1001F800EC40030824230370704700BF012310B4A8
:1002080015211424222244704171C27003700371B5
:1002180083705DF8044B70472DE9F0410B78057B3E
:10022800DB43DFB200F1130200F11D0302F8015FA6
:100238009342FBD1DFF890E000F12701002203F898
:10024800012F9942FBD114210524002647FA04F313
:1002580003F00103002B1E4414BF4FF019084FF0A0
:100268000A0814F0010FF6B214BFAC464FF0000CA8
:100278000023CA1810FA82F20133434582F814C0E9
:10028800F7D15A1E92B20132013C8B18621C9BB204
:1002980001D01946DAE716F0010F14BF19240A2411
:1002A8000022991810FA81F10132A2420D75F8D195
:1002B80013449BB25A1C0344002192B21975AEF83C
:1002C80000200261BDE8F081541D00202DE9F04FA7
:1002D800DFF890A0BAF802300B3383B01FFA83F925
:1002E80001F1060B4FF001084FF0000C002711F840
:1002F80001EB3E464C460122A4F10B039BB201914F
:1003080005E001339BB2017B29759C4208D0C518D2
:10031800002AF6D1C51801339BB29C422A75F6D142
:1003280003190136092F019983F814C0F6B20CD0CD
:10033800092E15D008FA07F313EA0E0F14BF01228D
:1003480000220C34A4B20137D6E709F178095945DF
:100358001FFA89F9CAD1AAF802C003B0BDE8F08F24
:100368000022EEE7541D00202DE9F047DFF85C80FD
:10037800B8F8043004331FFA83FC01F109094FF07F
:10038800010E11F8017B64460026231F0EFA06F2BF
:100398009BB23A40C2B1B0F80CA0C51801339BB269
:1003A8009C4285F814A0F5D101360434082EA4B275
:1003B800EBD10CF1200C49451FFA8CFCE1D100234C
:1003C800A8F80430BDE8F0879246E6E7541D0020FF
:1003D80010B40268047B11680223A340194209D0B3
:1003E8000649406800240C7001684FF6FE742140ED
:1003F800016053605DF8044B704700BFD86C002063
:10040800436A826970B4D154436A0469426B013308
:10041800A34228BF00234362DAB1116811F0010139
:1004280001D070BC7047856A86699D422E44D660AB
:100438000BD3641B546081621368002143F00103ED
:1004480080F8441070BC136070475D1B5560836270
:10045800F2E7026D136843F080031360E1E700BF21
:10046800026B10B462B1036CC2684469D11A013BD3
:10047800615C5DF8044B08BF13460364C8B270475B
:10048800016A4369C4685B5C0131A14228BF114617
:1004980001625DF8044BD8B2704700BF436B13B1DB
:1004A80090F844007047836A406A181AB0FA80F0DE
:1004B80040097047416A836A99420AD3CB1A416B53
:1004C800026961B14968501E0B4483420AD2C01ABE
:1004D800704702691144CB1A416B0029F2D1501EB2
:1004E800C01A704700207047036B43B1026C5B6809
:1004F80093422FBF981AC0689B1AC0187047C269E8
:10050800036A9A422FBFD01AC0688018C01A704771
:100518000A4B30B503F1140493F900205D78072ADB
:10052800C8BF143A811804330D7313F8025C85545C
:1005380013F8012C0A76A342EED130BDE424030857
:1005480003682DE9F041DF691FB13B46BDE8F04182
:100558001847002A164611DD04460D460E4400E0F1
:1005680023689B68204698470028F9D0236815F827
:10057800011B1B6820469847AE42F1D1BDE8F081C7
:1005880000232322027043708370C37070472D23A9
:1005980043702E2303712F23C3717047002870B551
:1005A8001EDB0928044620DD012303EB83035B00DF
:1005B800B0FBF3F2092AF8D87BB10E4EB4FBF3F086
:1005C8000928CCBF57223022A6FB03E5024403FBCF
:1005D8001044EB0801F8012BF0D100230B7070BD1B
:1005E8002D230B7040420131DBE7303001F8010B5D
:1005F800F3E700BFCDCCCCCC884230B44FF0010437
:100608002ED301FB04F4B0FBF4F58D42F9D284B18A
:10061800AAB901E0B0FBF4F5092DCCBF572230226E
:100628002A4404FB150003F8012BB4FBF1F4002C59
:10063800F0D100221A7030BC7047B0FBF4F5092DD8
:10064800CCBF372230222A4404FB150003F8012BC3
:10065800B4FBF1F4002CF0D100221A7030BC7047C2
:100668000546002AEBD1D7E703685A1C02601970C7
:10067800704700BF2DE9F047089C2578002B80467D
:1006880089460CBF4FF0200A4FF0300A661C35B37C
:10069800002A29DD334601E0024698B113F8011B10
:1006A800501E0029F8D1971E60B13D46013D5146C4
:1006B8004046C8476B1C002BF8DC257827EAE77012
:1006C800013055B1041B29464046C847301916F871
:1006D800015B002DF7D1BDE8F087BDE8F087002A5F
:1006E80004DC2846BDE8F0870020EBE7571EDCE76E
:1006F8000A44914251D030B441F2210411F8013B2F
:1007080080EA0320430010F4004F84EA03059BB2FB
:10071800ADB208BF1D466B0015F4004F84EA030014
:100728009BB280B208BF1846430010F4004F84EA19
:1007380003059BB2ADB208BF1D466B0015F4004F10
:1007480084EA03009BB280B208BF1846430010F445
:10075800004F84EA03059BB2ADB208BF1D466B008B
:1007680015F4004F84EA03009BB280B208BF184614
:10077800430010F4004F84EA03059BB2ADB208BFF2
:100788001D466B0084EA030015F4004F85B298B249
:1007980018BF28468A42B1D130BC70478368426886
:1007A800D0ED037A00EB83010133934281ED040A13
:1007B800836004BF0023836000EB830393ED047A16
:1007C800036870EE277A9A42C0ED037A77EEC77A0B
:1007D800C0ED037A0CDA013307EE103AF8EEC76A77
:1007E800B7EE007A87EEA60A036030EE070A704774
:1007F80007EE102AB8EEC77A87EE870A704700BF5F
:1008080090ED097A90ED004AD0ED0A6AD0ED014AE0
:10081800D0ED047A90ED035AD0ED025AA4EE007A96
:10082800B0EE406AB0EE470AB0EE667AA6EE247AD9
:1008380067EEC07AA0EE457AE6EE257A80ED097A71
:10084800C0ED0A7A704700BFD0ED057A90ED013A05
:10085800D0ED003AD0ED064A90ED024A90ED077AC5
:1008680090ED035A90ED086AD0ED045AC0ED067A6F
:10087800F0EE406A27EE830AC0ED056AA3EEA60AE9
:1008880080ED087AA4EE240AA5EE470AA5EEC60A6A
:1008980080ED070A704700BFD0ED007A90ED017A2D
:1008A80030EE670AE7EE007AB0EE670AC0ED007A2C
:1008B800704700BF704700BF704700BF2DE9F04F79
:1008C800DFF81CB2DFF81CE2BBF80020DEF8086095
:1008D800BBF90430BBF90250BBF90A80C2EB2614FD
:1008E80004FB04F424135200C2EBE60203FB04F3F6
:1008F80005FB02F29B1303EBE223B3F5FA364FEA4A
:10090800E37589B045F1FF373246A6FB0645CDE9C8
:10091800024502FB07F205EB4202CDE90467029E9D
:10092800BBF90840039208FB02FC4FEAE87906FB92
:1009380009CC3A46A8FB0689049ECBF81830E5177F
:1009480004FB02F206FB0522A4FB0667E1441744F8
:100958004FEA182242EA096200924FEA29220192DC
:100968003D03DDE90078340345EA16553F19BBF825
:100978000660069048EB05083C1C48F5004503EB6B
:100988008302A4FB068906FB0599803213124FEAFD
:1009980069064FEAE977079356EA07038A4600F0A3
:1009A8009280DDE90489BBF90E20DEF80C40BBF922
:1009B80010004946C4F5801ED317DDE9024502FB45
:1009C80001F108FB0311A2FB08230B444FEA43493A
:1009D8002B46C11700FB03F304FB0133A0FB040102
:1009E800BBF90C401944E30001937346DC1700235C
:1009F800009349EAD2394FEA4248DDE9002310EB77
:100A0800080041EB0901E50712184FEACE744B4183
:100A180045EA5E05A41A65EB0305221945EB0503B3
:100A280012196B4199019001801841EA926159416C
:100A38008B00820043EA9073101943EB05018B0089
:100A4800820043EA907310460019194632463B4625
:100A580069412EF045FFBBF916204C13450B45EABA
:100A6800C14502FB04F6D31705FB0366A2FB052369
:100A78003344BBF9146002FB04F405FB034406FB92
:100A880001FEA2FB0523F717234400FB07EE540ED3
:100A9800A6FB0067774444EAC3144FEAD648001916
:100AA8004FEA636548EA473869414FEAE74918EB76
:100AB8000008BBF9124049EB01094FEA182646EA3B
:100AC800096620013618069B0BB1360A1E60BAF17A
:100AD800000F02D0079BCAF8003009B0BDE8F08FBC
:100AE80080370020541D0020704700BF704700BFAA
:100AF80050F8043C012280F83520143803B1184717
:100B0800704700BF4FF400630382704790F8493084
:100B180013B1002280F849201846704770B5044682
:100B280082B01830256D94F85C106B460622A847F1
:100B3800A8B19DF804009DF800609DF801109DF88B
:100B480002509DF803209DF8053041EA062143EA4A
:100B5800002342EA0522A184E2842385012002B011
:100B680070BD00BF70B5044682B00830256A6B4678
:100B780006223B21A847A8B19DF804009DF8006013
:100B88009DF801109DF802509DF803209DF805304E
:100B980041EA062143EA002342EA05226182A28251
:100BA800E382012002B070BD30B490E81200057BEA
:100BB80043690222AA404A602268586A996A4FF635
:100BC800FE752A408842226004D1012283F844201D
:100BD80030BC70479C695A6B0C44D4600DD81869B6
:100BE8000024411A51609C621168002041F0010103
:100BF80083F8440030BC11607047411A5160986214
:100C0800F2E700BF70B40468037B2268022101FA8E
:100C180003F31A4213D042690A49582000FB021212
:100C28004FF6FE7650685289C568006829683140D9
:100C38002960C168D24392B20A40C260636070BC46
:100C4800704700BF7845002030B4094B1C7864B168
:100C5800084B002503EBC4041A6899885562D068CC
:100C680008330143A342D160F6D130BC704700BFBE
:100C7800984900209C49002010B40268047B116840
:100C88000223A340194209D00649406800240C7089
:100C980001684FF6FE742140016053605DF8044B13
:100CA800704700BFB2410020F0B5064683B00D463C
:100CB8000024012714E003290CBF03220122C3F3F7
:100CC800011E6946C3F3810330468DF805208DF86F
:100CD80006E08DF8073020F00DFC0134102C0FD001
:100CE8002B8807FA04F21342F7D0AB78E978009220
:100CF800022903F003028DF80420DCD10A46DEE75E
:100D080003B0F0BDF0B4334C00EB800004EB80047A
:100D18006468002C5BD0304E49004FF42040CDB2BF
:100D28003060A169090444D460682C4F45F0807193
:100D3800384041F4903101434FF420406160306005
:100D480003E0411E002838D00846A1698F07F8D56E
:100D58004FF42040A262306002E0421E68B31046A1
:100D6800A2691106F9D562681C4945F0007545F479
:100D780080350A4015434FF420406560306002E03A
:100D8800421ED0B11046A2699207F9D5A362A369A1
:100D98004FF420409B06306005D4431E68B11846C6
:100DA800A3699B06F9D520233060E3610120F0BCDC
:100DB8007047411E08B10846B3E7094A1388013352
:100DC8009BB24FF0FF3131601380F0BC7047204672
:100DD800F0BC7047D844002000450020009800FC73
:100DE80004450020134600200A4668218AE70023AC
:100DF800262203600270272282700122436002715A
:100E08008371704770B5448806460D46C4F30B04D9
:100E180022460021284631F0ACFA3369094A934248
:100E280009D3094A934206D2224628461946BDE804
:100E380070402FF01DB823B121462846BDE8704008
:100E4800184770BDB08203085883030870B54E6810
:100E5800054630462EF09AF8314604460246286880
:100E68002FF006F82A68131901333B212B6011551E
:100E780070BD00BF08B51CF011FE024B024ADA60D3
:100E8800FEE700BF00ED00E00400FA05024A034B4C
:100E98001278197829F0EEB8B81D0020B91D002085
:100EA8002DE9F0470569C3681D4028D00F4606465E
:100EB8004FF000484FF00009B5FA85F328FA03F21D
:100EC800D2431B3B32611540042B16D8DFE803F0F0
:100ED8003129211903007B6A002B32D003F1FF3A34
:100EE8001FFA8AFAC7F824903C6A34B1236820466E
:100EF800514698476468002CF8D1002DDCD1BDE834
:100F0800F0873868716B036889B29847002DD3D190
:100F1800F5E77868B16B036889B29847002DCBD1A3
:100F2800EDE7B868F16B036889B29847002DC3D123
:100F3800E5E7F868316C036889B29847002DBBD1A2
:100F4800DDE7F36A1FFA83FACEE700BF30B504463F
:100F5800006D61710368A26823F00103036087B024
:100F6800A379009213F004023DD04FF4805213F09D
:100F78000203019244D102934FF480630022039349
:100F880011F00103059237D1049308238D076946B0
:100F980048BF049321F028FA6079236DA17900F005
:100FA8000202002A15BF4FF440324FF480324FF44A
:100FB8000034002410F0010F586808BF2246CC07FF
:100FC8004CBF024320EA02025A609A6809074CBFE4
:100FD80042F0080222F008029A601A6842F0010200
:100FE8001A6007B030BD13F0020301920BD04FF422
:100FF800005513460295C1E7042304930C23C5E763
:101008004FF40053B7E70293B8E700BF10B50446A2
:10101800006DA160036823F001030360A37986B023
:1010280013F00402009141D04FF4805213F00203F0
:10103800019244D102934FF4806362790393D107FC
:101048004FF000030493059345BF0423049308233A
:101058000C236946920748BF049321F0C5F96079CB
:10106800236DA17900F00202002A15BF4FF4403227
:101078004FF480324FF40034002410F0010F586808
:1010880008BF2246CC074CBF024320EA02025A603E
:101098009A6809074CBF42F0080222F008029A60D9
:1010A8001A6842F001021A6006B010BD13F002037C
:1010B800019207D04FF4005113460291BDE74FF457
:1010C8000053B7E70293B8E72DE9F34105690646EF
:1010D8000F467DBBD0F80080C8F30A0323B3002372
:1010E800D6F80080019323F023F8042819D1224C64
:1010F800236943F001032361BBB2A8F8003023F051
:1011080017F804282ED108F102030193019B3F0C24
:101118001F8023F00DF82369042823F001032361BD
:1011280025D06FF0010505E023F002F8042805D06A
:101138004FF0FF35284602B0BDE8F0810E4C236918
:1011480043F002032361C4F81480236943F0400389
:10115800236122F0EDFF2369042823F002032361B1
:10116800BDD0E5E7236923F001032361D9E733689C
:1011780004333360DEE700BF00200240F8B50446C0
:101188000D468E180027B54201D12069F8BDE368E5
:10119800591CE160234415F8012B1A720429F2D175
:1011A800A1682046FFF790FFE7602061EBE700BFEA
:1011B800F0B583B004466B46062203211E2021F0B9
:1011C800ADFB00283CD09DF800509DF801109DF81B
:1011D80002709DF803209DF804609DF8053041EAEF
:1011E800052142EA072243EA062309B212B21BB2DA
:1011F800144D06EE901A07EE102A07EE903AF8EE14
:10120800E66A95ED005AD5ED025A95ED016AB8EEF9
:10121800C77AF8EEE77A66EE856A27EE257A67EEF2
:10122800867AFDEEE66ABDEEC77AFDEEE77A16EE3F
:10123800901A17EE102A17EE903A2180A280638048
:1012480003B0F0BD0000002070B582B06B460622E6
:10125800F721762021F062FB9DF801209DF80430EB
:101268009DF800609DF803509DF802409DF8050028
:10127800074912011B0142EA063243EA053342EAF2
:10128800141243EA1013CA608B6002B070BD00BF2D
:10129800541D0020682021F041BB00BF10B44C0948
:1012A800012250F8243001F01F0102FA01F10B432A
:1012B80040F824305DF8044B704700BF00210A4A0B
:1012C8000B4604E00133242B0BD012F80C1C884287
:1012D80002F10C02F6D1054803EB430300EB83004F
:1012E80070470020704700BF3426030820260308F3
:1012F80000210A4A0B4604E00133242B0BD012F8D4
:101308000C1C884202F10C02F6D1054803EB43039A
:1013180000EB830070470020704700BF2C260308AD
:1013280020260308022828BF022010B4084C094BC5
:10133800207000EBC00200EB820207495DF8044B05
:10134800013003EB4203C0B20B6024F0ADBA00BF1A
:101358008E840020708C0020A484002038B5434B74
:101368005A899989914224BF00225A81198ADA89B7
:10137800914224BF0022DA81DA7892B1072A10D08C
:101388003B4C3C48A27801210025062A017099703F
:10139800DD719D7152D92379DFED376A002B3CD17D
:1013A80038BDDA79002A4ED09A783248DFED326AB1
:1013B8000178042A38BF042207EE902AB8EEE77AAB
:1013C80007EE901A27EE267AF8EEE77A9A7067EE1B
:1013D800877A274CA2780025062A9D712BD8274B9F
:1013E80003EB8203D3ED056AF4EEE76AF1EE10FA37
:1013F80010DDC6EE877AFDEEE77A17EE903A102BED
:10140800A8BF1023012BB8BF0123DBB28B4228BF32
:101418000B4603702379002BC2D0013A032ABFD8A8
:10142800B7EE000A80EE260A2EF096FE2388984230
:1014380038BF208038BDDFED106AD5E7DFED107AC0
:10144800B0EE677ACBE79A780A48DFED0E6A017842
:1014580007EE102A07EE901AB8EEC77AF8EEE77A88
:1014680027EE267A67EE877AB3E700BF0C70002074
:101478004C450020087B00206F120338E424030841
:101488006F12833A6F12033938B50D4C0D4DAC42CB
:1014980006D2616820461434FFF7B4FCAC42F8D396
:1014A800094B0A4C0A4818600025257027F0B4F942
:1014B800084B094A65701A60BDE838401EF05CBBED
:1014C800787E0308B0820308A48400208E8400205C
:1014D800708C002048380020A8840020F0B50C2922
:1014E8002BD8DFE801F06F2A2A2A4C2A2A2A2B2A2D
:1014F8002A2A0700046AB2F80CE097881668674D34
:1015080024F480540462036A4468C16923F40053D4
:1015180043EA0E3321F4E641A84243EA073341EA9D
:10152800062100F0B58005F50065A84200F0B080FE
:1015380092684460C16102640362F0BD046A9689DE
:101548009588D2F800E0554F24F480740462036A49
:101558004468C16923F4007343EA062321F0730148
:10156800B84243EA052341EA0E017ED04C4DA84219
:101578007BD092684460C161C2630362F0BD046AB3
:1015880096899588D2F800E0444F24F0100404624C
:10159800036A4468816923F0200321F0807143EADB
:1015A800061321F4E641B84243EA051341EA0E2145
:1015B80048D03B4DA84245D092684460816182631F
:1015C8000362F0BD046A9389B2F804E01768334EE9
:1015D80024F001040462056A4468816943EA0E0341
:1015E80021F4803125F002059BB221F07301B0424D
:1015F80043EA050341EA070114D0294DA84211D056
:1016080005F54065A8420DD005F58065A84209D0CA
:1016180005F58065A84205D09268446081614263FF
:101628000362F0BDD689158A578A23F0080333432D
:101638003D43D68824F4407423F00403ADB2334309
:101648002C43E9E7D589178AD68823F0800343EA33
:10165800051324F44064558A23F0400344EA8704C0
:1016680043EA061344EA8504A6E7D589178AD6888B
:1016780023F4006343EA052324F44054558A23F4F1
:10168800806344EA071443EA062344EA051470E732
:10169800158A24F4804444EA851449E7002C014063
:1016A800003401402DE9F84F4FF48C7200218F4827
:1016B8008F4CDFF864928F4D8F4E904FDFF85C822D
:1016C80030F057FE8E488F49DFF854E2DFF854C2F5
:1016D80000221359834200F0F880B3F1804F00F0E4
:1016E800F680AB4200F0F580B34200F0F480BB42D4
:1016F80000F0F380734500F0F280634500F0F1805C
:10170800434500F0F080DFF820A2534500F0A780A1
:101718000AF5806A534508BF092300F0A1801432F6
:10172800F02AD6D1DFF8C881774F784D08F1F00656
:101738004FF0030A4FF0020998F804301C09013CE5
:10174800052C03F00F0300F2838037F8140040FAE9
:1017580003F2D2077CD54FF0010B0BFA03F3013BE0
:1017680018402EF00DF96A4B1B5D184415EBC004A8
:101778006ED055F83030674898F8081003F13842B1
:10178800920A825C02F01F005209022A0BFA00FB3F
:1017980000F09480032A00F08A80012A05D1594A72
:1017A800584852694BEA02024261B4F804E0BEFAB2
:1017B8008EF2C2F11F0292B2D00803EB800002F051
:1017C8000702046A92004FF00F0C0CFA02FC24EA9C
:1017D8000C040462046A01FA02F222430024026241
:1017E8004FF0010C224603E0102A04F102042FD026
:1017F8000CFA02F030EA0E0102F10102F4D1D3F83A
:1018080008B00AFA04F1C9430BEA010BC3F808B09F
:10181800D3F808B0C3F808B0B3F804B01FFA8BFBCC
:101828002BEA00009880988880B298801868084051
:101838001860D3F800B009FA04F040EA0B00186009
:10184800D868102A01EA0001D96004F10204CFD156
:1018580008F1140846457FF46FAFBDE8F88F0823F8
:1018680009EBC3034FF0010B93F834A00AF01F03F0
:101878004FEA5A1ABAF1020F0BFA03F30BD0BAF176
:10188800030F0ED0DA457FF44AAFD1F814A043EA2B
:101898000A034B6143E7D1F818A043EA0A038B61B6
:1018A8003DE7D1F81CA043EA0A03CB6137E7154AA4
:1018B8001448D2694BEA0202C26176E7114A11481C
:1018C80092694BEA020282616FE70023C8E70123AD
:1018D800C6E70223C4E70323C2E70423C0E70523BE
:1018E800BEE70623BCE70723BAE700BF906B0020DA
:1018F800EC400308000400400008004000100040CD
:10190800002C0140001002406C4503083083002081
:101918007845030880450308E42403080040014093
:10192800001400400034014000440140002867D002
:1019380003682DE9F04F03F138445C4EA40A0125F1
:10194800345D04F01F066409022C05FA06F558D028
:10195800032C00F0A580012C58D08088B0FA80F4C0
:10196800C4F11F04A4B2E50803EB850504F00704DD
:101978002E6AA4000F27A74026EA07062E622E6AC1
:1019880001F00307A2407C1E3243012CC1F3810CF5
:10199800C1F300182A62C1F341113CD9C60700F10E
:1019A8008980850700F19580440700F1A38002072C
:1019B80000F1B180C60600F1BF80850600F1CD8038
:1019C800440600F1DB80020600F1E980C60500F15B
:1019D800F780850500F10581440500F113810205B2
:1019E80000F12181C60400F12F81850400F13D81B9
:1019F800440400F14B81020400F15981BDE8F08FE5
:101A080070472B4CA6693543A561A6E7284C666943
:101A180035436561A1E7002422464FF0010E4FF0DF
:101A2800030904E00132102A04F10204E6D00EFA98
:101A380002F636EA0005F5D1D3F808A009FA04F54C
:101A4800ED430AEA050AC3F808A0D3F808B00CFA6F
:101A580004FA4AEA0B0AC3F808A0B3F804A01FFA6C
:101A68008AFA2AEA06069E80B3F804A008FA02F663
:101A780046EA0A06B6B29E801E682E401E60D3F85B
:101A880000A007FA04F646EA0A061E60D3F80CA07E
:101A980001FA04F605EA0A0A46EA0A05DD60C1E722
:101AA800034CE6693543E56157E700BF8045030805
:101AB800001002401A6822F003021A601A683A43BA
:101AC8001A60DA6822F003020A438507DA607FF5B4
:101AD8006BAF1A6822F00C021A601A6842EA870291
:101AE8001A60DA6822F00C0242EA81024407DA60DE
:101AF8007FF55DAF1A6822F030021A601A6842EA70
:101B080007121A60DA6822F0300242EA0112DA603B
:101B180002077FF54FAF1A6822F0C0021A601A68F0
:101B280042EA87121A60DA6822F0C00242EA811299
:101B3800C606DA607FF541AF1A6822F440721A606F
:101B48001A6842EA07221A60DA6822F4407242EA06
:101B580001228506DA607FF533AF1A6822F4406205
:101B68001A601A6842EA87221A60DA6822F4406228
:101B780042EA81224406DA607FF525AF1A6822F42A
:101B880040521A601A6842EA07321A60DA6822F488
:101B9800405242EA0132DA6002067FF517AF1A684E
:101BA80022F440421A601A6842EA87321A60DA68F8
:101BB80022F4404242EA8132C605DA607FF509AF75
:101BC8001A6822F440321A601A6842EA07421A6018
:101BD800DA6822F4403242EA01428505DA607FF58C
:101BE800FBAE1A6822F440221A601A6842EA874259
:101BF8001A60DA6822F4402242EA81424405DA6037
:101C08007FF5EDAE1A6822F440121A601A6842EAAB
:101C180007521A60DA6822F4401242EA0152DA6086
:101C280002057FF5DFAE1A6822F440021A601A68CE
:101C380042EA87521A60DA6822F4400242EA815284
:101C4800C604DA607FF5D1AE1A6822F040721A60D5
:101C58001A6842EA07621A60DA6822F0407242EAB9
:101C680001628504DA607FF5C3AE1A6822F040622B
:101C78001A601A6842EA87621A60DA6822F04062DB
:101C880042EA81624404DA607FF5B5AE1A6822F050
:101C980040521A601A6842EA07721A60DA6822F03B
:101CA800405242EA0172DA6002047FF5A7AE1A6870
:101CB80022F040421A601A6842EA87771F60DA68A1
:101CC80022F0404242EA8171D960BDE8F08F00BF3E
:101CD80010B50409013C052C17D80D4B33F8142016
:101CE80000F00F0042FA00F313F001030DD00123B6
:101CF80003FA00F0013810402DF042FE054A064B69
:101D0800125D104403EBC00010BD002010BD00BFE1
:101D18006C450308784503083083002001490248D0
:101D2800FFF7BEB8806C0020004801400149024816
:101D3800FFF7B6B8306C0020004001400149024866
:101D4800FFF7AEB8086C00200008004001490248BF
:101D5800FFF7A6B8E06B00200004004002494FF0EE
:101D68008040FFF79DB800BFB86B002010B5064C47
:101D780006482146FFF794F804F1C8010448BDE875
:101D88001040FFF78DB800BF906B0020002C014079
:101D98000044014001490248FFF782B8906B0020D7
:101DA800002C01402DE9F0410468514DA30AAB42D3
:101DB80000F084800AD94F4DAB4277D00135AB4251
:101DC8005FD0023DAB426DD0BDE8F0814A3DAB42E9
:101DD80070D00135AB4258D0B3F5801FF4D14FF025
:101DE800480E012647794FEA970C00296AD0B000BF
:101DF800634685190227D4F80C809F400CEB4503F5
:101E0800BFB23D4D03F1040C47EA080745F823101B
:101E180045F82C20E760EFF31181502282F31288F5
:101E2800821905EBC2021369002B32D01362043306
:101E3800821905EBC202576917B11F605369043351
:101E4800821905EBC202976917B11F6093690433C1
:101E5800821905EBC202D76917B11F60D369043331
:101E68000027CAB21F6082F31188304405EBC00016
:101E7800036A8BB9E3684FF6FE721340E360BDE86E
:101E8800F0814FF4887E0626ACE74FF0980E0326C3
:101E9800A8E705EB0E03CBE7E36843F00103E36033
:101EA800BDE8F0814FF0C00E04269BE74FF0E80E26
:101EB800052697E74FF0700E022693E74FF0200EA5
:101EC80000268FE7BF08022306FA03F0BB40DB4376
:101ED800E768094D9BB23B4087190CEB470CE36060
:101EE8000CF1040345F82C1045F8232093E700BFB4
:101EF8004B00100051001000906B002030B50368B3
:101F08005C4D18885C4CB4FBF2F20139013AAB42E3
:101F180094B283B089B282B266D05848834263D003
:101F2800B3F1804F60D0A0F5983083425CD000F5C3
:101F38008060834258D0524883425BD000F580606D
:101F480083427DD022F4407200F58C3092B28342F5
:101F58001A80D9621C850ED0484A93420BD002F5EC
:101F68004062934207D002F58062934203D002F5A3
:101F78008062934201D100221A8601225A611A888E
:101F88003C4992B242F001028B421A8062D0B3F10E
:101F9800804F61D03B4A934260D002F58062934201
:101FA8005ED002F5006293425CD002F580629342F3
:101FB8005AD002F59032934258D002F540629342CB
:101FC80056D002F5806293421ED002F58062934299
:101FD80008BF092219D002A84FF0012340F8043D98
:101FE80020F08CFD03B030BD254822F070028342FA
:101FF80092B2A3D101201A80D9621C8558611A882F
:1020080092B202431A80C5E708221F4B03EBC203B2
:1020180001A893F835408DF80440012300228DF87B
:1020280005308DF807308DF8062020F067FD1B2C51
:10203800D8D1164B019301A820F060FD03B030BD44
:1020480001201A80D9621C8558611A8892B202430D
:102058001A809CE70022D8E70122D6E70222D4E7BB
:102068000322D2E70422D0E70522CEE70622CCE7F6
:102078000722CAE7002C014000A24A0400340140AC
:102088000010004000040040E42403081901000186
:10209800204B98422DD0B0F1804F2CD0A3F594332B
:1020A80098422AD003F58063984228D003F500634C
:1020B800984226D003F58063984224D003F59033E4
:1020C800984222D003F54063984220D003F58063FC
:1020D800984207D003F58063984208BF092202D0CE
:1020E8000020704708220C4B03EBC20393F834001E
:1020F80070470022F7E70122F5E70222F3E70322FF
:10210800F1E70422EFE70522EDE70622EBE70722D5
:10211800E9E700BF002C0140E42403082DE9F04F53
:10212800013085B0C3B203938C4D8D4F8D4C8E4ECC
:102138000A230293DFF8349220F072FF4FF4FA7A00
:102148004FF0100C4FF47A70D9F80430C3F3080339
:10215800002B40F0C580EFF31183002B40F0C080C6
:102168002968A26800BF2B689942F9D1D7F800E026
:1021780000FB0EF39B1AB3FBFEF300FB01314FF09B
:10218800010E0191D9F80430C3F30803002B40F085
:102198008B80EFF31183002B40F086802B68A168B9
:1021A80000BF2A689342F9D1D7F800B000FB0BF2C0
:1021B800521AB2FBFBF200FB0323019A9B1AB3F5F8
:1021C8007A7FDFD3BAF1010ABED1039B002B40F01E
:1021D800C1804FF47A7ADFF8949150464FF0100C92
:1021E800D9F80430C3F30803002B40F09680EFF3CE
:1021F8001183002B40F091802968A26800BF2B68EA
:102208009942F9D1D7F800E000FB0EF39B1AB3FB13
:10221800FEF300FB01314FF0010E0191D9F80430B3
:10222800C3F3080323BBEFF311830BBB2B68A1682F
:1022380000BF2A689342F9D1D7F800B000FB0BF22F
:10224800521AB2FBFBF200FB0323019A9B1AB3F567
:102258007A7FE3D3BAF1010AC2D1029B013B029310
:102268007FF468AF414B424ADA6005B0BDE8F08FB1
:10227800EFF311888CF31288A1682368DB0344BF4D
:10228800C6F800E0A1682B6832685FFA88F888F31E
:102298001188D7F800801A4400FB08F35B1AB3FBD7
:1022A800F8F300FB0233D0E7EFF311888CF31288C0
:1022B800A1682368DB0344BFC6F800E0A1682B6867
:1022C80032685FFA88F888F31188D7F800801A44D2
:1022D80000FB08F35B1AB3FBF8F300FB02336CE76F
:1022E800EFF311828CF31288D4F808E02368D9033D
:1022F80003D501233360D4F808E02B683168D2B2E3
:1023080082F311883A68194400FB02F3A3EB0E0329
:10231800B3FBF2F300FB013131E7EFF311828CF3E9
:102328001288D4F808E02368D90303D50123336061
:10233800D4F808E02B683168D2B282F311883A6881
:10234800194400FB02F3A3EB0E03B3FBF2F300FB0B
:10235800013160E7184620F0D3FC3AE73C450020FD
:102368004045002010E000E03845002000ED00E086
:102378000400FA052DE9F04F013085B0C3B203938C
:102388000B4602918B4C8C4E002B00F099808B4DA4
:102398008B4FDFF8309220F043FE4FF4FA7A4FF07B
:1023A800100C4FF47A70D9F80430C3F30803002BEB
:1023B80040F0DE80EFF31183002B40F0D9802968CC
:1023C800A26800BF2B689942F9D1D7F800E000FB5A
:1023D8000EF39B1AB3FBFEF300FB01314FF0010E25
:1023E8000191D9F80430C3F30803002B40F087802B
:1023F800EFF31183002B40F082802B68A16800BFA7
:102408002A689342F9D1D7F800B000FB0BF2521AB0
:10241800B2FBFBF200FB0323019A9B1AB3F57A7F08
:10242800DFD3BAF1010ABED1039B002B40F0BD8077
:102438004FF47A7ADFF88C9150464FF0100CD9F8A7
:102448000430C3F30803002B75D1EFF31183002B7D
:1024580071D12968A26800BF2B689942F9D1D7F8D1
:1024680000E000FB0EF39B1AB3FBFEF300FB013107
:102478004FF0010E0191D9F80430C3F3080313BBE0
:10248800EFF31183FBB92B68A16800BF2A68934258
:10249800F9D1D7F800B000FB0BF2521AB2FBFBF2ED
:1024A80000FB0323019A9B1AB3F57A7FE3D3BAF1B1
:1024B800010AC4D1029B013B0293002B7FF467AF52
:1024C80005B0BDE8F08FEFF311888CF31288A1688E
:1024D8002368DB0344BFC6F800E0A1682B683268B4
:1024E8005FFA88F888F31188D7F800801A4400FB4F
:1024F80008F35B1AB3FBF8F300FB0233D2E7EFF300
:1025080011888CF31288A1682368DB0344BFC6F8DE
:1025180000E0A1682B6832685FFA88F888F31188B0
:10252800D7F800801A4400FB08F35B1AB3FBF8F3F2
:1025380000FB023370E7EFF311828CF31288D4F8B2
:1025480008E02368D90303D501233360D4F808E0F1
:102558002B683168D2B282F311883A68194400FBBB
:1025680002F3A3EB0E03B3FBF2F300FB01317FE7A9
:10257800EFF311828CF31288D4F808E02368D903AA
:1025880003D501233360D4F808E02B683168D2B250
:1025980082F311883A68194400FB02F3A3EB0E0397
:1025A800B3FBF2F300FB013118E7184620F0A8FB53
:1025B8003EE700BF10E000E0384500203C45002021
:1025C8004045002000ED00E0204B5B68C3F30803A2
:1025D80030B4BBB9EFF31183A3B91D4B1D4C186878
:1025E800A16800BF1A689042F9D11B4B1C684FF4D0
:1025F8007A7202FB04F3591AB1FBF4F130BC02FB06
:1026080000107047EFF31182102383F312881149E9
:102618008C680B6813F4803F104B02D001201860BF
:102628008C680B49D2B20D68186882F311880A4B7E
:1026380019684FF47A72284402FB01F31B1B30BC63
:10264800B3FBF1F302FB0030704700BF00ED00E080
:102658003C45002010E000E04045002038450020BF
:102668002DE9F84F8046FFF7AFFF254E2549DFF8E3
:10267800A0E0254A254D844610274FF47A7401209E
:10268800DEF80430C3F30803D3B9EFF31183BBB901
:102698000B68D2F808A000BFD1F800904B45F7D1DD
:1026A800D6F800B004FB0BF9A9EB0A09B9FBFBF952
:1026B80004FB0393A3EB0C034345E1D3BDE8F88F78
:1026C800EFF3118A87F31288D2F808B01368DB0396
:1026D80044BF2860D2F808B00B68D5F800905FFABC
:1026E8008AFA8AF31188D6F800A0994404FB0AF301
:1026F800A3EB0B03B3FBFAF304FB0933DAE700BFE0
:10270800404500203C45002010E000E0384500200E
:1027180000ED00E02DE9F04FDFF830C1474A4849A5
:10272800484E494D8046102718F1FF38C0F0848084
:10273800DCF80430C3F30803002B5CD1EFF31183FA
:10274800002B58D10B68946800BF08688342F9D100
:10275800D6F800904FF47A7000FB09FEAEEB040E39
:10276800BEFBF9FE00FB03EEDCF80430C3F30803FC
:102778004FF47A740120FBB9EFF31183E3B90B68C6
:10278800D2F808A000BFD1F800904B45F7D1D6F891
:1027980000B004FB0BF9A9EB0A09B9FBFBF904FB30
:1027A8000393A3EB0E03B3F57A7FBDD2DCF80430B4
:1027B800C3F30803002BDFD0EFF3118A87F31288E5
:1027C800D2F808B01368DB0344BF2860D2F808B019
:1027D8000B68D5F800905FFA8AFA8AF31188D6F860
:1027E80000A0994404FB0AF3A3EB0B03B3FBFAF331
:1027F80004FB0933D5E7EFF3118487F31288D2F885
:1028080008901368D80303D501232B60D2F80890E9
:102818000B682868E4B284F31188D6F800A04FF456
:102828007A7400EB030E04FB0AF3A3EB0903B3FB72
:10283800FAF304FB0E3E97E7BDE8F08F10E000E0E6
:102848003C450020404500203845002000ED00E0D0
:1028580030B4EFF31183102282F312880649074C33
:102868000A680748013200250A602560DBB2026861
:1028780083F3118830BC70473C4500203845002060
:1028880010E000E01D4B70B59C68236D226BDD697C
:10289800C2B1636B2BB12B0702D5236D08221A62D4
:1028A80070BD2A06F7D5A26A616A8A421FD0511CF8
:1028B800A069A162825C2069266D81423285EAD3D3
:1028C800A362E8E7A906E4D5E26A1AB1988C80B257
:1028D8009047DEE7E1699B8C6069DBB24E1CE661DC
:1028E8004354E169E368994228BFE261D1E7226D68
:1028F800136823F080031360CDE700BFF02D00209C
:102908001D4B70B55C68236D226BDD69C2B1636BCA
:102918002BB12B0702D5236D08221A6270BD2A0637
:10292800F7D5A26A616A8A421FD0511CA069A162C8
:10293800825C2069266D81423285EAD3A362E8E78A
:10294800A906E4D5E26A1AB1988C80B29047DEE70E
:10295800E1699B8C6069DBB24E1CE6614354E16916
:10296800E368994228BFE261D1E7226D136823F03A
:1029780080031360CDE700BFF02D00201D4B70B51C
:102988001C68236D226BDD69C2B1636B2BB12B0709
:1029980002D5236D08221A6270BD2A06F7D5A26AED
:1029A800616A8A421FD0511CA069A162825C2069B9
:1029B800266D81423285EAD3A362E8E7A906E4D509
:1029C800E26A1AB1988C80B29047DEE7E1699B8C85
:1029D8006069DBB24E1CE6614354E169E3689942E1
:1029E80028BFE261D1E7226D136823F080031360EA
:1029F800CDE700BFF02D002003685B6A03B11847DC
:102A0800704700BF03681B6A03B11847704700BFCF
:102A180003682DE9F041DF691FB13B46BDE8F0418D
:102A28001847002A164611DD04460D460E4400E0FC
:102A380023689B68204698470028F9D0236815F832
:102A4800011B1B6820469847AE42F1D1BDE8F081D2
:102A580003689B69184700BF0368DB68184700BF15
:102A680003689B68184700BF03685B68184700BF86
:102A780003681B68184700BF014B1868F8E700BFD8
:102A8800601F0020054B53F8203033B11A689B882B
:102A9800918A0B4218BF1B049361704708450020B8
:102AA8002DE9F04F4A484B4B4B4C4FF090414FF0BB
:102AB800010A4FF002094FF004084FF0080C4FF0DC
:102AC800100E20274026802530F8022B12F0010F27
:102AD80003D01960A3F804A0083312F0020F03D042
:102AE8001960A3F80490083312F0040F03D019609A
:102AF800A3F80480083312F0080F03D01960A3F874
:102B080004C0083312F0100F03D01960A3F804E0D2
:102B1800083312F0200F02D019609F80083312F09A
:102B2800400F02D019609E80083312F0800F02D047
:102B380019609D80083312F4807F05D04FF4807BA4
:102B48001960A3F804B0083312F4007F05D04FF4DD
:102B5800007B1960A3F804B0083312F4806F05D025
:102B68004FF4806B1960A3F804B0083312F4006FB7
:102B780005D04FF4006B1960A3F804B0083312F4C1
:102B8800805F05D04FF4805B1960A3F804B0083368
:102B980012F4005F05D04FF4005B1960A3F804B08D
:102BA800083312F4804F05D04FF4804B1960A3F816
:102BB80004B00833D20B04D04FF4004219609A8055
:102BC800083301F58061A1427FF47EAFBDE8F08F44
:102BD8006C4503083083002000180048002852D0B4
:102BE800036803F138422DE9F04F920A504DAA5C70
:102BF80002F01F0552090124022A04FA05F443D001
:102C0800032A00F09080012A43D001F003077A1EBE
:102C1800012AC1F3810CC1F300188088C1F3411166
:102C28003CD9C60700F18880850700F194804407E5
:102C380000F1A280020700F1B080C60600F1BE8054
:102C4800850600F1CC80440600F1DA80020600F126
:102C5800E880C60500F1F680850500F10481440589
:102C680000F11281020500F12081C60400F12E81D5
:102C7800850400F13C81440400F14A81020400F11A
:102C88005881BDE8F08F70472A4A95692C439461B2
:102C9800BBE7284A55692C435461B6E7002422460D
:102CA8004FF0010E4FF0030904E00132102A04F13D
:102CB8000204E6D00EFA02F636EA0005F5D1D3F89A
:102CC80008A009FA04F5ED430AEA050AC3F808A0C2
:102CD800D3F808B00CFA04FA4AEA0B0AC3F808A0B9
:102CE800B3F804A01FFA8AFA2AEA06069E80B3F807
:102CF80004A008FA02F646EA0A06B6B29E801E68E2
:102D08002E401E60D3F800A007FA04F646EA0A0629
:102D18001E60D3F80CA001FA04F605EA0A0A46EA8E
:102D28000A05DD60C1E7034AD5692C43D4616CE725
:102D380080450308001002401A6822F003021A6056
:102D48001A683A431A60DA6822F003020A438507D0
:102D5800DA607FF56CAF1A6822F00C021A601A6804
:102D680042EA87021A60DA6822F00C0242EA81021B
:102D78004407DA607FF55EAF1A6822F030021A6005
:102D88001A6842EA07121A60DA6822F0300242EA48
:102D98000112DA6002077FF550AF1A6822F0C0020C
:102DA8001A601A6842EA87121A60DA6822F0C002CA
:102DB80042EA8112C606DA607FF542AF1A6822F449
:102DC80040721A601A6842EA07221A60DA6822F426
:102DD800407242EA01228506DA607FF534AF1A684C
:102DE80022F440621A601A6842EA87221A60DA6896
:102DF80022F4406242EA81224406DA607FF526AF77
:102E08001A6822F440521A601A6842EA07321A60B5
:102E1800DA6822F4405242EA0132DA6002067FF5AB
:102E280018AF1A6822F440421A601A6842EA8732D8
:102E38001A60DA6822F4404242EA8132C605DA6052
:102E48007FF50AAF1A6822F440321A601A6842EA1B
:102E580007421A60DA6822F4403242EA01428505E4
:102E6800DA607FF5FCAE1A6822F440221A601A680C
:102E780042EA87421A60DA6822F4402242EA814232
:102E88004405DA607FF5EEAE1A6822F440121A6043
:102E98001A6842EA07521A60DA6822F4401242EAD3
:102EA8000152DA6002057FF5E0AE1A6822F44002AA
:102EB8001A601A6842EA87521A60DA6822F44002F5
:102EC80042EA8152C604DA607FF5D2AE1A6822F06F
:102ED80040721A601A6842EA07621A60DA6822F0D9
:102EE800407242EA01628504DA607FF5C4AE1A686E
:102EF80022F040621A601A6842EA87621A60DA6849
:102F080022F0406242EA81624404DA607FF5B6AE9C
:102F18001A6822F040521A601A6842EA07721A6068
:102F2800DA6822F0405242EA0172DA6002047FF560
:102F3800A8AE1A6822F040421A601A6842EA8777F7
:102F48001F60DA6822F0404242EA8171D960BDE828
:102F5800F08F00BF10B1036882881A85704700BFE0
:102F680010B1036882889A61704700BF38B10029A0
:102F78008388026814BF002110218B409361704739
:102F88000E4B1B8801463BB90D4B0E4A1B78106847
:102F98000BB981F00101E9E70B4B5A691AB118B96D
:102FA8001A68106058747047084A18681188084AE7
:102FB80092FBF1F201210260597470471445002018
:102FC80016450020184500201C45002034450020E7
:102FD80020A1070010B40A4B0A4A1C780123834039
:102FE800234052F8200029B9B3FA83F149095DF862
:102FF800044BBBE7191C18BF01215DF8044BB5E76A
:1030080006450020084500201C4C08B50121022077
:10301800FFF7E0FF237803F00502052A2AD003F022
:103028000903092B08D000210120FFF7D3FF002155
:103038000846FFF7CFFFFEE7114A124B11681A68DE
:103048000B68114C4FF6FE7003400B601388206824
:1030580023F001031B041B0C138018B12922002341
:103068008271C37102224E21FEF760FC2068FFF7CF
:1030780071FFD8E71AF0C2FD2378D0E7E42D0020CD
:10308800C4250020C82500206026002030B1036830
:1030980082881B8A1A4214BF01200020704700BF93
:1030A80038B5044690F84D0000285AD104F11805A7
:1030B800636D80226B21284698476420FFF72AFB1E
:1030C800636D07226821284698476420FFF722FB92
:1030D800636D00226B21284698476420FFF71AFB8E
:1030E800636D01226B21284698470F20FFF712FBDA
:1030F80094F84720636D022A8CBF1A2218221B21DC
:10310800284698470F20FFF705FB636D18221C21FE
:10311800284698470F20FFF7FDFA636D94F846207C
:103128001A21284698470F20FFF7F4FA636D94F8A0
:1031380048201921284698476420FFF7EBFA636D69
:1031480012223721284698470F20FFF7E3FA28462E
:10315800636D0122382198470F20BDE83840FFF7FA
:10316800D9BAFEF7B5FD0546FFF790FF00289DD1B7
:1031780015B12023E871AB7128460021FFF72EFD19
:103188002146054B41F8143F284623F02FFC2846DA
:1031980020F0D0F88AE700BFF90A00082DE9F041CD
:1031A8000B4E346873691C400FD0DFF82880012764
:1031B800B4FA84F3C3F11F0307FA03F558F82300A0
:1031C80003689847AC437561F2D1BDE8F08100BF50
:1031D80000040140486B00202DE9F0410B4E346893
:1031E80073691C400FD0DFF828800127B4FA84F3F4
:1031F800C3F11F0307FA03F558F82300036898473B
:10320800AC437561F2D1BDE8F08100BF0004014014
:10321800486B00202DE9F0410B4E346873691C405F
:103228000FD0DFF828800127B4FA84F3C3F11F0315
:1032380007FA03F558F8230003689847AC4375610B
:10324800F2D1BDE8F08100BF00040140486B0020C6
:103258002DE9F0410B4E346873691C400FD0DFF83C
:1032680028800127B4FA84F3C3F11F0307FA03F592
:1032780058F8230003689847AC437561F2D1BDE85C
:10328800F08100BF00040140486B00202DE9F041A7
:103298000B4E346873691C400FD0DFF82880012773
:1032A800B4FA84F3C3F11F0307FA03F558F82300AF
:1032B80003689847AC437561F2D1BDE8F08100BF5F
:1032C80000040140486B00202DE9F0410B4E3468A2
:1032D80073691C400FD0DFF828800127B4FA84F303
:1032E800C3F11F0307FA03F558F82300036898474A
:1032F800AC437561F2D1BDE8F08100BF0004014024
:10330800486B00202DE9F0410B4E346873691C406E
:103318000FD0DFF828800127B4FA84F3C3F11F0324
:1033280007FA03F558F8230003689847AC4375611A
:10333800F2D1BDE8F08100BF00040140486B0020D5
:10334800084A094808B5936943F0010393610021CD
:1033580040222FF00EF8054B4FF0FF321A60C3F8E9
:10336800032008BD00100240486B0020886B002035
:103378002DE9F041044618460D46164698462BF0AE
:1033880005FE2768E6722844A07229467D694346EF
:1033980032462046AC46BDE8F0416047036810B5A8
:1033A80004461B689847236820469B689847A37B78
:1033B8000133A37310BD00BF08B52120FEF788FCB8
:1033C8000C4B186018B1112200238271C37120219F
:1033D800FFF704FC2020FEF77BFC074B186018B1B0
:1033E800112200238271C3712021BDE80840FFF734
:1033F800F5BB00BFE82D0020EC2D0020427A02B971
:10340800704710B504460368406804F10A019847FC
:103418000023637210BD00BF437A5A1C0344D2B222
:1034280042729972037A934200D802B9704710B574
:1034380004460368406804F10A0198470023637250
:1034480010BD00BF30B40B4D002305F1800101E031
:10345800272B0CD011F8132082424FEA430403F1C2
:103468000103F5D12C4494F8810030BC704700204A
:1034780030BC7047E4240308064B07498B4202D34B
:103488000023184670471A88C2F30B029042F8D0FE
:103498001433F3E7787E0308B0820308024A1368FE
:1034A80023EA000010607047808D00202DE9F04766
:1034B800A84FA94E13F0F0FEBE421ED2DFF82083BB
:1034C800DFF820934446258862197DB14A450DD21C
:1034D800052D0BD933886188C3F30B03994200F09B
:1034E800D880144625886219002DEFD171683046BE
:1034F8001436FDF787FCBE42E4D3984A5378022B72
:1035080040F2EC8000239649537013789548022BBB
:10351800016000F2DF8003EBC301934A03EB8103F0
:1035280002EB4303914C1846236025F075F9904A45
:103538001378A3F1170102290FD98E4911F8330026
:10354800002840F0D180D8000144497829B18A493F
:1035580011F83330002B00F0F580884B9A78042A54
:1035680000F0E78032B91A88B2F5F07F84BF4FF4D3
:10357800F0721A808249834A0B681A40002A00F0C8
:10358800E480DE0700F1D0805D0400F1C8801807F0
:1035980000F1C0809A0100F1B7809B0400F1AD8072
:1035A80023689A8CD98C914224BF00229A84FDF713
:1035B800D5FE20F037FB10B9734821F0D9FA18F07E
:1035C800BDFF0021302271482EF0D3FE704B2668D3
:1035D80003F1500102E00433994279D01A78002AA5
:1035E800F9D19C78D8788442F5D26A496A4B91F827
:1035F80000E06A486A4D1C6B6A4B2860C827642142
:1036080011FB0E71DFF8E0E15960674F30F8041CD8
:10361800664DAEF8001000219960D96019615961B2
:103628009961D96183F8201083F821103A702E60CF
:103638000CB116F0B9F95E4B9FED5E5A1B885E4AD5
:103648009FED5E6A557D5E4C5E495F48086006EEF8
:10365800903AF8EEE66A138AC5EE265A07EE103A53
:10366800538A127DC4ED005A07EE903AB8EEC77A35
:10367800564BF8EEE77A1D725A7227EE067A67EE15
:10368800867ABDE8F04783ED017AC3ED007A13F03E
:10369800EBBD63799B077FF424AF716894F804A0AD
:1036A8003046FDF7AFFB3388BAEB133F0BD1738875
:1036B8007068AA1FC3F30B039A4204F10601A8BF5E
:1036C8001A462CF0D5FB1436BE42FFF4FBAE14E7C5
:1036D80001228AE700231370234B23E7204903EBD9
:1036E800430301EB830110E7D8000D186D68002D26
:1036F8007FF42AAF1725157026E73548FFF7CEFE69
:103708004020FFF7CBFE4BE746F20900FFF7C6FE65
:103718000B6842E72F48FFF7C1FE0B683AE72E48CF
:10372800FFF7BCFE0B6832E72C48FFF7B7FE0B68C3
:103738002AE71A8BB2F57A7FBFF41CAF4FF47A727E
:103748001A8317E71823137007E743F001030B6088
:1037580017E700BFB0820308787E03088E84002034
:10376800A884002048380020708C0020A484002001
:10377800F836002044460308D44203084C4500208C
:10378800808D002009600002D86F0020241F0020CF
:10379800FC36002000400020084200208834002029
:1037A800FC9200208441002037020020581F00208E
:1037B800EC1D0020C0C9FB48541D002017B7D138A4
:1037C800F01D0020C43800203661023DA0380020DA
:1037D800094000020160000209200002086000029E
:1037E80007F003080000040892340020F8B51A4DC9
:1037F8002B789F2B2ED16B78BE2B2BD10522174906
:10380800A81C2EF001FE28BB072229464FF6FF70A0
:10381800FCF76EFF124FEC1D22884AB1A618BE4273
:1038280018D2052A16D92146FCF762FF3446F3E779
:1038380021460222FCF75CFF0222A118FCF758FF80
:103848000634084B641B1C8041F60F53C31A5842B8
:103858005841F8BD0020F8BD00F00308274D0308C3
:1038680000000408982F00202DE9F04FDFF854914C
:103878004F4F8DB00326A7EB090718220DEB020066
:1038880000212EF076FD4B4BCDF8189007971A695A
:10389800120604D5484A5A6002F188325A60012259
:1038A8008DF82C203422DA60444B454C18689A88ED
:1038B80004909B79ADF8142004A9072206A88DF876
:1038C8001630FDF75BFC072204A94FF6FF70FCF7E2
:1038D8000FFFDFF8F4B080464FF0000A5C4536D39E
:1038E8000CAC002524F82C5D0222214606A8FDF721
:1038F80045FC022221464046FCF7FAFE40BAC04386
:10390800ADF80800022202A906A8FDF737FC0998BD
:1039180060B108ABC0F10402294618442EF029FD15
:10392800089906A8FDF7D0FB09950A909DF82C3058
:103938000A9A23B11F490B6943F080030B61013ECA
:103948002DD0002A99D1FFF751FF50B32CE065889C
:103958008DF80DA0C5F30B05AA1DADF80820228827
:10396800C2F30B01120BADF80A108DF80C2002A956
:10397800062206A8FDF702FC062202A94046FCF72B
:10398800B7FE616880462A4606A8FDF7F7FB61681E
:1039980040462A46FCF7ACFE143480469EE7002ACF
:1039A800D1D00520FEF7BAFB0DB0BDE8F08F00BFFF
:1039B800000004080020024023016745B2250308DF
:1039C800787E030800F00308B082030808B513F0F6
:1039D80063FCFFF749FF13F047FCFFF767FD012081
:1039E800BDE8084021F060BF08B5FDF74DFD13F0B4
:1039F80053FCFFF739FFBDE8084013F035BC00BFA2
:103A080008B513F049FCFFF72FFFBDE8084013F095
:103A18002BBC00BF0378202B024600F10100F9D02F
:103A2800092BF7D02D2B2CD02B2B03BF5378B7EEB7
:103A3800000A0246B7EE000AA3F13001C8B209280D
:103A48009FED467A10D8F2EE046A07EE901AF8EE67
:103A5800E77A12F8013FE7EE267AA3F13001C8B2FF
:103A68000928B0EE677AF0D92E2B4CD003F0DF038B
:103A7800452B0BD0F7EE007A67EE276A20EE260A70
:103A880070475378BFEE000A0246D5E710B4517864
:103A98002D2959D02B290ABF9178501C901C00243D
:103AA800A1F13003092B53D8002303EB830301EB67
:103AB800430310F8011FA1F13002092AA3F13003D2
:103AC800F3D9B3F59A7F28BF4FF49A73072B42D9DD
:103AD800DFED236A1A46F7EE007A083A072A67EEFE
:103AE800A67AFAD803F007032BB1F2EE046A013B79
:103AF80067EEA67AFBD124B3C7EE276A5DF8044BBC
:103B080020EE260A70475378A3F13001C8B209287D
:103B180002F10102AAD8F2EE046AF0EE665A07EE44
:103B2800901AF8EEE77A12F8013F87EEA66AA3F139
:103B38003001C8B2092866EEA56A37EE067AEED9D2
:103B480094E767EE276AD9E7901C91780124A7E7E4
:103B5800F7EE007ACFE7F7EE007AC5E7000000003D
:103B680020BCBE4CB5EEC00ADFED317AF1EE10FA9A
:103B7800CCBF30EE270A30EE670ADFED2E7A20EE52
:103B8800270A30B5FDEEC07A87B017EE904A054691
:103B980084EAE470002303A9A0EBE4700193009386
:103BA800029320F0E7FC002CACBF20232D2303A8B0
:103BB8008DF800302BF0EAF9012803A924D0022857
:103BC8002DD0032805BF3023684668468DF801309C
:103BD8002EF0F5FB68462BF0D9F90338C4B222461B
:103BE800694628462EF049FC00232B5528462BF021
:103BF800CDF92E22431C2A540DEB0401E8182EF0AF
:103C0800FBFB284607B030BD302368468DF80130ED
:103C18008DF802308DF803302EF0D1FBDAE730232F
:103C280068468DF801308DF802302EF0C8FBD1E7D8
:103C38006F12033A00007A442DE9F0410646154612
:103C48000846B6FBF2F43CB905FB1464124B1B5D45
:103C580000F8013BBDE8F081B4FBF2F767B90E4B01
:103C680005FB174705FB1464DA5D00F8012B1B5DA3
:103C780000F8013BBDE8F081B7FBF2F8B8F1000F9E
:103C880002D04046FFF7D8FF05FB1878024B13F81F
:103C9800082000F8012BE3E72C4D030830B4026834
:103CA8001146531C036011F8024B0160D31C517874
:103CB80003609378151D05601B0443EA0123D0783F
:103CC800234343EA006030BC704700BF0368591CB7
:103CD8001A46016012F8021B0260587841EA002077
:103CE800704700BF38B50446006815462CF0C0F888
:103CF80022682A44226038BD036810B40A0A5C1C92
:103D080004601A7003685A1C026019705DF8044B4D
:103D1800704700BF03685A1C026010B4197003682A
:103D28000A0A5C1C04601A7003680A0C5C1C0460B4
:103D38001A700368090E5A1C026019705DF8044B6A
:103D4800704700BF03685A1C026019700368090AAB
:103D58005A1C0260197070472DE9F047002488B09A
:103D680080460F461E46A14605AD531C03931178A5
:103D780039B3252933D1931CCDF81090039350788B
:103D880030284ED04FF0000AA0F13003DBB2092BE7
:103D980042D96C2819D0642800F0938024D82528AB
:103DA8001CD063D9582876D063281BD13178404677
:103DB800B847039A531C0393117804360134002939
:103DC800D7D1204608B0BDE8F087039B5A1C039260
:103DD8001B78642B7CD02AD8252B54D1252140462A
:103DE8000134B847039AC0E7732833D044D97528FB
:103DF8004FD106F1040E30682B4600220A21764680
:103E0800FCF7FAFB049A0095534639464046FCF7FE
:103E180031FC039A0444A8E704AA03A920F086FB0E
:103E2800B7E7D31C039390784FF0010AACE7732BE4
:103E380010D05BD9752B3AD0782B96D1A3F15802C4
:103E4800B2FA82F2306852092B4610210436FCF788
:103E5800D3FBD7E73368049A0093394600234046DA
:103E6800FCF708FC04360444039A7EE70028B9D11D
:103E7800204608B0BDE8F0876E28B3D1039A3368AE
:103E880004361C6071E72AD9582BD7D0632B8DD004
:103E98006BE77828A6D1A0F15802B2FA82F230680E
:103EA80052092B461021FCF7A7FB0436AAE706F1B6
:103EB800040E30682B4600220A217646FCF79CFB4C
:103EC800A0E7331D306829461E46FCF767FB99E7D3
:103ED800331D306829461E46FCF760FB92E7002B2D
:103EE8007FF443AF204608B0BDE8F0876E2BC6D0FC
:103EF8003BE700BF0EB400B584B005AB019053F8A2
:103F0800042B0649039301A8FFF726FF019B002213
:103F18001A7004B05DF804EB03B07047710600082E
:103F28000FB430B583B006AB0B490C4853F8042BDB
:103F3800096800680193FFF70FFF094C05462068E0
:103F480003685B6998470028F9D0284603B0BDE8A4
:103F5800304004B0704700BFDC2D0020E02D002069
:103F6800601F0020DFED2B7AB4EEE70AF1EE10FABD
:103F78004ADDDFED296A9FED297A01E0B0EE670A94
:103F8800B4EEC70AF1EE10FA70EE667AF6DC9FED31
:103F9800247AF4EEC77AF1EE10FA38D5DFED1E6A0E
:103FA8009FED207A01E0F0EE407AF4EEC77AF1EE68
:103FB80010FA37EEA60AF6D4DFED1B7AB4EEE70A5C
:103FC800F1EE10FA14DDDFED137A37EEC00A60EE79
:103FD800006A9FED166A9FED167ADFED167AA6EE57
:103FE800867A20EE266AE6EE877AA6EE270A7047DA
:103FF800DFED117AB4EEE70AF1EE10FA44BFDFED17
:10400800087A37EEC00AE2E7F0EE407ABFE7B0EE92
:10401800670AD1E7DB0F4940DB0FC940E4CB164103
:10402800DB0F49C0E4CB16C1DB0FC93F92E741B9AA
:104038009730083C15A82ABEDB0FC9BF41404A008B
:1040480011F0800F82F0D503D2B2DBB208BF13465D
:10405800590013F0800F81F0D502C9B2D2B208BF5F
:104068000A46510012F0800F81F0D503C9B2DBB2C5
:1040780008BF0B46590013F0800F81F0D502C9B272
:10408800D2B208BF0A46510012F0800F81F0D50362
:10409800C9B2DBB208BF0B46590013F0800F81F09C
:1040A800D502C9B2D2B208BF0A46510012F0800F39
:1040B80081F0D503C9B2DBB208BF0B465A0082F0C3
:1040C800D50013F0800FD2B2C0B208BF10467047B7
:1040D80080EAE073A3EBE0738B4205DB002801DD87
:1040E800401A704702D17047002070470844704753
:1040F80009B909E0194690FBF1F301FB13030846DF
:10410800002BF7D1084670470146FBE710B507EECC
:10411800901A2DED028BB8EE678ADFED227A28EE31
:10412800008A044628EE278AB0EE480A2CF060F888
:10413800F0EE408AB0EE480A2BF0BCFFF7EE007AAA
:104148009FED197AF0EE675AE8EE875A0023A361CB
:10415800B0EE676AC7EEA56A63612362E361A36292
:104168006362A8EEC76ABDEC028B77EEC07AB6EE42
:10417800007AF8EE005A27EE877A20EE250A27EE15
:10418800267A26EE266A67EEA67A20EE260A84EDBF
:10419800046AC4ED017A84ED007A84ED027A84ED34
:1041A800030A10BD27D4D236F304353F4B0901F07A
:1041B8001F0150F82320012303FA01F1114214BF13
:1041C80018460020704700BFF0B5484B48491A68A8
:1041D800096883B00123560200935CBF03F1805342
:1041E8000093D4005CBF43F010030093880744BFDA
:1041F80043F0C60300934F0744BF43F008030093FE
:104208000E073C4948BF43F02003097848BF009394
:10421800D40548BF43F0006301F0EF0048BF0093A6
:1042280008286D4655D00E2953D0D0033248009B3C
:1042380000784CBF43F4204343F40053D7044CBFE9
:1042480043F0C84343F0884300280CBF07200F20E1
:10425800960648BF43F48073540748BF43F40033BD
:1042680043F400245205009402D5244A1279A2BBD3
:10427800182936D001900027012639462846FCB275
:10428800FFF794FF60B11E4B002203F5D87103E0DD
:104298008B420FD013F80C2CA24203F10C03F7D178
:1042A8000137242FE9D195E80300164B83E8030072
:1042B80003B0F0BD7A0904F01F0455F8223006FA5D
:1042C80004F4013723EA0404242F45F82240D4D10A
:1042D800E9E743F480530093A7E743F4C01300933E
:1042E800C6E7009B43F060730093C3E77C4A002055
:1042F800B47C0020F836002074450020E8850020B2
:104308002C260308B01D00202DE9F84F4E014FF070
:10431800000B174D8146904606F120075C4659462A
:1043280028465FFA8BFAFFF741FFC0B1A64215D8BD
:10433800A74213D900200F4A014604E0013124297D
:1043480014D012F80C0C504502F10C02F6D10A4BAD
:1043580001EB410103EB81014846C04701340BF1F1
:10436800010BBBF1240FDAD1BDE8F88F0021F3E788
:10437800B01D00202C26030820260308B0F1FF3FBB
:104388000AD0022810B403DC5DF8044BFCF7BABC71
:1043980000205DF8044B7047002070472DE9F0437A
:1043A800322083B0FEF7B6F90022104611231E21F1
:1043B800FFF7E4FF602301221E210020FFF7DEFF44
:1043C8006420FEF7A7F96846FCF7F2FE0024DFF840
:1043D8008C81254626460A27012302221E21002019
:1043E800FFF7CCFF3220FEF795F96846FCF7E0FEB0
:1043F800BDF900E0BDF90210BDF904208E457346F1
:10440800A8BF0B469342A8BF134643454FF001008F
:1044180076440D441444C0F29180FEF733FB013F0B
:10442800DAD14FF001090022104612231E21FFF7AE
:10443800A5FFDFF828810A27012302221E21002078
:10444800FFF79CFF3220FEF765F96846FCF7B0FEDF
:10445800BDF900E0BDF90210BDF904208E45734690
:10446800A8BF0B469342A8BF134643454FF001002F
:10447800A6EB0E06A5EB0105A4EB02045BDBFEF739
:1044880001FB013FD8D107EE906AF8EEE76A07EE24
:10449800905AB8EEE77A07EE904ADFED2A5A9FED78
:1044A8002A5A2A4EF8EEE77A85EEA66A00221046C6
:1044B80070231E21C5EE876A85EE277AB0EEC66A9C
:1044C800F0EEE66AF0EEC77A86ED006AC6ED016A9C
:1044D800C6ED027AFFF752FF202301221E21002099
:1044E800FFF74CFF0023184602221E21FFF746FF64
:1044F8006420FEF70FF9B9F1000F04D14FF07E5395
:1045080033607360B360124C206810B1FEF7BEFDD3
:1045180018B9012003B0BDE8F0830E490E4B41F8ED
:10452800183F206822F062FA20681EF003FF01207D
:1045380003B0BDE8F0834FF00009A4E74FF000098D
:1045480071E700BF00406F4601C05E4600000020D2
:1045580070370020541D0020C108000801F0FFFF3B
:10456800F0B585B005460DF10703012202210C20A4
:104578001EF0D4F918B19DF80730DB0703D40024E6
:10458800204605B0F0BD02AB062203210C201EF028
:10459800C5F90DF10703012209210C201EF0BEF90F
:1045A80004460028EBD09DF8070010F00C00E6D177
:1045B8009DF809E09DF808109DF80B709DF80A20F9
:1045C8009DF80D609DF80C3041EA0E2142EA072261
:1045D80043EA0623C1EB8131C2EB8232C3EB83335A
:1045E800890092009B0029806A80AB800A220123FF
:1045F8000C21FFF7C3FEC3E700B5002383B01846BC
:104608000A220C21FFF7BAFE1420FEF783F80F23C5
:104618000A220C210020FFF7B1FE0A20FEF77AF8E3
:1046280001AB032210210C201EF078F90A20FEF7B6
:1046380071F8002318460A220C21FFF79FFE0A2072
:10464800FEF768F80DF10303012202210C201EF089
:1046580065F90DF10303012209210C201EF05EF912
:1046680001230A220C210020FFF788FE012003B055
:104678005DF804FB3123F422762100207EE600BF9A
:10468800F0B5574B574A97B01968914200AF00F000
:104698009C805549554A00234FF47000C1F88800A2
:1046A8003B607B60136843F48033136003E03B682E
:1046B800B3F5A04F09D0136803F400337B603B685F
:1046C80001333B607B68002BF1D0484B1B6813F427
:1046D800003318BF01237B607B68012B4BD0424D10
:1046E800424B434AEA60434A596A11605A6A424E49
:1046F80042F080725A625A6907F1580442F4FC0287
:1047080041F6FF715A6124F8501D032321464FF0EA
:104718009040BB72FCF7C8FA4FF6FF732146374842
:104728003B81FCF7C1FA21463548FCF7BDFA214622
:104738003448FCF7B9FA21463348FCF7B5FA214664
:104748003248FCF7B1FA20461CF0E0FCBB6830495F
:10475800304AA1FB031330499B0CF02400204FF092
:10476800070E5C370B60566085F823409060C2F8EE
:1047780000E0BD46F0BD294A1C4B122111605A6861
:104788005A605A685A605A6842F480625A605A6895
:1047980022F47C125A605A6842F4E8125A601A6885
:1047A80042F080721A601A689201FCD559680F4A63
:1047B80021F003015960596841F0020159605368BA
:1047C80003F00C03082BFAD189E700221A6062B6BD
:1047D800134B1B6883F30888124B1B689847FEE746
:1047E800FC9F0020EFBEADDE00ED00E000100240AF
:1047F8000005FA05784A00203F1901000004004826
:1048080000080048000C0048001000480014004848
:1048180083DE1B4310E000E04045002000200240FA
:1048280000D8FF1F04D8FF1F064A002351688142A1
:1048380002F11C0204D001330C2BF7D10020704781
:10484800D8B270476400002070B50F4C0F4DC0EB14
:10485800C00004EB8004686926693043686182B04F
:104868009209667BA1600025012101A863618DF88A
:1048780004608DF805208DF806508DF807101EF09D
:104888003DF902B070BD00BF640000200010024076
:10489800074BC0EBC00030B403EB8000054C056942
:1048A80063692B4363610176427630BC704700BF71
:1048B80064000020001002402DE9F04F554C54F8D8
:1048C800204083B0002C60D0656D1F469046524B47
:1048D8006A682265A160236004F15A014FF480736D
:1048E80004F5AD726161A261E36023610646287E2A
:1048F8001DF084FEE86858B1FFF796FF721CD2B22B
:104908000C21FFF7C5FF236DEA6822632433E364B3
:10491800A86890B1FFF788FF721C8146D2B20B21BC
:10492800FFF7B6FF2346EA7E3C494846FFF78CFF6F
:10493800236DAA6862632833A36494F85900FDF7CD
:10494800C7F9814694F85800FDF7C2F93A0782463C
:1049580095F819B01DD5B9F1000F1AD017F0110F3D
:104968004FF00B0306F1010614BF4E213E2189F8D2
:10497800063089F807605A464846FCF7D7FFFB0718
:1049880043D5236B6BB3636B5BB3204603B0BDE8C1
:10499800F08F17F0010F0CBF2E274E2718F0020FCB
:1049A8000DD0B9F1000F0AD00B22731C89F806202C
:1049B80089F8073048465A463946FCF7B7FF18F0D9
:1049C800010FDED0BAF1000FDBD001360C238AF8D4
:1049D80007605A4639468AF806305046FCF7A6FF63
:1049E800CFE72B7FAA7E8DF804209B0900210122A6
:1049F80001A88DF805308DF806108DF807201EF0F7
:104A08007DF8204603B0BDE8F08F4846FEF7A2FACD
:104A1800B7E700BFF02D0020BC250308B10B000844
:104A28000348D0F83C3113B100F59A701847704725
:104A3800640000200348D0F8203113B100F58C70D1
:104A480018477047640000200348D0F804310BB1C0
:104A5800FC301847704700BF640000200348D0F8B6
:104A6800E8300BB1E0301847704700BF6400002001
:104A78000348D0F8CC300BB1C4301847704700BF9A
:104A8800640000200348D0F8B0300BB1A8301847B4
:104A9800704700BF640000200348D0F894300BB181
:104AA8008C301847704700BF640000200248836FAD
:104AB8000BB1703018477047640000200248C36D7E
:104AC8000BB1543018477047640000200248036C4B
:104AD8000BB1383018477047640000200248436A19
:104AE8000BB11C30184770476400002002488368E7
:104AF80003B11847704700BF640000201749184BDE
:104B0800184A194810B4D1F8884044F47004C1F820
:104B180088401C6844F001041C605C6822405A60AC
:104B28001A6822F0847222F480321A601A6822F419
:104B380080221A605A6822F4FE025A60DA6A22F069
:104B48000F02DA621A6B002410404FF000621863FB
:104B58009C608A605DF8044B704700BF00ED00E080
:104B6800001002400CC07FF8CCFC00FF2DE9F04F8C
:104B7800B0F908502DED048B0D81EDB2382D8FB0B2
:104B88000C4600F08C82804691462ED9802D00F08C
:104B9800908079D8522D00F0E78040F23482542D6D
:104BA80000F0D4826E2D40F011817D4B0A681B887D
:104BB8007C4DFF2BA8BFFF23511C21601370A968EF
:104BC80081F3100189B22046FFF7BCF8764B2046E6
:104BD8001988FFF7B7F8296801F30F0189B2204651
:104BE800FFF7B0F801252B4647E0042D00F0A2821C
:104BF80040F2F181202D00F09B8040F20F82242D9D
:104C080000F09282282D40F0E1800B68DFF8B8812F
:104C1800664E591C022221601A70236806275A1C06
:104C280022601F7023680A22591C21601A702368A9
:104C380001255A1922601D70B8F800102046FFF7A8
:104C480081F8B8F802102046FFF77CF823685A1953
:104C580022601F7023685022591921601A70236836
:104C68000022591921601A7031882046FFF76AF826
:104C780071882046FFF766F82B46284663810FB0F7
:104C8800BDEC048BBDE8F08F822D24D0C0F0768275
:104C9800A02D00F06782FE2D40F09880444D05F16C
:104CA800080635F8021B2046FFF74CF8AE42F8D14B
:104CB80098E70B683F4A581C0A211288206019702F
:104CC8002168FF2A01F10103A8BFFF220125236003
:104CD8002B460A70D1E70B68374A324D1178374AAC
:104CE800581C20601970D1882046FFF72BF82C4BF0
:104CF80022681B88FF2B02F10101A8BFFF23216056
:104D08001370A96881F3100189B22046FFF71AF8D9
:104D1800296801F30F0189B22046FFF713F8284BE1
:104D280022681978531C012523602B461170A4E7CB
:104D38000B68224D591C6A7821601A7023682A78FA
:104D4800591C21601A702368AA78591C21601A70AE
:104D5800E9882046FEF7F6FF23682A79591C216066
:104D68001A7022686979DDE70A68164E531C032118
:104D7800236006F10C0711703346062001212268D2
:104D8800551C256011702268BB4202F101012160A7
:104D9800107000F0AA819979D8790633EFE700BF3F
:104DA800CC850020D0850020704100200C260020F2
:104DB800E44100201C260020F685002078410020D0
:104DC80073410020F42A0308501E0020A5F10A03AD
:104DD800E72B00F2EA80DFE813F0CA02E800E800F7
:104DE800E800E800E800E800E800E800E800E8007B
:104DF800E800E800E800E800E800E800E800E8006B
:104E0800E800E800E800E800E800CA04E800E80074
:104E1800E800B904E800E800E8009105E80020058A
:104E2800E8000705E800FB04E800D505E800AF0541
:104E3800E800DA05E800E800E800C302A605E80093
:104E48009F05E800E8009605E800E800E800E800AB
:104E5800E800B602E800E800E800E8007607E800A5
:104E68005407E8002D071507E800E800E800E80007
:104E7800E800E800E8009106E8006606E800370662
:104E8800E800ED05E800C507E800E800E800E800EC
:104E9800D5069207B00488047604E800E8005D04AB
:104EA8004F04E800EB03A903E800E800E800E80085
:104EB8009D03E800E8007B03E800E800E8003E0402
:104EC80025046B032D03E800E800E8001D03E80053
:104ED8001203E800E800E800E800E800E800E8005D
:104EE800E800E800E800E800E800E800E800E8007A
:104EF800E800D506E800E800E800E800E800E80077
:104F0800E800E800E800E800E800E800E800E80059
:104F1800E800E800E800E800E800E800E800E80049
:104F2800E800E800E800E800E800E800E800E80039
:104F3800E800E800E800E800E800E800E800E80029
:104F4800E800E800E800E800E800E800E800E80019
:104F5800E800E800E800E800E800E800E800E80009
:104F6800E800E800E800E800E800E800E800E800F9
:104F7800E800E800E800E800E800E800E800E800E9
:104F8800E800E800E800E800E800E800E800E800D9
:104F9800E800E800E800E800E800E800E800E800C9
:104FA800E800E800E8000603DB02742D00F03A810F
:104FB800772D48D1D8F80030D8F804209A421EBF7F
:104FC8005A1CC8F8002019789F4A08BF00212046BB
:104FD800FFF79AF906E6022D00F01C8100F209811C
:104FE800012D7FF4F3AE0B680022591C21601A7062
:104FF80023685A1C22601D7022682421531C2360D8
:105008002B46117039E6442D7FF4E0AE002A3FF4B8
:10501800E9AD8E4B136001252B462EE6052D7FF456
:10502800D5AE0B228A492046FEF75CFE0822894944
:105038002046FEF757FE0125072287492046FEF73E
:1050480051FE2B4619E6F52D00F0208198E848001E
:10505800292DA6EB030601F0498640F2B486392DC6
:1050680000F0DA86532D40F00F875A1CC8F800204C
:105078001978721E0329D2B20DD84B1EDBB2774DB8
:10508800774803EB430305EB430301705B7811B1E9
:105098009A4201F0B2874FF0FF352B46EDE50B68D9
:1050A800704901255A1C22601D7023680522581971
:1050B80020601A7023680A22581920601A70236821
:1050C8000022581920601A7023680A78581920603D
:1050D8001A7023684A78581920601A7022688978EB
:1050E800531923602B461170C7E55D4B21681A7868
:1050F800481C20600A70002A3FF474AD013AD2B20D
:1051080002EB420206EB42025278002A3FF46AADF3
:105118000132D5180133226813F8011F501C9D4233
:1051280020601170F7D15DE54F4B19682046FEF7F6
:10513800F1FD57E52A464D492046FEF7D3FD0021EB
:105148002046FEF7FFFD22680021EBE50B680021F1
:105158005A1C2260197022680125531923602B46B6
:1051680011708AE5424B08461968FEF7D3FD414B9A
:1051780020461968FEF7CEFD3F4BD6E73F4A404E22
:105188009368116803EB83034FF6FF725B00934249
:10519800A8BF13469142A8BF114623EAE37321EA48
:1051A800E1719DB289B20A22002713E0B368316821
:1051B80003EB83034FF6FF725B009342A8BF1346CD
:1051C8009142A8BF114623EAE37321EAE1719DB237
:1051D80089B250222368581C206020461A70FEF7B6
:1051E800B1FD013729462046FEF7ACFD022FDDD17F
:1051F800F8E40B680222591C21601A702368012503
:105208005A1922601D7022680021531923602B4609
:10521800117032E504221B4920460125FEF762FD84
:105228002B462AE5D8F80030D8F804209A421EBF49
:105238005A1CC8F800201978134A08BF00212046D4
:10524800FFF762F8CEE400BF890100087D0E000870
:10525800644D0308704D03087C4D0308F42A0308C5
:10526800DC6C00205F8C0020808D00205C4D0308E2
:10527800ACF7FF1FB0F7FF1FB4F7FF1FD0250020C2
:1052880010260020544D0308550E0008D8F80030A9
:10529800D8F804209A4241F01D86B34BFF221A72B7
:1052A8004FF00008B14D15F011FE41463022B048CC
:1052B80085F800802DF05DF88DF814809DF8143085
:1052C8000B2B01F2F086AB4FA94E42469DF81430E5
:1052D80003EB430307EBC3035B7CE3B19DF8143096
:1052E80003EB430307EBC3035B69A3B19DF81430D9
:1052F80003EB430307EBC3032021586946F8220058
:10530800FDF76CFC2B7856F82300FDF729FE2A7868
:105318000132D2B22A709DF814300133DBB28DF815
:1053280014309DF814300B2BD0D92368591C2160F8
:105338001A70B9F1000F3FF455AC8F4BC9F8003023
:1053480001252B4699E4236800255A1C226029462A
:1053580020461D70FEF7DEFC29462046FEF7DAFCE3
:10536800002120460125FEF7D5FC2B4685E483481D
:1053780029F00CFE00287FF735AC804B1D182268F9
:1053880013F8011B501CAB4220601170F7D129E4BF
:105398007B4B03F1700522681978501C206011704E
:1053A80022685978501C2060117022689978501C26
:1053B800206011702268D978501C20601170226812
:1053C8001979501C2060117022685979501C20608E
:1053D8001170226899790733501C9D422060117022
:1053E800D9D1FFF7FFBB674D2046A989FEF7AAFC74
:1053F800698920460125FEF7A5FC2B463DE4624B52
:105408006249B3F9003081FB0321DB17C3EBA1012B
:10541800FFF7E4BB5E4D2046A98AFEF793FCE98AB4
:105428002046FEF78FFC298B20460125FEF78AFCD3
:105438002B4622E4DFF874E10027FEB27146002310
:105448002268501C206016702268501C206013705F
:10545800226811F8010F0133551C062B25601070C6
:10546800EED10137062F0EF1060EE6D14949002389
:105478002268501C206017702268501C206013702E
:10548800226811F8010F0133551C0B2B2560107091
:10549800EED123684049581C072220601A702368FF
:1054A8000022581C20601A70226891F8F01039E424
:1054B80023683A4A34491078324A5D1C25601870CE
:1054C80023689278581C20601A702268897829E429
:1054D800334D05F16006A9882046FEF733FCE988BC
:1054E8002046FEF72FFC29892046FEF72BFC23686F
:1054F800AA7A591C21601A702368EA7A591C21601B
:105508001A7055F80C1B2046FEF704FCB542E2D190
:10551800FFF768BB234952232268501C2060137090
:1055280011F8013F002BF7D1FFF75CBB1E4D00239C
:105538002268286803EB4301561C405C2660107003
:105548002A6820680A44461C5278266002702A6835
:1055580020680A4401339278411C0A2B21600270AA
:10556800E6D1FFF73FBB00BFB01D0020B97800208F
:1055780024320020408100202580020892840020E7
:105588001C7A002084340020643700206766666631
:105598004C4500204F4100206C4000200C7000203A
:1055A800E47B0020E4250308A48400202B4100208C
:1055B800BA4D23682A68591C127821601A702B6822
:1055C80022689978531C2360002311702A68216887
:1055D8001A4401335279481C032B20600A70F5D114
:1055E80023682A68591C127A21601A7023682A686D
:1055F800591CD27821601A7023682A68591C1279BC
:1056080021601A702B6820465989FEF79BFB236896
:105618002A68591C527A21601A702B6822685978B6
:10562800FFF780BB22689E4B9E491878551C256061
:10563800107022685878551C2560107022689B7875
:10564800501C20601370C98820460125FEF77AFB9C
:105658002B46FFF712BB934D20462988FEF772FBB5
:1056680069882046FEF76EFBA98820460125FEF7CB
:1056780069FB2B46FFF701BB8B4B20461968FEF7E9
:1056880049FB8A4B204619880125FEF75BFB2B4610
:10569800FFF7F3BA864D20462988FEF753FB698841
:1056A8002046FEF74FFBB5F904308249DA1781FB33
:1056B8000313C2EBA30399B220460125FEF742FB70
:1056C8002B46FFF7DABA7C4E3378002B3FF48AAAD0
:1056D8007A4F002537F8021F2046FEF733FB337850
:1056E80001359D42F6DBFFF77DBA754D754EDFF843
:1056F8000482DFF80492DFED748ADFED749A9FED7F
:10570800749A05F1200708E020460435FEF71AFBD5
:10571800BD4206F118063FF465AA717C0029F3D052
:1057280095ED008AB0EE480A2AF016FD98F8003088
:10573800002B41F09B8381B2E6E7102265492046A1
:105748000125FEF7CFFA2B46FFF797BA624D2046A0
:105758002988FEF7F7FAA9882046FEF7F3FA29897F
:1057680020460125FEF7EEFA2B46FFF786BA5B4D79
:105778005B4F05F15006002128785A4A0B4607E08E
:105788000133242B02F10C0200F0FD8212F80C1CEC
:105798008842F5D103EB4303226807EB8303511CCE
:1057A80093F844302160137023686A78591C21608B
:1057B8001A702368AA78591C21601A702368EA783D
:1057C8000435591CB54221601A70D4D1FFF70ABAC2
:1057D800454D05F1800655F8041F2046FEF79AFA54
:1057E800B542F8D1FFF7FEB9404D05F14006B5F8CE
:1057F80080102046FEF7A6FA236895F88220591CE7
:1058080021601A70236895F883200435591CB54225
:1058180021601A70EBD1FFF7E5B9354D23682A7A74
:10582800591C21601A70A98B2046FEF78BFA298B28
:105838002046FEF787FA698B2046FEF783FA23682D
:10584800EA7C591C21601A70E98C2046FEF77AFA26
:10585800298D2046FEF776FA2368AA7F591C216015
:105868001A70236895F82020591C21601A70A98C99
:105878002046FEF767FA2368EA7A591C21601A70F5
:10588800E9682046FEF746FA23682A7C591C2160FD
:105898001A70226895F82110FFF744BA483800209A
:1058A800C01D0020E83F0020E01D0020142100203A
:1058B8005C42002067666666CC8400203A8B002034
:1058C80054340020408100200000404200407444CD
:1058D80000E0824444340020182E0020FC360020CA
:1058E800E42503082C260308684000206C400020AB
:1058F8004C4A0020744500207C4A0020B64B2268A0
:105908001978FFF70FBA0822B44920460125FEF797
:10591800E9F92B46FFF7B1B92268B14B501C9978C9
:10592800206011707AE622680121531823600D4621
:105938000B461170FFF7A1B9AA4B03F15A0522686B
:105948005979501C2060117022681978501C206009
:10595800117022685978501C20601170226899785B
:10596800501C206011702268D978501C206011707A
:10597800226819790633501C9D4220601170DED1CF
:10598800FFF730B9954B2268597DFFF7CBB9964D93
:10599800964E05F1300795F902100023F2568A4217
:1059A80000F0F4810C33482BF8D10835BD42F2D110
:1059B800FFF718B900212046FEF7C4F90021204658
:1059C800FEF7C0F900212046FEF7BCF92268884D91
:1059D8000023511C2160137022682968501C91F81B
:1059E8002F102060117022682968501C91F83A1015
:1059F8002060117022682968501C91F83B102060C3
:105A080011702268511C216013702268511C21609A
:105A180013702268511C216013702B682046D98F9F
:105A2800FEF790F92B682046998FFEF78BF92368CB
:105A38002A68591C92F8312021601A702B68226854
:105A480093F83210FFF76EB96A4D23686A79684E89
:105A5800591C21601A7033682046198CFEF772F9B8
:105A680033682046598CFEF76DF969892046FEF7A0
:105A780069F9A9892046FEF765F933682046998CAB
:105A8800FEF760F933682046D98CFEF75BF9E9899F
:105A98002046FEF757F9298A20460125FEF752F9D4
:105AA8002B46FFF7EAB8534EF378002B01F0D1816B
:105AB80023680822591C21601A702368012299184A
:105AC80021601A7023684C4D591C2A7921601A707C
:105AD8002368AA78591C21601A7029882046FEF785
:105AE80031F9698A2046FEF72DF92368F279591CA5
:105AF80021601A702268E978FFF714B924F09EFA39
:105B0800FF28064601F012820EA9002501F82E5D35
:105B18000DF109008DF8095024F070FA0EA800F86C
:105B28002D5D24F05FFA0EA800F82C5D24F04EFAE3
:105B38000EA820F8245D24F03DFA23685A1C226040
:105B48001E7023689DF80920591C21601A7023686B
:105B58009DF80A20591C21601A7023689DF80B20B3
:105B6800591C21601A7023689DF80C20591C21606B
:105B78001A70BDF8141020460125FEF7E3F82B46ED
:105B8800FFF77BB80DF1140900220592DFF870A029
:105B98001A4B03920492C9F80420904601214FF64B
:105BA800FF7B07E008F10108B8F10B0F01F0B680A0
:105BB8001AF9011F4E1CF5D04BFA08F2D007F1D59F
:105BC8001A8842FA08F2D207ECD548460193FBF747
:105BD80065FB019BE6E700BFF83600204C4A002031
:105BE800541E0020F0380020D86F0020E049002023
:105BF800A48400200C7000204C450020D8410020CF
:105C0800142603082268914B0125511C2160157048
:105C180022689978501920601170226819785019F3
:105C28002060117022685978531923602B4611702F
:105C3800FFF723B82368864D01269A1922601E7043
:105C48001CF0DAF8002841F03C81824B2268511C94
:105C580021601070226841F2B410511C185C216058
:105C680041F27811107059582046890AFEF752F807
:105C7800E96B204649080125FEF74CF82B46FEF74C
:105C8800FCBF754E3378002B3EF4ACAF734F002544
:105C9800B846236817F81520591C21601A7098F81F
:105CA800011001EB810101EB810101F2EE2189B2C2
:105CB8002046FEF747F8337801359D4208F102087F
:105CC800E7DBFEF78FBF2368654D591C2A782160F2
:105CD8001A7023686A78591C21601A7069882046EE
:105CE800FEF730F823682A79591C21601A70E98870
:105CF8002046FEF727F82268297AFFF713B8594E8D
:105D0800338AB3F5007F06F1340594BF01270427D1
:105D1800403655F8041B91FBF7F1204689B2FEF78F
:105D280011F8AE42F5D1504D504F05F10C06B5ECC7
:105D3800010AD7ED087A80EE270A2AF00DFA81B217
:105D48002046FDF7FFFFB542F1D1494D05F10C069C
:105D580055F8041B204689B2FDF7F4FFAE42F7D18F
:105D6800FEF740BF2368434A4349D078434A5D1C45
:105D78002560187023681278581C20601A702268F1
:105D8800C978FEF7CFBF00231B7AFFDE23685A1CB1
:105D98002260197029882046FDF7D4FF2368EA7825
:105DA800591C21601A7023682A79591C21601A70BD
:105DB8002368AA79591C21601A7023686A79591CCA
:105DC80021601A70F1E5212D5ED11A46591CC8F8D8
:105DD80000102B4D12F8021B6970C8F800205A7881
:105DE8002A70DA1CC8F800209B78AB704046FDF793
:105DF8006DFFD8F80030E880591C1A46C8F8001022
:105E080012F8021B2971C8F800205B786B714FF0FB
:105E1800FF352B46FEF731BF5A1CC8F800201A7808
:105E28000A2A7FF438A99A1CC8F80020154A59781C
:105E38001170D91CC8F8001099785170191DC8F84C
:105E48000010DB789370FFF726B900BF858D00201E
:105E580098890020F4520020CC84002004330020CC
:105E680000400020084200204878002020700020D0
:105E78004C4200208434002064370020743700200E
:105E8800784100205F8C00200B3DEF2D3FF603A9E1
:105E980001A252F825F000BF7F6C00089F5000084F
:105EA8009F5000089F5000089F5000089F5000080E
:105EB8009F5000089F5000089F5000089F500008FE
:105EC8009F5000089F5000089F5000089F500008EE
:105ED8009F5000089F5000089F5000089F500008DE
:105EE8009F5000089F5000089F5000089F500008CE
:105EF8009F5000089F500008116C00089F50000830
:105F0800F76B00089F500008D56B00089F500008E9
:105F18009F5000089F500008C16B00089F50000860
:105F28000B6B00089F500008D36A00089F500008B8
:105F3800AB6A00089F500008976A00089F50000845
:105F4800356A00089F500008ED6900089F50000856
:105F58009F5000089F5000089F500008ED4B000814
:105F68009F500008CD6900089F5000089F50000806
:105F7800B16900089F5000089F5000089F50000812
:105F88009F5000089F5000089F5000089F5000082D
:105F98009F5000089F5000089F500008656900083E
:105FA8009F500008DD6800089F5000089F500008B7
:105FB800A96800089F5000089F5000089F500008DB
:105FC8009F5000089F5000089F5000089F500008ED
:105FD8004D6700089F500008236800089F5000087C
:105FE800076700089F500008A76600089F50000830
:105FF800796600089F5000089F5000089F500008CD
:106008009F5000089F5000089F5000089F500008AC
:106018009F5000089F5000089F5000089F5000089C
:106028009F5000089F5000089F5000089F5000088C
:106038009F5000089F5000089F5000089F5000087C
:106048009F5000089F5000089F5000089F5000086C
:106058009F5000089F5000089F5000089F5000085C
:106068009F5000089F5000089F5000089F5000084C
:106078009F5000089F5000089F5000089F5000083C
:106088009F5000089F5000089F5000089F5000082C
:106098009F5000089F5000089F5000089F5000081C
:1060A8009F5000089F5000089F5000089F5000080C
:1060B8009F5000089F5000089F5000089F500008FC
:1060C8009F5000089F5000089F5000089F500008EC
:1060D8009F5000089F5000089F5000089F500008DC
:1060E8009F5000089F5000089F5000089F500008CC
:1060F8009F5000089F5000089F5000089F500008BC
:106108009F5000089F5000089F5000089F500008AB
:106118009F5000089F5000089F5000089F5000089B
:106128009F5000089F5000089F5000089F5000088B
:106138009F5000089F5000089F5000089F5000087B
:106148009F5000089F5000089F5000089F5000086B
:106158009F5000089F5000089F5000089F5000085B
:106168009F5000089F5000089F5000089F5000084B
:106178009F5000089F5000089F5000089F5000083B
:106188009F5000089F5000089F5000081F66000895
:106198009F500008E16500089F500008F16400085E
:1061A800D76400087F6500089F500008BD64000898
:1061B8009F50000893640008816400082164000867
:1061C8009F500008F96300089F5000089F5000087E
:1061D800D7630008A36300088F63000861630008A1
:1061E80039630008176300089F500008FF62000821
:1061F8009F5000089F5000089F5000089F500008BB
:106208009F5000089F5000089F5000089F500008AA
:106218009F5000089F5000089F5000089F5000089A
:106228009F5000089F500008E56200089F50000832
:106238009F5000087B6200089F5000089F5000088C
:106248009F5000089F5000089F5000089F5000086A
:106258009F50000861620008CE4B1B78DB073EF5B3
:106268001AAF0125FDF7CCFBFDF720F92B46FEF709
:1062780004BD5A1CC8F800201A780F2A3EF60BAF46
:10628800991CC8F80010C2EBC202C3495878885458
:10629800D81CC8F800000A4499785170191DC8F82C
:1062A8000010D9789170591DC8F800101979D1706B
:1062B800991DC8F8001059791171D91DC8F8001036
:1062C8009979517103F10801C8F80010DB799371CD
:1062D800012522F00DFA2B46FEF7CFBC4046FDF70C
:1062E800F5FCAE4EB0814046FDF7F0FC012570810B
:1062F8002B46FEF7C2BC4046FDF7E8FCA84A00EB77
:1063080080004300012513802B46FEF7B6BC4046AB
:10631800FDF7DCFCA34EB0824046FDF7D7FCF082C7
:106328004046FDF7D3FC012530832B46FEF7A5BC7C
:106338001A46591CC8F8001012F8020BC8F80020B9
:10634800DA1C5978C8F800209A7819F0A3FB0028BD
:106358007EF448ACFEF79FBE1A46591CC8F80010D8
:10636800914912F8020B0870C8F800208B495A7836
:106378008A70DA1CC8F80020894A9B789370012536
:106388002B46FEF77ABC894B894918684A220125B1
:1063980029F06EFD2B46FEF770BC19465A1CC8F84A
:1063A8000020844A11F8020B1070C8F800105978C0
:1063B8005170D91CC8F800109B7893704046FDF7BF
:1063C80085FC7D4B0125D8802B46FEF756BC404600
:1063D800FDF77CFC784E30804046FDF777FC7080F6
:1063E8004046FDF773FC0125B0802B46FEF745BCFF
:1063F800724F3B78002B3EF4F5AB714E00254046BA
:10640800FDF764FC17F014FB3B78A6EC010A013594
:106418009D42F4DBFEF7E6BB0F2E7EF43CAE5A1C21
:10642800C8F800201D78072D3EF635AE654F40466A
:106438000C26FDF74BFC06FB05F6BD19A880404667
:10644800FDF744FCE8804046FDF740FCD8F80030F2
:1064580028811A46591CC8F8001012F8021BA972A4
:10646800C8F800205B78EB724046FDF717FC012561
:10647800B8512B46FEF701BC4046FDF727FC524BAE
:10648800012518802B46FEF7F8BB5A1CC8F80020D7
:106498001878060600F10A863E4B1B78DD073EF5A4
:1064A800A1AB032828BF00200125FAF73BFF2B46A4
:1064B800FEF7E3BB374B1B78D8073EF593AB0125B6
:1064C800FDF792FAFCF7F2FF2B46FEF7D6BB314BED
:1064D8001B78D9073EF586AB3C4B4FF4C8720125B3
:1064E8001A802B46FEF7C9BB092E7EF6D4AD384F6D
:1064F8001A46591C3D68C8F8001012F8021B29708A
:10650800C8F800205A78AA70DA1CC8F800209A78CF
:10651800642A03F10401A8BF64226A71C8F8001054
:10652800DA78642A03F10501A8BF6422AA71C8F8C1
:1065380000101A79EA719A1DC8F800205A79642A5D
:1065480028BF6422D91D2A72C8F800109A79EA7007
:1065580003F10802C8F80020DB792B714046FDF7EB
:10656800B5FB0A2E688140F0AC85012515F0E6FFE1
:106578002B46FEF782BB074B1B78DA073EF532AB9A
:10658800144A1378012543F0040313702B46FEF7D1
:1065980074BB00BF9B4400201C7A00208434002078
:1065A800643700204C4500200C700020A484002093
:1065B8005C2E0308C01D0020E83F00202034002086
:1065C800EC3E0020E47B0020BC1D00202693002028
:1065D8004838002038350020D24A1068DA1C0146B5
:1065E8002133951EC8F8005012F8035C0D70551E33
:1065F800C8F8005012F8025C4D70C8F8002012F874
:10660800015C8D700332934201F10301E9D122F05C
:1066180047FAFEF7E7BAC6F34706122E3EF63BAD39
:10662800B6B10EAB0DF1120703EB4605B946263D90
:106638004046FDF74BFB29F8020F4D45F8D1BA4B00
:1066480037F8022F23F8022F4F45F9D1112E09D818
:10665800B64A7300023B13440021223223F8021F7A
:106668009A42FBD1B24A01231D461370FEF705BBBF
:106678001A46591CC8F80010AE4912F8020BC87027
:10668800C8F80020AC495A780A70DA1CC8F800200B
:10669800AA4A9B78D37001252B46FEF7EEBA4046EE
:1066A800FDF714FB4046FDF711FB4046FDF70EFBD6
:1066B800D8F800309B4D9A1C2F68C8F800205A78EB
:1066C80087F82F20DA1CC8F800209A7887F83A2033
:1066D8001A1DC8F80020DA7887F83B200733C8F875
:1066E80000304046FDF7F2FAF88740462F68FDF77C
:1066F800EDFA112EB88700F20E85286887E75A1C34
:10670800C8F80020874D8E4F1B78D5F800907B7114
:106718004046FDF7DBFAA9F820004046D5F800907E
:10672800FDF7D4FA052EA9F8220000F20685FAF73B
:1067380015FE20F037FF2868012516F0ADFF2B461F
:10674800FEF79BBA4046FDF7C1FA054623F076FCF2
:10675800FF283EF447AAB5F57A7F80F0C4840DF18E
:106768003809002309F8243DEE08494603A88DF8A6
:106778000C30013623F042FC9DF80C30F6B205F0DF
:106788000705B34205F1010503D19DF81430AB426A
:1067980003D02946304623F03DFCD8F80030D8F81D
:1067A8000420D21A012A7EF71DAA5A1C0EA8C8F87E
:1067B800002000221D7800F82C2D23F013FC9DF8F2
:1067C8000C30AB420AD05F4B1B683BB19A79AA42A6
:1067D80004D31B681B690BB128469847D8F80030CA
:1067E8005A1CC8F80020484600221D788DF814204D
:1067F80023F0ECFB9DF81430AB423EF4F3A9514B67
:106808001B68002B3EF4EEA91B685B69002B3EF465
:10681800E9A928469847FEF7E5B91A46591CC8F869
:106828000010474E12F8021BB170C8F80020464904
:106838005A780A70DA1CC8F80020444D9A782A71F0
:106848001A1DC8F80020DB78092BA8BF0923404689
:10685800AB70FDF73BFAD8F80030D8F80420288050
:10686800D11A012907DD4046FDF730FAD8F8003083
:10687800D8F8042068829A4240F08284FAF76EFDC4
:10688800D8F80030D8F804209A423EF4ABA95A1C34
:10689800C8F800201B78EB7001252B46FEF7EDB9F0
:1068A8002B4A1278012A3EF69DA919465A1CC8F8A7
:1068B8000020284A11F8020B9070C8F80010597887
:1068C8001170D91CC8F800109B78537001252B460D
:1068D800FEF7D3B95A1CC8F800201E78112E3EF6D0
:1068E800DAAB9A1CC8F800201B4D5B7805F8163007
:1068F8004046FDF7EBF940F6CA039842A8BF184690
:1069080040F2EE23984205EB4601B8BF1846012530
:10691800A0F2EE222B46192092FBF0F24A70FEF705
:10692800ACB900BFA4840020DE300020E030002095
:10693800043100208434002074370020643700209C
:106948000C700020D8840020087B00204C450020D3
:10695800848D0020858D0020043300201A46591CA0
:10696800D34DC8F8001012F8021B2970C8F800208F
:106978005B786B704046FDF7A9F9D8F8003068805D
:106988005A1CC8F800201B782B714046FDF79EF969
:10699800D8F80030E8805A1CC8F800201B782B7201
:1069A80001252B46FEF769B9C24A03F108010133F4
:1069B800C8F8003013F8010C02F8010F9942F6D11B
:1069C800FEF710B9591C1A46C8F80010BA4912F84F
:1069D800020B8870C8F800205B784B7001252B46A5
:1069E800FEF74BB90722B6FBF2F2C2EBC201761AE8
:1069F8007EF451ABD2B2571EFFB2002A3EF4F2A881
:106A0800DFF8B8A201375A1CC8F8002093F9001023
:106A1800AA4B002593F902208A4200F0A48201358E
:106A2800062D03F10803F5D1FEF735BB5A1CC8F84B
:106A380000201A780E2A3EF62EAB991CC8F80010D2
:106A48005D78032D3EF627AB9D48062101FB02F138
:106A58004218DE1C5571C8F800609D784554191D10
:106A6800C8F80010D9785170591DC8F80010197964
:106A78009170991DC8F800105979D170D91DC8F8BE
:106A880000109B79137101252B46FEF7F6B85A1CA6
:106A9800C8F800208B4A1B78537501252B46FEF752
:106AA800ECB85A1CC8F800201D781F2D3EF6F3AA32
:106AB800052E7EF4F0AA4046FDF7F0F8824B43F825
:106AC800250019F059F8FEF78DB87F4D05F14006FD
:106AD8004046FDF7FBF8D8F80030A5F88000591CAF
:106AE8001A46C8F8001012F8021B85F88210C8F878
:106AF80000205B7885F883300435AE42E8D1FEF794
:106B080071B85A1CC8F800206E4D1B782B7240468D
:106B1800FDF7DCF8A8834046FDF7D8F828834046FF
:106B2800FDF7D4F8D8F8003068835A1CC8F800205C
:106B38001B78EB74082E7EF655A84046FDF7C6F87C
:106B4800E8844046FDF7C2F80C2E28857EF64AA850
:106B5800D8F800301A46591CC8F8001012F8021B61
:106B6800A977C8F800205B7885F820304046FDF703
:106B7800ADF8102EA8847EF635A8D8F800305A1C37
:106B8800C8F800201B78EB724046FDF787F8D8F864
:106B98000030E8605A1CC8F800201A782A74162EAB
:106BA8007EF620A89A1CC8F800205B7885F821306A
:106BB80001252B46FEF761B85A1CC8F80020434A45
:106BC8001B78137001252B46FEF757B84046FDF792
:106BD8007DF83F4E30604046FDF778F870604046DB
:106BE800FDF774F80125B0602B46FEF746B8394E1C
:106BF800002333604046FDF751F83368012503430D
:106C080033602B46FEF739B85A1CC8F800201878AC
:106C180013283EF640AA9A1CC8F800205D782E4A30
:106C2800002105E00131242902F10C023EF433AAC7
:106C3800167AAE42F6D1294D294A0C2606FB015197
:106C4800DD1C91F83C1002F82010C8F8005002EB47
:106C5800800299785170191DC8F80010D878907082
:106C6800581DC8F800001F491B790868D37015F033
:106C7800F3FBFDF7B7BF1C4B102E4FF0000228BFE7
:106C880010261A605A609A60DA601A74002E3DF471
:106C9800A9AFD8F8002016440132C8F8002012F82D
:106CA800011C03F8011BB242F6D1FDF79BBF00BFE0
:106CB800004000204B4A0020541E0020D86F0020BE
:106CC800F03800204C4A00206C400020F8360020A4
:106CD800182E0020808D002020260308E4250308B4
:106CE800FC360020A4840020928400205A1CC8F896
:106CF80000201B780A2B00F02181502B7EF4CBA9B1
:106D08004046FCF7E3FFCD4E30804046FCF7DEFFFF
:106D18004FF0FF3570802B46FDF7AFBFDFF85CB34F
:106D28004FF000084FF0080A08F10108B8F1240FE5
:106D38001BD0C8F120020AFA02F22BFA08F6A8F1D1
:106D4800200316432AFA03F31E4306F00102002328
:106D58001343E9D05FFA88F015F078FB0028E3D0F8
:106D680041464846FAF79AFADEE7B54B1B78DF0743
:106D780000F1E9800026B34FB04602E00136242E28
:106D88000ED031463846FDF711FA0028F6D03146C4
:106D98004846FDF70BFA002856D108F10108EDE73F
:106DA800A94BAA4EB3F850102046FCF7CBFFA84BCE
:106DB8001988204689B2FCF7C5FFA64B1A6853010B
:106DC80003F02001C2F340030B43C2F3800143EAFE
:106DD8004103C2F3C00143EA8103C2F3401143EA0D
:106DE800C10102F0100211432046FCF7ABFF03A9D2
:106DF80004222046FCF776FF23683178964A581C0F
:106E08002060197011886429A8BF64212046FCF706
:106E180099FF962D00F09C8000212046FCF792FFF8
:106E28002168B8F1190348BFA8F11203A3F3C403FA
:106E38004A1C226020460B701A4604A90125FCF75B
:106E480051FF2B46FDF719BF414603A8FAF726FA6A
:106E5800A3E72368B178814A581C20601970236819
:106E68001278591C21601A70FEF72CBED9F8003030
:106E780013F48053B4EEE88A00F09F80F1EE10FA24
:106E880013DBB4EEC98AF1EE10FA00F29980DFED57
:106E9800747A9FED747A77EEC87AB4EEC78AF1EE09
:106EA80010FAB0EE678A40F28B804FF47A71B5EE33
:106EB800408AF1EE10FA40F2DC5308BF1946FEF79B
:106EC80023BC95F82420684B002A40F0D98030462E
:106ED800FEF7BCBE5A1C1946C8F80020594811F8DC
:106EE800022B0272C8F800105B784372042A06D994
:106EF800FF2A3EF4D5A922680021FDF713BF5B499C
:106F08000978994203D8022AF5D1FF2BF3D12368D7
:106F180001255A1922601D70B9F1000F3DF462AEC7
:106F2800534BC9F800302B46FDF7A7BE2268012550
:106F3800531923602B461070FDF79FBE4046FCF79F
:106F4800C5FE4C4EE0E6059B43F00103059311E7AF
:106F580023680322591C21601A7023687278591C0F
:106F680021601A705CE70AEBC509404689F80210EF
:106F7800FCF7ACFED8F800202AF835001346511C5F
:106F8800C8F8001013F8021B89F80310C8F800307D
:106F9800537889F80430D31CC8F80030937889F8FE
:106FA8000630131DC8F800300136D27889F805205C
:106FB800B7427FF428ADFDF715BEF1EE10FA68DB95
:106FC800F7EE007A78EE677AB6EE007AF0EE696A44
:106FD800E7EE876A40F2E932FDEEE67A17EE901A9C
:106FE800B1F5FA6FA8BF4FF4FA619142B8BF1146E4
:106FF80089B2002B3EF488AB59E7831C0021196045
:10700800596019726AB1511CD8F800200144013B3B
:107018000132C8F8002012F8010C03F8010F994258
:10702800F6D1154B1B78002B3EF435A84FF0FF35F1
:1070380020F042FA2B46FDF720BE00BF0C260020A8
:107048009B440020B01D0020AC1600208E84002038
:1070580004450020B47C00209A2F0020087B0020E3
:1070680000C0884400C08244F4520020203400202C
:10707800950E0008501E0020B825002090E33FF42C
:107088005978022909D003290CBF04203046FEF79D
:10709800DDBD4FF47A71FEF737BB042A34BF0220F6
:1070A8000320FEF7D3BD4246FEF73FB900F07F004C
:1070B800032828BF0020012513F066FF2B46FDF7A3
:1070C800DCBDD8F800303A68591CC8F800101978A7
:1070D80051720B2E3FF449AA991CC8F800105B782E
:1070E8005370FFF742BA0DF11409484622F062FFC7
:1070F800BDF81430AB423FF450AB264B1B68002B55
:107108003FF44BAB1B689B69002B3FF446AB28460A
:107118009847FFF742BBD8F800302968581C1A4630
:10712800C8F8000012F8020B81F83100C8F80020F6
:107138005B7881F83230FFF7E0BA4046FCF7C6FDCD
:1071480078814046FCF7C2FDB8814046D5F80090EA
:10715800FCF7BCFDA9F824004046D5F80090FCF7E0
:10716800B5FD0D2EA9F826007FF6E1AA4046FCF7EA
:10717800ADFDF8814046FCF7A9FD3882FFF7D7BA84
:107188005A1CC8F800201B78003318BF0123F3717C
:10719800FFF774BBD88400202DE9F04F2DED028B4A
:1071A800C54B1B7891B0072B059001F0788200231E
:1071B8000793C24BD3F800A01AF4806F40F06086A2
:1071C800BF4B1B6806931C0700F10486BD4BBE4DE0
:1071D800B3F80090BD4CBE4BBE491F68B1F906809C
:1071E8007A89904580F29F84BB4B4FF07E521A609B
:1071F800DFF8F8B294F90820B1F900C0BBF81860BC
:10720800207994F805E0002AACEB060314BF0122AC
:107218004FF0FF32002B40F3EE84B3F5FA7FC0F253
:10722800F0844FF4FA731B1A07EE903AF8EEE77AF7
:10723800B445C5ED007A03DAF1EE677AC5ED007A58
:10724800B1F902C0ACEB0603002B40F3E184B3F5BF
:10725800FA7FC0F2E3844FF4FA731B1A07EE903AF0
:10726800F8EEE77AB445C5ED017A03DAF1EE677A0C
:10727800C5ED017AB1F90430991B0029D8BFF11A7C
:10728800B1F5FA7F80F249847145D8BF4FF0000EFE
:1072980000F3458402FB0EF207EE902AF8EEE77A37
:1072A800B342C5ED027ABCBFF1EE677AC5ED027A4A
:1072B8001AF48053049300F0E980B8F5FA6F424657
:1072C800A8BF4FF4FA62B2F57A7FB8BF4FF47A726A
:1072D800A2F57A728149DFF818E281FB0230D317F0
:1072E800C3EB6013581C6FF0630C3EF910003EF9B5
:1072F80013E00CFB0323A0EB0E0003FB00F381FB60
:107308000321DB17C3EB61139E440FFA8EFE07EED1
:1073180090EA049BB8EEE78A85ED038A002B40F0DB
:10732800BC8519F04003089340F0C584069B13F010
:10733800140F03D019F4027F40F07286684B1B7853
:1073480023B1BBF81A30434580F2A68494F8326022
:107358001EB119F0030F40F0668794F838209BF8A7
:107368001F30002A40F0C6859BF81E60002E00F0F2
:10737800C380022E00F05187032E00F0338759494D
:1073880049880233DBB2002A00F03987002900F06F
:10739800368755480668B1FBF6F10EB2A4F8686066
:1073A800ABB307EE906AF8EEE77AF7EE006A86EE7E
:1073B800A77A012BD5ED007AD4ED1F6A77EEE67A2D
:1073C80067EE877AC4ED1B7A21D0D5ED017AD4ED2A
:1073D800206A77EEE67A022B67EE877AC4ED1C7A8C
:1073E80015D0D5ED027AD4ED216A77EEE67A032B33
:1073F80067EE877AC4ED1D7A09D0D5ED037AD4ED0E
:10740800226A77EEE67A67EE877AC4ED1E7A2A4911
:107418000978092901F08C84002E72DD93B394ED6C
:107428001F7AD4ED1B7A77EE877A012BC4ED1F7A89
:10743800C5ED007A21D094ED207AD4ED1C7A77EE50
:10744800877A022BC4ED207AC5ED017A15D094ED28
:10745800217AD4ED1D7A77EE877A032BC4ED217A51
:10746800C5ED027A09D0D4ED227A94ED1E7A77EE32
:10747800877AC4ED227AC5ED037A013B022BB8BFA7
:107488000223DBB2002A18BF02233BE0BBF81A1024
:107498008845C0F2FF83B8F5FA6FD4BFC1EB080383
:1074A800C1F5FA634FF47A7202FB03F2C1F5FA618F
:1074B800B2FBF1F20EE700BFFA3600207C4A00204A
:1074C800B47C0020D8410020F8850020BC1D002095
:1074D800483800203C8B0020182500201F85EB51E0
:1074E80037020020CC840020E03600204C4A0020DF
:1074F8004C3800200AD7233CA4F86860002A00F022
:107508006F8102233A785FED056AB97807EE902A11
:10751800F8EEE77AB0EE007A67EEA67AD24AF4EE91
:10752800C77AF1EE10FA107840F35084DFEDCF6A95
:1075380037EEC77AB0EE676AA7EE266AF0EE466ABB
:1075480095ED007A9FEDCA6ADFF848E3DFF848C393
:1075580027EE066AF0EEC65ACEED005A8CED006AA8
:1075680099B107EE101AB8EEC75A9FEDC27A66EEC7
:10757800064A25EE075AB7EE007A37EE457A64EEEA
:10758800A54AA5EE247A26EE076A9FEDBB7A7A799A
:1075980026EE877A27EE067AAAB1DFEDB66A9FED66
:1075A800B76A65EEA65A06EE902AF8EEE66A66EE27
:1075B800A56AF4EEC66AF1EE10FA40F3E6859FED8F
:1075C800B06A27EE067A0C289FEDAE8ADFEDAE6A28
:1075D800DFF8C88200F0B485B4EEC87AF1EE10FA8C
:1075E80098BFB0EE478AB4EEE68AF1EE10FAB8BF5B
:1075F800B0EE668A88ED008A002B00F0E680B0EED7
:10760800007AF4EEC77AF1EE10FA05DD37EEC77AA4
:10761800DFED966AE7EE267A95ED017ADFED946A5A
:1076280027EE267AF0EEC75A8CED017ACEED015A94
:1076380099B106EE901A9FED8F6AF8EEE66A27EE8A
:10764800075A66EE866AB7EE006A36EE666A25EE77
:10765800255AA6EE856A27EE067ADFED876ABA799B
:1076680067EEA67A67EE877AFAB107EE102AB8EEC7
:10767800C77A9FED806ADFED816A27EE257A27EECB
:10768800067AB4EEE67AF1EE10FA00F37A85B5EEF2
:10769800C07AF1EE10FA01F18380B7EE006A36EE97
:1076A800477AC6EE076A67EEA67A0C2800F02985A5
:1076B800DFED746A9FED747AF4EEE67AF1EE10FA73
:1076C80088BFF0EE667AF4EEC77AF1EE10FAB8BF2A
:1076D800F0EE477A012BC8ED017A76DD7B78DFED95
:1076E800656A07EE903AF8EEE77AB0EE007A67EE50
:1076F800A67A7B7AF4EEC77AF1EE10FA05DD37EE5A
:10770800C77ADFED5A6AE7EE267A95ED027ADFED61
:10771800586A27EE267AF0EEC75A8CED027ACEED3B
:10772800025A9BB106EE903A9FED526AF8EEE66A6D
:1077380027EE075A66EE866AB7EE006A36EE666A84
:1077480025EE255AA6EE856A27EE067ADFED4A6A07
:10775800FB7967EEA67A67EE877AFBB107EE103AF7
:10776800B8EEC77A9FED436ADFED446A27EE257AC3
:1077780027EE067AB4EEE67AF1EE10FA00F3FD840D
:10778800B5EEC07AF1EE10FA01F10680B7EE006AA4
:1077980036EE477AC6EE076A67EEA67A0C2800F03E
:1077A800A884DFED386A9FED387AF4EEE67AF1EED8
:1077B80010FA88BFF0EE667AF4EEC77AF1EE10FAA6
:1077C800B8BFF0EE477AC8ED027A092800F088843D
:1077D8009BF82150002D40F03E84002384F8383077
:1077E8002A4D2B4F95F82420DFF8B480DFF8B4A099
:1077F800531E082B00F21181DFE813F02D01A901B7
:10780800A4000F0156000900BD010F01AB0198F853
:107818000030002B40F0C1842B68287A03EB00204D
:107828001FF090FD2B7A0133DBB2022B2B7240F054
:10783800638100201CF0D4FF00201CF0D1FF1CF055
:10784800F9FF00F01F00052801F065831AF092F88F
:10785800EE68002E00F0A58300222B6969680120DC
:10786800B04795F82420C3E7FA360020D7A368412B
:107878006F12033B0AD7233C00004843A4707D3FA6
:107888000000C84200C0F94400C0F9C4988900202B
:107898003C450020442500203825002020250020D4
:1078A800AA440020580002404FF4007128681AF0DA
:1078B80019F8012800F0EC84C0F0D385022840F0C4
:1078C8001B811AF08FF81AF055F8EE68002E00F0B8
:1078D8006883002210462B696968B04795F8242010
:1078E80086E71021D14819F0FDFF002840F00281F9
:1078F800049001217F2025F0DDFD01288146049BAD
:1079080040F0F8801846022125F0D4FD002801F047
:10791800A881012840F0EE8016213A2025F0CAFD02
:10792800431C9B02EB631AF05DF83068FBF712FB0F
:1079380000210A2019F0F2FF002840F0F7860323FF
:1079480085F8243010210CA819F0CCFF002840F04D
:10795800D3809DF83A209DF839009DF83C109DF899
:107968003D309DF83B60120442EA00620A431B0165
:107978009DF83E109DF83100DBB243EA111342EA4C
:10798800062203F5FA636A632B879DF832209DF877
:10799800383042EA002201F00F01180903F00F0302
:1079A80085F83A106A859DF830109DF8332085F8DF
:1079B80032309DF8343085F8281085F82C209DF851
:1079C80035109DF8362085F82D309DF8373085F82C
:1079D800303085F8310085F82E1085F82F201AF000
:1079E80001F8AB7E002B00F03981914A138823F00F
:1079F80040031B041B0C1380138823F038031B045B
:107A08001B0C138013889BB243F0400313800021A2
:107A18000422296285F824200323DBB2022B71D9C2
:107A2800042A00F0C280082A00F0BF80814B1B782E
:107A380023B9814EB278002A40F0278505980BF0CB
:107A480003FC7E4B1B78072B00F0798411B0BDEC4A
:107A5800028BBDE8F08F7A4E3068FBF77BFA002185
:107A6800084619F05BFF814619F0BCFFB9F1010F18
:107A780042D1002330686B76FBF76CFA40F2AB1109
:107A8800082019F04BFF052800F00E84012800F0AB
:107A98000B8619F0A7FF6B7E002B01F038820223BA
:107AA80085F824303068FBF755FA6B7E022B14BF3B
:107AB8004FF000094FF080490021372019F02EFFC0
:107AC8004946292019F02AFF814619F08BFFB9F1A0
:107AD800000F11D16B7E022B00F01A8685F81A90E0
:107AE8003068FBF737FA0021092019F017FF002842
:107AF8003FF4F7AE19F076FF95F82420531EDBB259
:107B0800022B8DD84F4B69691B685B1AC82B8AD921
:107B180019F030FF95F8242082E74FF4FA71A1EBB1
:107B28000E0EFFF7B7BBB8F5FA6FC0F2A7803B7A25
:107B3800C3F1640307EE903A9FED437A434BF8EEA6
:107B4800E77A67EE877AC3ED007AFFF751BB3C4EC0
:107B5800A8E708261CF06EFEFF2800F01B84013EF3
:107B6800F8D16B693A68FA339342C5D219F002FF2B
:107B780095F824203CE61CF05DFEFF284FF008062F
:107B880005D0013EEDD01CF055FEFF28F9D12B6A37
:107B98000022012B2A7641F26884EA69013B01320E
:107BA8002B620823EA6185F82430294D1AF0CEFAB1
:107BB8006B78022B00F0FA83032B7FF437AF41F286
:107BC800B813EB5C002B41F0698041F2A403EB5C35
:107BD800002B41F06D8041F2E803EB5C002B41F093
:107BE800628041F22C13EB5C002B3FF41FAF194865
:107BF80023F010FE1AE7A6EB0C03B3F5FA7FBFF6E5
:107C080010AB9842FFF60FABDFED137AFFF710BB0E
:107C1800A6EB0C03B3F5FA7FBFF61DAB9842FFF64F
:107C28001CABDFED0D7AFFF71DBB00BFD889002024
:107C380000380040E3410020858D0020FA360020FE
:107C4800AC4400203C4500200AD7233C18250020DE
:107C5800F45200202064002000000000D24E30685A
:107C6800FBF778F94FF40071102019F057FE06461B
:107C780019F0B8FE002E3FF4B8AE77E7387AA8EBD3
:107C8800020303FB00F3C2F5FA6293FBF2F3C3F1BC
:107C980064034FE71A4609E4C44B1B78012B00F034
:107CA8004383192B00F040830E2B3FF44FAB082B76
:107CB8003FF44CAB3DE3BE4BBE49B3F90430628997
:107CC800DFEDBD6A9FEDBD7A81FB0301DB17C3EBD6
:107CD800A1039B1A1BB207EE903AF8EEE77A67EE1B
:107CE800A67A77EE876ABDEEE66A16EE103A20337A
:107CF800402B40F26F83DFEDB26ABDEEE77A17EEF4
:107D0800103A2033402B00F262839FEDAE7AF4EEF6
:107D1800C77AF1EE10FA40F3DF87DFEDAB5A9FED3B
:107D2800AB6A01E0F0EE477AF4EEC67AF1EE10FAAB
:107D380037EEE57AF6DCDFEDA67AB4EEE77AF1EE17
:107D480010FA40F1CD87DFEDA05A9FEDA26A01E05D
:107D5800B0EE677AB4EEC67AF1EE10FA77EE257ACD
:107D6800F6D49FED967AF4EEC77AF1EE10FA00F3A6
:107D780096829FED997AF4EEC77AF1EE10FA44BF35
:107D88009FED937A77EE677A67EEA75A9FED935A3D
:107D98009FED936A9FED937AA5EE856A27EEA55A23
:107DA800A5EE867AE5EE077A95ED016AD5ED005ADB
:107DB80027EEC67A65EEA77AA5EEA67AE6EE267ACB
:107DC80085ED007AC5ED017AFFF7B0BAF0EE676A83
:107DD800FFF7B6BB844D854BD5ED027AB3F800901A
:107DE800734B744AB3F90430814CB2EE0E7AF0EE5C
:107DF800E76AF4EEC76AF1EE10FA82FB03124FEA63
:107E0800E37338D519F0040F35D02188C3EBA203EA
:107E18005B1A9BB21AB212F1B30FBCBF03F5B4736D
:107E28001AB2B32AC8BFA2F5B4737249C8BF1AB24E
:107E3800237A0978002B4FF6FF7318BF0123080730
:107E48007FF5C9A96C49096812FB03F30A7E6B49DF
:107E58009BB212FB03F381FB03121A44DB17C3EB3B
:107E6800221307EE103AB8EEC77A77EEC77AC5ED57
:107E7800027AFFF7B0B9C3EBA2032380FFF7ABB9CF
:107E88005F488368002B3FF49BA900F144019847A1
:107E98005C4BD3F800A0FFF793B91D215A48FCF7B3
:107EA80085F900283FF43DAA584BDB78002B7FF476
:107EB80038AADFED577A574938EE678AC6F5FA636C
:107EC800FDEEC87A1BB2CDED087ABDF92020120369
:107ED80081FB0201D217C2EBA11203FB02F343F3A9
:107EE8000F33334407EE903AF8EEE77AC5ED037A9C
:107EF800FFF717BA48484449D0F8EC00096844F637
:107F08002066B042A8BF3046B0F57A7FB8BF4FF4BC
:107F18007A7080B2C906608740F1CA810499002945
:107F280000F042843449D1F800C0BCF836E04FEA8A
:107F38005E0E384EE16BD5ED037AA6FB006086092C
:107F4800642090FBF6F01428BDEEE77A04EB4108B4
:107F5800A8BF142001318142E16317EE109AA4BF33
:107F68000021E16304EB4101A8F84090B1F9401009
:107F780007EE101AB8EEC77A77EEC77AFDEEE77A01
:107F8800CDED047ABDF9100080EAE071A1EBE07153
:107F9800714500F3928621494FF07E500860FFF743
:107FA800E3B995F8242023E4AC440020F8360020F7
:107FB8005C4200206766666635FA8E3CDB0FC93F77
:107FC80000000000DB0F4940DB0FC940E4CB16413D
:107FD800DB0F49C0E4CB16C1DB0FC9BF92E741B93B
:107FE8009730083C15A82ABEF8850020D841002003
:107FF800BC1D002038350020A4840020898888888A
:10800800207000207C4A0020303500208441002068
:1080180000007A44D34D6210AC16002028000020DE
:10802800CC4B1B7813F0100300F05281227B23699C
:1080380095ED017A002A0CBF01224FF0FF3203FBB5
:1080480002F307EE903AF8EEE77A77EE877AC5ED15
:10805800017AFFF773B91E21BF48FCF7A7F800287B
:108068003FF4BBAB089B002B7FF4B7AB94F88C3084
:10807800AB4240F07F86B94BD4ED247AD3ED006A49
:1080880098ED025ADFEDB65A9FEDB66A27EEC57A2B
:1080980068EE277AA8EE267AE5EE267AB4EEE57A37
:1080A800F1EE10FA88BFB0EE657AB4EEC67AF1EE5A
:1080B80010FAF4EEE57AB8BFB0EE467AF1EE10FAAF
:1080C80088BFF0EE657AF4EEC67AF1EE10FAB8BF22
:1080D800F0EE467A88ED007AC8ED027AFFF77DBBAC
:1080E800FDEEC87AA04A17EE903A9680D380FFF743
:1080F8006FBBBDEEE77A9C4B17EE102A9A80FFF70C
:1081080050BB9FED977ADFED976A9749F4EEC77AEF
:10811800F1EE10FA98BFB0EE677AFDEEE77AB4EEAA
:10812800E67AF1EE10FA17EE902AB8BFB0EE667A4A
:10813800012B88ED017A4A803FF7D0AAFFF748BBA8
:10814800B4EEC87AF1EE10FA98BFB0EE478ABDEEE9
:10815800C77AB4EEE68ADFF81092F1EE10FA17EE5D
:10816800102AB8BFB0EE668A88ED008AA9F8002008
:10817800002B7FF444AAFFF72BBBDFED7C6AFFF7E7
:108188000BBBDFED7A6AFFF78EBAF7EE005A75EE91
:10819800E66A85EEA66AFFF714BA754B19688E036E
:1081A8007FF541AC4FF400325A60DAF80020714B89
:1081B8004FF6FE710A40CAF800201A89D2077DD40A
:1081C8001FF070F80028FBD16A4A938823F0020355
:1081D8001B041B0C938098F80030002B7FF429AB0C
:1081E800FFF71ABB9BF82010C1EB411001EB80018F
:1081F800C900023389B2DBB2002A7FF4C7A8B4F8F9
:108208006860013E36B2002EA4F868603FF706A900
:10821800002A7FF476A9FFF7E3BA618F01F57A7136
:1082280089B2FFF7AEB8544BDFED547A93ED080AE4
:10823800B4EEE70AF1EE10FA40F2958228F022F83F
:10824800D4ED0D7A20EE270A27F086FFB0F5617F7E
:1082580000F3B18207EE900AF8EEE76ADFED487A9C
:1082680066EEA76A07EE906AB8EEE77AFDEEE67A60
:1082780017EE903A2033402B40F263869FED410A77
:1082880027F06AFF00B207EE900AB8EEE77A6CE2D0
:108298006B693A6864339342FFF413AB2CE49FEDA7
:1082A8003A7A77EE677A6FE585F81990FFF7F1BBB0
:1082B8001AF0805F7FF432AEFFF756B89A891A89B0
:1082C800D007FBD41EF0EEFF00287FF479AF7BE7E0
:1082D800E279002A40F08882B4F91460A179A8EB09
:1082E800060383EAE370A0EBE370884240F3158548
:1082F80003EBD37301225B10A36284F82C2022774E
:1083080023691E44B6F5FA6FA8BF4FF4FA66B6F5AE
:108318007A7FB8BF4FF47A7607EE906AF8EEE77A7C
:10832800C5ED037AFFF70AB8184B9B7B002B7FF447
:108338000DA8174A0023AB609360FFF707B8FAF758
:1083480043F9079A084B801A988011B0BDEC028B4C
:10835800BDE8F08F3835002030350020200000209F
:1083680000C0F94400C0F9C4E44100200000C8423C
:108378000000024000380040783800208FC2753C69
:10838800D06D393A00000000DB0F494060820020C0
:108398002025002019F026FB042385F82430C84D39
:1083A80019F0D4FE6B78022B7FF406ACAB784FF053
:1083B80001082746072B00F20184DFE813F0A50324
:1083C8002D04BF032803CC038F0399033403DFED87
:1083D800CF7AE9E4F4EEC77AF1EE10FA40F38F852C
:1083E800DFEDB85A9FEDB86A01E0F0EE476AF4EEA7
:1083F800C66AF1EE10FA36EEE57AF6DCDFEDC26A0F
:10840800B4EEE67AF1EE10FA40F17585DFEDAD5A7B
:108418009FEDAE6A01E0B0EE667AB4EEC67AF1EE90
:1084280010FA77EE256AF6D49FEDA97AF4EEC76ABA
:10843800F1EE10FA40F38B819FEDA67A77EE666A2B
:1084480066EEA65A9FEDA45A9FEDA46A9FEDA47A02
:10845800A5EE856A26EEA55AA5EE867AE5EE076AA8
:108468004BE419F0BFFAEE680423002085F82430A5
:108478002876002E3FF499AB2B692A686968B047C3
:1084880095F82420531EFFF73ABB964F3B78013BE3
:108498000A2B59D8DFE813F099028B027F02650294
:1084A800580058005102E901C601A8020B00022A2F
:1084B80038D18D4BDFF848821B78002B40F0DC87E1
:1084C800D8F8005045B32B7833B395F82820002A04
:1084D80040F053812B7EAA6385F83C20042285F85E
:1084E800282013F008036A6AEA622A6303D0744AF0
:1084F80041F29413D3586B634FF00009C5F82490E8
:10850800C5F80890C5F80C90284624F089FF052383
:10851800C5F8409085F8283000220423C8F80020C8
:1085280088F81430714B724A5B681268C8339342FA
:1085380004D31EF0BDF8002800F03782B278032A71
:1085480001F03A8001233B70022A00F01681F3788B
:10855800002B3FF473AA674B1B68D90440F1788558
:10856800654B9B8807EE903AF8EEE77A634991ED00
:10857800012AD1ED022A91ED033AD1ED043A91EDA9
:10858800054AD1ED064A91ED075AD1ED085A91ED09
:10859800096AD1ED0A6A91ED0B7AB4EE672AF1EE19
:1085A80010FAF4EE672A14BF01230023F1EE10FA43
:1085B800B4EE673A18BF43F00103F1EE10FAF4EE97
:1085C800673A18BF43F00103F1EE10FAB4EE674AB8
:1085D80018BF43F00103F1EE10FAF4EE674A18BF32
:1085E80043F00103F1EE10FAB4EE675A18BF43F0F6
:1085F8000103F1EE10FAF4EE675A18BF43F00103D5
:10860800F1EE10FAB4EE676A18BF43F00103F1EE19
:1086180010FAF4EE676A18BF43F00103F1EE10FA9E
:10862800B4EE677A18BF43F00103F1EE10FA18BFF1
:1086380043F00103002B40F0448491ED007AB4EE3E
:10864800677AF1EE10FA40F03C84294DD4F89C107A
:108658002B68994200F23C843B78012B3FF4EEA949
:1086680094F89B20002A3FF4E9A90B2B0DD801228E
:108678009A4040F6030112EA01060BD112F4C06FCA
:1086880003D0093B012B41F21A80184B2A685A6023
:108698000B233B70002384F89B30FFF7CFB9F9F721
:1086A80093FF0790FEF785BD0CA81EF089FE9DF884
:1086B8003330AB2B04BF02236B76FFF7EAB900BF58
:1086C800F4520020DB0FC940E4CB1641E4CB16C1BD
:1086D800DB0FC93FDB0F494092E741B99730083CAF
:1086E80015A82ABE848D0020C0360020D43600206C
:1086F8003C4500207C4A0020E83F0020EC3E00205A
:10870800A46A0020DB0FC9BFDB0F49C000000000CE
:108718003068FAF71FFC49463A2019F0FFF88146FD
:108728000CA81EF04DFEB9F1000F07D019F05AF948
:1087380019F020F995F82420FFF75AB819F052F9E2
:108748000C9B1BBAC3F38073AB76FFF7C9B91FED57
:10875800137AF4EEC76AF1EE10FA44BF1FED167AE9
:1087680077EE666A6CE61FED177AD5ED037A77EE39
:10877800877AC5ED037AFEF7F0BDAD4A41F2B5132D
:10878800D35C002B00F0BA8794F89B3001223A7032
:10879800002B3FF453A97DE7F7EE006AFEF7FCBF14
:1087A800F7EE006AFEF77FBFA249D1F800C0BCF916
:1087B80036E0FFF7BEBB07EE906ADFED9F6AB8EEC2
:1087C800E77A66EEA65A9FED9D5A9FED9D6ADFED0A
:1087D8009D7AA5EE856A26EEA55AE5EE867AE5EE3F
:1087E800276A26EE870A4BE5B4F91410A279A8EB9C
:1087F800010686EAE670A0EBE670904240F37482C8
:108808008845C8BF524207EE902A95ED037AA361C6
:10881800F8EEE77A012077EE277A2077C5ED037A1C
:10882800FEF78CBD1A2013F011FED0B1864B1B88C1
:10883800BBB9864B45201D681DF07AFF0E201DF040
:1088480077FF284610F006F9059D284610F002F932
:108858007F4A4FF480510A23284611803B7010F05C
:108868009BF910F097FCB2786EE61DF0E3FE794BA9
:1088780093ED000A27F070FC774B93ED000A8046D1
:1088880027F06AFC814640201DF0B6FE002840F023
:108898008C80724D724A2B6892F801E0492B00F2E5
:1088A8009B85DFE813F039072E07F606F006E90680
:1088B800E206DB06D406CB06BF06610A570A500A51
:1088C800420A3B0A340A2D0A220A170A0C0A010A2C
:1088D800F609EB09E009D509C409EA08DA08CA0863
:1088E800BA08AA089A088A087A08720862085A0810
:1088F80052084A0842083A08310828081F08170889
:108908000F080608FD07F507ED07890781077B07AC
:1089180075076E07670760075807BC09A909A20908
:108928009B0994098D09380931092A0923091C0969
:1089380015090E0907090109FA081DF07BFE494BC4
:10894800002105208DE80300A3F1080202915320BD
:1089580010F040FC48BB414BB278186008233B70CC
:10896800F2E51DF067FE404A0292A2F10C032921AC
:1089780001930091A2F10A035021163A492010F000
:1089880029FC90B9354BB27818604FF0FF31596027
:1089980007233B70D8E5314D1DF04CFE334A6B6818
:1089A800126864339342C0F02585B278CCE5022A78
:1089B80000F0B1832D4B29491B684B602C480023DC
:1089C8000B60032103603970BEE52A4B1B78D90779
:1089D8007FF5BAAD80201CF01BF808B10BF05AFAED
:1089E80010F0E2FCB278AFE5234B1B78002B00F0C7
:1089F8008A821A2013F02AFD002840F0848294F815
:108A08009B30002B40F07F8209233B7029E741F21D
:108A180070133C46EB5C002B3FF408A8174822F083
:108A2800F9FEFFF703B803233C466B70FEF7FEBF61
:108A3800F4520020A484002084F9223F92E741B92F
:108A48009730083C15A82ABE3A3500203C3500204E
:108A58002635002048350020DC3F0020D436002091
:108A68008E840020242A0308462803083C45002059
:108A78003C6B00209B4400204C370020646400209D
:108A88002B690622652BAA7032D92A78032A14BFCB
:108A98006FF0FF026FF07F02A3F1650303EA0203A0
:108AA80003F1010314BF4FF4807280229A422B61B4
:108AB8001ED23268EC6802321E19964280F0778521
:108AC800CF4A6C60D16FAE60490203FB01F3052108
:108AD800146042F81C3C42F8183CA970AA68C949BD
:108AE800012022F003FB012840F056850623AB70D5
:108AF8000021C54821F06EFE012840F04D85AB7875
:108B08000133DBB2AB7055E400230DF1300949465F
:108B18001846092218F074FF01283C467EF486AFF7
:108B28000C9A92F8FE31552B00F0508241F2B412A3
:108B380002210123A9546B70FEF778BFB34B009351
:108B48000320A87030230522B149AF483C4622F0E3
:108B58003BFAFEF76BBF2A782B7DAE4EDFF8A4A256
:108B6800032A14BF4FF480794FF08009002B3ED0C0
:108B7800012BFBD1A84BD5F804C01B6832684FEA1B
:108B8800432E00244FF0FF33B3FBFEFE1EEB0C0018
:108B980044F100010024A14202F1020208BF904200
:108BA80038BF0CEB0E029D49022019F069F8032822
:108BB80000F2C581DFE800F0020502053C46FEF739
:108BC80035BF6C68AB6829691A1B8A4284BFEC60A0
:108BD8002A6103283FF454AF0133B3FBF9F209FBD0
:108BE80012320AB14B449B1A00226B602A75326814
:108BF80051460232002019F043F8032800F29F8101
:108C080001A353F820F000BFC58B00085F8C000853
:108C1800C58B0008898A00083C460DF1300941F2ED
:108C2800FC164946A8590023092218F0E9FE012834
:108C38007EF4FCAE00230C9A2B70B2F80B30B3F51F
:108C4800007F00F0438441F2B41203210123A954A8
:108C58006B70FEF7EBBE6B6885F814800133AB6070
:108C680088E704212C2024F025FC032106904E20BF
:108C780024F020FC0C210490362024F01BFC049ADC
:108C8800069B911C421C8A4009FA03F3A2FB0301CC
:108C9800420A42EAC152EA63FEF745BE604822F042
:108CA800B9FDFEF792BF5F4822F0B4FDFEF799BF09
:108CB8005D4822F0AFFDFEF78EBFBCF838109FED7F
:108CC8005B7A07EE901AF8EEE77A594967EE877AE9
:108CD800C1ED007AFEF748BBB0EE677AFFF72BB814
:108CE800F0EE477AFFF73DB8227F12B1626A237728
:108CF800226223690B44B3F5FA6FA8BF4FF4FA63F5
:108D0800B3F57A7FB8BF4FF47A7307EE903AF8EE6E
:108D1800E77AC5ED037AFEF711BB237F002B3FF4FA
:108D2800EFAA636A84F82C2022772362FFF7E8BA57
:108D380095ED000A0493069227F00EFA3D49DFF8F4
:108D480014C1D1F8EC10DFF810E1069AAEF8000073
:108D58008CFB013CC917C1EBAC1107EE901AF8EE79
:108D6800E77A049BFDEEE77A17EE901AAEF8021048
:108D7800FEF752BB07EE905ADFED2F6A9FED377A68
:108D880084F88C50F8EEE77A67EEA67A77EE876A71
:108D9800BDEEE66A16EE103A2033402B40F26881A9
:108DA800DFED266A264BBDEEE77AC3ED006A17EEC3
:108DB800103A2033402B00F258819FED297AF4EEC7
:108DC800C77AF1EE10FA40F32984DFED1E5A9FEDC1
:108DD8001E6A01E0F0EE477AF4EEC67AF1EE10FA78
:108DE80037EEE57AF6DCDFED197AB4EEE77AF1EEE4
:108DF80010FA40F11084DFED135A9FED156A39E03F
:108E080088640020F85200206464002029A5020824
:108E1800204F0308FC64002004650020FC52002059
:108E2800AC640020DC630020986300206F12833A52
:108E380028000020AC16002035FA8E3C0000000007
:108E480020000020DB0FC940E4CB1641DB0F49C0EE
:108E5800E4CB16C1D34D6210E4410020DB0FC93FBB
:108E6800DB0F494092E741B99730083C15A82ABE64
:108E7800B0EE677AB4EEC67AF1EE10FA77EE257A9C
:108E8800F6D41FED0A7AF4EEC77AF1EE10FA40F341
:108E980036811FED0D7A77EE677A67EEA75A1FEDD8
:108EA8000F5A1FED0F6A1FED0F7AA5EE856A27EEA0
:108EB800A55AA5EE867AE5EE077AC4ED247AFFF77F
:108EC800DFB8A04B1B6803F59C530833C4F89C30EB
:108ED8003B78012B7EF4B2AD94F89B30002B7EF4E6
:108EE800ADAD032A00F0DC8310F05EFA012384F8AC
:108EF8009B30FEF7A3BDF0EE476AFFF795BAB0EED8
:108F0800667AFFF77BBA05980FF046FEA9E485F864
:108F18002430FEF78BBD8B4BEE681B686B61072313
:108F280085F82430002E3EF481AD2B692A686968E3
:108F38000120B04795F82420531EFEF76EBD2B7D07
:108F480014E6DFED817AF4EEE76AF1EE10FA40F309
:108F5800D283DFED7E5A9FED7E6A01E0F0EE676A0C
:108F6800F4EEC66AF1EE10FA76EEE57AF6DCDFED9D
:108F7800796AF4EEE67AF1EE10FA40F1B283DFEDA9
:108F8800735A9FED756A01E0F0EE667AF4EEC67AE0
:108F9800F1EE10FA77EEA56AF6D4DFED707AF4EE0A
:108FA800E76AF1EE10FA04DDDFED677A77EEE66A3C
:108FB80007E4DFED6B7AF4EEE76AF1EE10FA44BFEE
:108FC800DFED647A77EEE66AFFF7FBBB92F8FF31D4
:108FD800AA2B7FF4ABADD2F8C6314BB192F8C211CF
:108FE800A1F10B0001282DD901F0F701062929D09C
:108FF800D2F8D6314BB192F8D211A1F10B00012869
:1090080020D901F0F70106291CD0D2F8E6314BB17E
:1090180092F8E211A1F10B00012813D901F0F70130
:1090280006290FD0D2F8F631002B3FF47FAD92F825
:10903800F221A2F10B01012904D902F0F702062A54
:109048007FF474AD41F2FC1101226B50AA70E6E581
:10905800444B1B78002B40F0F881434B1B8B07EEE9
:10906800903AF8EEE77AFFF781BADFED407A24E725
:10907800F4EEC77AF1EE10FA40F3B682DFED335A18
:109088009FED336A01E0F0EE476AF4EEC66AF1EE4E
:1090980010FA36EEE57AF6DCDFED2E6AB4EEE67A03
:1090A800F1EE10FA40F19D82DFED285A9FED2A6A11
:1090B80001E0B0EE667AB4EEC67AF1EE10FA77EE19
:1090C800256AF6D49FED257AF4EEC76AF1EE10FA18
:1090D80040F3BF819FED1C7A77EE666A66EEA65A6A
:1090E8009FED235A9FED236A9FED237AA5EE856AAB
:1090F80026EEA55AA5EE867AE5EE076A52E69FEDBA
:10910800187AF4EEC77AF1EE10FA44BF9FED117A9F
:1091180077EE677AC1E6DFF8648098F81430052B9B
:109128003FF643AC01A252F823F000BF9D9300081C
:10913800B389000821930008E79100081D920008F0
:10914800DB9300083C450020DB0F4940DB0FC9409A
:10915800E4CB1641DB0F49C0E4CB16C1DB0FC93F96
:10916800DB0FC9BF744500204C45002000000000FB
:1091780092E741B99730083C15A82ABEA46A002096
:10918800D8F8042092F91A104B1C5C460AD0BF4B41
:1091980001F5817103EB0113FF20D9796FF3000109
:1091A800D971907692F91B104D1C15D0B74D01F569
:1091B800817105EB011305EB0115DB79E979C3F33F
:1091C8004503012BC6BF03F1FF33DBB20023FF20A9
:1091D80063F34601E971D076032388F81430AC486C
:1091E800D8F804100378002B7FF4DFAB002900F0D7
:1091F800998291F82830002B7FF4D7AB2838442285
:1092080026F036FE0021D8F8040021F097FB002351
:10921800C8F80430D8F81050DFF894A2DFF894E2C8
:10922800DFF894C29B4B05F1010BAAFB0B59ACFB71
:109238000B5CAEFB0BE50695974DA5FB0BE508957A
:10924800069D0FCBAD090995089D4FEAD90E4FEA47
:109258005C1C6D0B0DF13009CDF810C00695AAFB0A
:109268000EC5CC46ACE80700049A8CF80030AAFB7F
:1092780002020998D20801460892ED08AAFB0112D9
:10928800069905EB8505AEEB4505AAFB011AD10841
:10929800089A089501EB8101049DA0EB41014FEA72
:1092A800DA0A069802EB8202A5EB42020AEB8A0A66
:1092B800764D41F2A403A0EB4A0A0EEB8E0E0898F5
:1092C800EB5CABEB4E0E0EF1300C303001F1300E92
:1092D80030320AF1300A01218DF836008DF837C096
:1092E8008DF835208DF834E08DF833A088F8141007
:1092F800002B00F0808141F2E803EB5C002B00F0CA
:10930800798141F22C13EB5C002B00F0D08104230F
:1093180088F81430FFF749BB604DDFF8A091DFF8FB
:10932800A0A1A3460BAA2946D8F8040021F0CCF93D
:10933800012849464FF0030240F059810B9C204612
:10934800002C3FF41DAF2378002B3FF419AF29F010
:1093580082F8032251460028E4D104F1080029F0DC
:109368007AF803460028DDD154F8030F0C902279CF
:109378008DF834200CA88DF8353026F051FDD8F83A
:109388001030984203D90CA826F04AFD0346C8F8C5
:109398001030C7E73D4D6B78032B7FF406AB41F2E5
:1093A800A4020123AA5C88F81430002A00F0D181B5
:1093B80041F2E802AA5C002A00F0BC8141F22C13B9
:1093C800EB5C002B00F0B581002388F81430FFF720
:1093D800ECBAB278FFF7EEBA1DF06AF900283FF44C
:1093E800E4AA2F4BB2784FF4805119800A233B70BE
:1093F800FFF7AAB840201DF0FFF800287FF4D5AA8F
:109408002B68DFF8C080DFF8C0A04FF040090DE0FE
:109418001DF08EF9DAF800202B68013A0133B9F112
:109428000109CAF800202B6000F0438118F80330C6
:109438001846002BECD100234FF0FF322B60042399
:109448006A603B70B278FFF77FB8DFED167AFFF7F6
:109458008DB89FED157AF4EEC76AF1EE10FA44BFA5
:109468009FED127A77EE666A38E600F0B38004233F
:1094780085F82430FEF73EBB0021D8F8000021F023
:109488005DFA00287FF448A8FFF78FBAF45200204D
:10949800D4640020005403085917B7D1AC6A0020DF
:1094A8002635002000000000DB0FC9BFDB0F49C0D4
:1094B800CDCCCCCCD34D62101F85EB51344F030873
:1094C800384F0308D02703083C6B0020137C022B7D
:1094D8007FF4B9AB92F8FE31552B7FF4B4AB92F818
:1094E800FF31AA2B7FF4AFABD189AF59B64B0F44EC
:1094F8001F60567B41F21020731E7F2B2E503FF6C3
:10950800A2AB734236EA03037FF49DAB41F2182005
:109518007302013B2B50D08A00B9506ADFF85CE334
:1095280041F20423E850B2F811305B0103F2FF1353
:109538005B12CEF80030B2F813C0BCF1000F01D1B5
:10954800D2F820C0400019440144ACEB010141F2BB
:10955800082E40F6F47CB1FBF6F1614545F80E1093
:1095680040F2BB804FF6F476B14240F2BD80032151
:109578002970D26A95493B44184441F20C2641F2BD
:109588001C230978A851EA5009B922F015F9AB78DB
:109598000133AB70FEF74ABA02283C467EF446AA6D
:1095A80041F2B4120123AB546B70FEF73FBA20F0BE
:1095B800D5FF2B69FFF784BA854D28681BF0A0FBFF
:1095C800844B1B780022022B2A6000F09180B2782D
:1095D800FEF7B8BF18F008F902287EF48DAAFEF746
:1095E80089BAF0EE476A6DE5B0EE667A54E55C46F6
:1095F800FFF7DBB90B4603EB031305EB830000F51C
:109608008550754B009349463C232022043021F0B5
:10961800DBFCFFF7CAB9F0EE477A32E4B0EE677ABE
:10962800FFF7E1BB6D4B6E491A8A6E480FF088FA56
:109638002B68B27801332B60FEF786BF1FFA89F3D7
:109648001FFA88F2684969480FF07AFAF0E74FF094
:109658007E52674967480FF073FAE9E7664B674936
:10966800DA8A67480FF06CFAE2E7634B63499A8A33
:1096780064480FF065FADBE773783278624963482B
:109688000FF05EFAD4E7624A624963480FF058FA6D
:10969800CEE7624B624A634963480FF051FAC7E765
:1096A80080201BF0B5F900287EF4C8A91CE4022329
:1096B800A1E718F80330002B7FF477A9BBE6452013
:1096C8001DF036F8FF201DF033F858481DF004F857
:1096D80030461DF02DF8FEF7D8BF01232B70FFF799
:1096E800B2BAF0EE676A58E402222A70002241E713
:1096F8000AF0E8FB6BE7F0EE667A38E40222FEF740
:1097080026BF4B4A4B4B019200934B4A4B4B4C495B
:109718004C480FF015FA8BE7474A3E494A480FF084
:109728000FFA85E722F048F800287FF46BADFFF7C1
:109738003CB90223442202FB035303F58550434BF3
:109748000093102213234249043021F03DFCFFF717
:109758002CB91346EEE73F4A2349D3893E4852893C
:109768000FF0EEF964E73B4B24495A793B480FF078
:10977800E7F95DE7374B21491A7939480FF0E0F9E5
:1097880056E7344B1D49DA7836480FF0D9F94FE7D8
:1097980062791A4934480FF0D3F949E72279174911
:1097A80032480FF0CDF943E7314B14491B68314873
:1097B8009A8D0FF0C5F93BE72D4B10491B682E48D1
:1097C8005A8D0FF0BDF933E7F4640020D46400200B
:1097D800406B0020DD360020955B0208084200201F
:1097E80020790308145003080050030808500308A0
:1097F800EC4F0308F44F03084C450020D04F0308F2
:10980800E04F0308D44F0308BC4F0308C44F0308B4
:1098180092840020484F0308B04F0308704D030896
:10982800644D0308984F0308A04F0308F453030836
:10983800884F03087C4D03083C4F03085C4F03081E
:10984800644F0308744F03084C4F0308DD65020892
:109858002C4F03080C700020B8520308A8520308C4
:109868009452030888520308785203087C5203086C
:10987800A48400206452030854520308146500208D
:10988800A84BA9491B68A948DA8F0FF059F9CFE608
:10989800A44BA5491B68A6489A8F0FF051F9C7E653
:1098A800A04BA1491B68A34893F83B200FF048F947
:1098B800BEE69C4B9C491B689F4893F83A200FF0E2
:1098C8003FF9B5E6974B98491B689C481A8F0FF0EB
:1098D80037F9ADE6934B94491B689948DA8E0FF037
:1098E8002FF9A5E68F4B90491B68964893F83020CE
:1098F8000FF026F99CE68B4B8B491B68924893F82E
:109908002F200FF01DF993E6864B87491B688F4877
:1099180093F828200FF014F98AE6824B82491B68D5
:109928008B48DA8C0FF00CF982E67E4B7E491B6877
:1099380088489A8C0FF004F97AE67A4B7A491B68C2
:1099480085485A8C0FF0FCF872E6764B76491B680E
:1099580082481A8C0FF0F4F86AE6724B72491B6859
:109968007F489A7F0FF0ECF862E66E4B7D49D3F89A
:1099780000E07D489EF81C309EF81B209EF81DE0F4
:10998800CDF800E00FF0DCF852E6664B66491B683C
:1099980076481A7E0FF0D4F84AE6624B7149D3F83C
:1099A80000E073489EF816309EF815209EF817E0E0
:1099B800CDF800E00FF0C4F83AE65A4B6949D3F8FD
:1099C80000E06C489EF813309EF812209EF814E0D0
:1099D800CDF800E00FF0B4F82AE6524B6149D3F80D
:1099E80000E065489EF810309EF80F209EF811E0C0
:1099F800CDF800E00FF0A4F81AE64A4B5949D3F81D
:109A080000E05E489EF80D309EF80C209EF80EE0AF
:109A1800CDF800E00FF094F80AE6424B5149D3F82C
:109A280000E057489EF80A309EF809209EF80BE09F
:109A3800CDF800E00FF084F8FAE53A4B4949D3F83D
:109A480000E050489EF807309EF806209EF808E08F
:109A5800CDF800E00FF074F8EAE5324B4149D3F84D
:109A680000E049489EF804309EF803209EF805E07F
:109A7800CDF800E00FF064F8DAE52A4B3949D3F85D
:109A880000E042489EF801309EF800209EF802E06F
:109A9800CDF800E00FF054F8CAE53D4B22491A68AA
:109AA8003C480FF04DF8C3E592781F493A480FF04B
:109AB80047F8BDE5394B1C495A8A39480FF040F838
:109AC800B6E5364B18491A8836480FF039F8AFE52D
:109AD800324B15499A7834480FF032F8A8E52F4BE5
:109AE80011491A7931480FF02BF8A1E59BF80820A5
:109AF8000D492F480FF024F89AE5BBF824200A49AD
:109B08002C480FF01DF893E59BF8202006492A48B9
:109B18000FF016F88CE59BF81E20034927480FF034
:109B28000FF885E5A4840020D04F030848520308A5
:109B3800385203082052030804520308F05103085E
:109B4800D8510308C4510308B4510308A4510308A9
:109B580090510308805103087451030864510308A5
:109B680050510308E45003084851030840510308C2
:109B7800345103082C510308245103081C510308CD
:109B8800145103080C51030800510308F850030846
:109B9800808D0020E8530308DC5303084C4500205F
:109BA800C8530308B8530308A45303089053030881
:109BB8007C530308605303084453030830530308D5
:109BC80094F898206F4970480EF0BAFF30E56F4B53
:109BD8006C49DA786E480EF0B3FF29E56D4B694998
:109BE8001A786D480EF0ACFF22E56C4B6549DA78BF
:109BF8006B480EF0A5FF1BE5684B9FED6A7A1B8842
:109C08006049694807EE903AF8EEE77A67EE877A96
:109C1800FDEEE77A17EE902A0EF092FF08E5634A08
:109C28006349138A634892890EF08AFF00E5624B04
:109C3800624963480C2202FB0E3E9EF806309EF8ED
:109C480005209EF807E0CDF800E00EF079FFEFE47C
:109C5800594A4C495B480C2303FB0E2EBEF80A20D8
:109C68000EF06EFFE4E4544A464957480C2303FBC0
:109C78000E2E9EF808200EF063FFD9E44E4A4149A3
:109C880052480C2303FB0E2E9EF804200EF058FFBA
:109C9800CEE4494A3B494E480C2303FB0E2E9EF85E
:109CA80003200EF04DFFC3E4434A364949480C23CC
:109CB80003FB0E2E9EF809200EF042FFB8E43E4A40
:109CC800304945480C2303FB0E2E9EF801200EF068
:109CD80037FFADE4384A2B4940480C2303FB0E2ECE
:109CE8009EF802200EF02CFFA2E40C2303FB0EFECC
:109CF800314B244913F80E2039480EF021FF97E420
:109D0800384B20491A7838480EF01AFF90E4274B50
:109D18001C499A7835480EF013FF89E4344B1949E9
:109D28001A6834480EF00CFF82E4334B5B79012B40
:109D38007FF47EACB4F99430B4F996201C492F48CE
:109D48000EF0FEFE74E42E4B2E491A882E480EF0B3
:109D5800F7FE6DE428482D49837842780078009012
:109D68002B480EF0EDFE63E42A4B1B68D80402D49E
:109D78000C232B605CE4284B22491A7827480EF004
:109D8800DFFE55E4D04F030818530308643700205A
:109D98000853030874370020F8520308843400205D
:109DA800E85203080000C842DC5203080C70002087
:109DB80000500308C8520308A8840020E450030890
:109DC800F0500308D4500308C8500308BC500308D7
:109DD800B4500308A85003089C5003089450030883
:109DE8008C500308087B002078500308685003084B
:109DF800447800205C500308784100204C50030848
:109E080044350020207903084450030828500308EB
:109E180034500308403500205F8C00201C50030894
:109E28002DE9F04F9A4A9B49137895B0044609905A
:109E380000F59C4020300C900860002B00F07C84DA
:109E4800954909688C4240F29680944905910968C1
:109E58009348944CDFF888B20391013B137001F4E6
:109E6800805302900893002B40F09480029B5B7D06
:109E7800002B40F06283039B1E0400F11086039BB5
:109E8800DD050BD5099A884BDFF858A29A429AF853
:109E9800022000F2CD87002A40F0CE87834B04933E
:109EA800834D039B13F4805740F06783029BBBF9F3
:109EB80006605B8B9E42B4BF002601267D4B1B6863
:109EC80013F0805373D0049A127812F0010275D0FF
:109ED80002987949808C91ED037A07EE900AF8EEA2
:109EE800E77AB4EEE77AF1EE10FA80F2B086002E47
:109EF80069D194F8A410002965D1704870490068A8
:109F080090F830004FF0000EC1F800E0C1F804E00E
:109F1800C1F808E06B49002856D10870002A57D0CC
:109F2800039AD10654D5684A1278D20650D4002F25
:109F38004ED1002B4CD1039B5B0249D495F800C04D
:109F4800BCF1000F01F05785604B9B78002E41F063
:109F58008F853BB15E4A5F4B12681B689B1A002BCA
:109F6800C1F29D8510201BF0C1FB012384F8A530A8
:109F780095F800C02EE0494B05931B680393484AA7
:109F8800484C029203F48053DFF854B10893002B35
:109F98003FF46CAF00214748FAF708F900287FF42E
:109FA80065AF10F06FFB059B1B6803935EE7039A90
:109FB800500288D4049A127802F00102002184F831
:109FC800A410002E99D03F4901200870002AA7D17B
:109FD80095F800C0029ABBF900E0508B918BBBF951
:109FE80002208645CCBF8027002747F040038E45D6
:109FF800A8BF3B469B0843F080078242C8BF3B4648
:10A0080043F040078A42B4BF3A461A469208BBF961
:10A0180004E0BBF9067042F080038645C8BF1A46C3
:10A0280042F040038E45A8BF13469B0843F08002C8
:10A038008742D4BF1846104640F0400294F8A63034
:10A048008F42ACBF014611468B4200F018840023B2
:10A0580084F8A61084F8A730BCF1000F00F0A5859D
:10A06800059B1D4A1B68039203F00403002B40F074
:10A078000B830DF14808194D0023C8F8043005F189
:10A088005009129340F6330A192740F283362EE01E
:10A0980068320020DC300020643200207C4A002036
:10A0A8004C4A0020741E0020404B4C009B4400206A
:10A0B8003702002030350020F8850020A4840020D5
:10A0C800083400206025002038350020541E002068
:10A0D8003C45002040380020B47C0020FC3600209D
:10A0E8003C8B00208441002004354D4520D0AA78BF
:10A0F800EB789A4217FB0260F6D26978043117FBB5
:10A1080003623BF911305345A8BF5346B3F5617F4D
:10A11800B8BF4FF461739842E6DA9A42E4DB2978D3
:10A128002329E1D840460435F7F7B8F84D45DED184
:10A13800AB4B98E803001E78AA4B83E80300002E77
:10A1480000F032820121A748FAF730F8002840F0E1
:10A158000C81059B1B68DC0500F10281A24C238859
:10A168001DB225F00105AFB2BB42278000F0FB838A
:10A178009E4D02260F204FF014094FF0FF082E7055
:10A1880085F8019085F802801BF0B0FA31469548B1
:10A198002788FAF70BF8002840F0958727F0020384
:10A1A8009BB2BB4223800AD0904B1421FF22022588
:10A1B8000F201D7059709A701BF098FA27888C4BE5
:10A1C80002931978DFF850A2BB0708BF81F002019B
:10A1D800DAF80400C1F34001F8F7C8FE039B1B68D6
:10A1E80013F00A0F24D005217E48F9F7DFFF002875
:10A1F80000F0C68425886F0740F1E8867948062173
:10A20800F9F7D4FF002800F0A8846E0640F1FB8619
:10A2180007217448F9F7CAFF50B1764B764AB3F96B
:10A228000430764982FB0302DB17C3EBA2030B80E1
:10A238000C216C48F9F7BAFF2288002800F0B18099
:10A2480042F480739A42238009D0684B0225142176
:10A25800FF220F201D7059709A701BF047FA684B47
:10A268001B78082B00F0A9800E2B00F0A680059B18
:10A278001B685D0542D5634B1B79002B58D0142110
:10A288005848F9F793FF002856D122F0E3FB012044
:10A298001BF07EF990B3DFF8848100254FF0CC09DC
:10A2A80002E0DDB2022D29D809FB05F76B1C58F82E
:10A2B8000760002EF5D1C378534A90F9020052F88E
:10A2C8002330019603220092012132461AF042FD02
:10A2D800034605EB450000EB0010059353B13146EA
:10A2E80008EB8000CC2228F044F8059B48F807309A
:10A2F8000135EDB21DF0FCF80028D3D1049B1B7882
:10A30800D80740F18D804149414A01230B701370F1
:10A31800029BDAF80000197801F00101F8F726FE2F
:10A32800039B1B685B0700F1EB8015B0BDE8F08F5D
:10A33800049B1B78D907A8D53C201AF069FB002894
:10A34800DCD009F0A7FD3C201AF004FB0028D5D08A
:10A3580009F0A0FD3C201AF0FDFA0028F1D1CDE764
:10A368002C4BDB78002B3FF4F9AE039B1B68980756
:10A378007FF5F4AE1C4C2788F9073FF50FAF47F07F
:10A3880001039F4223803FF409AF184B1421FF2299
:10A3980002250F201D7059709A701BF0A7F92788A5
:10A3A800FCE622F480739BB29A4223807FF44DAF7F
:10A3B800134B1B78082B7FF457AF228822F04003F9
:10A3C8009BB29A4223803FF452AF084B02251421D6
:10A3D800FF220F201D7059709A701BF087F946E70D
:10A3E800E341002030350020D84100200C400020F7
:10A3F800064500205C42002067666666C61D002090
:10A40800F8360020E8850020044603089C44002014
:10A41800F41D0020844100200845002034870020D6
:10A42800AA4B93F80090B9F1000F5FD1DFF80083D1
:10A43800A74F18F8030C3E784146A8F1030511F020
:10A44800DBFF002800F0D482002E40F0268305F1BF
:10A458000801687911F0D0FF002841F0D1819D49A9
:10A46800A87A11F0C9FF002800F0D582022E41F029
:10A47800CB819949E87B11F0BFFF002841F0B081FA
:10A488009649287D11F0B8FF002800F0D582042EE7
:10A4980041F0AA819249687E11F0AEFF002841F090
:10A4A800A7819049A87F11F0A7FF002800F0D58266
:10A4B800062E41F0A1818C4995F8230011F09CFFEC
:10A4C800002840F0E886894995F8280011F094FFA3
:10A4D800002800F0D582082E40F0F386844995F8CC
:10A4E8002D0011F089FF002840F0D582814B012210
:10A4F8001A7024F05BFC039B1B685B077FF515AFA4
:10A50800032011F0A3FF002800F0F185238813F041
:10A5180008047FF40AAF08201BF0F6F97648774D57
:10A528007749784A784BBBF8066000682E80086047
:10A5380014601C6015B0BDE8F08F029A013BD27D13
:10A548003BF91330002A40F04983A3F57A73B3F539
:10A558007A7FA8BF4FF47A7323EAE37307EE903A41
:10A568009FED6A7AF8EEE77A67EE877A684AFCEE3A
:10A57800E77A17EE903A138081E41D216548F9F7D0
:10A5880015FE00287FF492AC634A029BD2881B8B8D
:10A59800BBF90660991A8E4240F32F8613449E42F7
:10A5A800B4BF0026012689E4DFF888915B4F09F1E2
:10A5B8005A054FF00108494619F8010C11F01CFF23
:10A5C800F8B199F8040099F8023099F803E000EB23
:10A5D800400104EB8101013BD1F8B42003EB4303B4
:10A5E8003B4493420DD094F8E02081F8B0E008FA9B
:10A5F80000F022EA0000C1F8B430C1F8B86084F86D
:10A60800E00009F10609A945D5D14549454A464B17
:10A618000968D2F8009093F800A0444D06910026EE
:10A628006B685BB31F784FB3AA68A9EB0202002AD4
:10A638000ADB94F8E0200121B14022EA010209F581
:10A64800FA7184F8E020A960BAF1000F16D02A78D0
:10A6580059780432D2B2002940F0FE8202993BF9BF
:10A668001220098B01F1C800824240F39A8594F8C0
:10A67800E0209B783241D10740F1FC850136042E59
:10A6880005F10C05CCD15DE594F8AB3053B1049BD2
:10A698001B78D80706D5029BBBF906205B8B9A422C
:10A6A80000F3DA8511211B48F9F780FD002800F036
:10A6B800B68294F8AE302BB994F8A93013B9322386
:10A6C800A4F8AC30012384F8AE30D2E49C440020D6
:10A6D80024000020E3390020E8390020ED3900206B
:10A6E800F2390020F7390020FC390020013A002017
:10A6F800063A0020F41D0020E01D0020D01D002097
:10A70800DC1D0020D41D0020CC1D0020AAF1823FB2
:10A718007041002030350020E83F0020442A03081B
:10A72800483800203C45002069410020241F0020B3
:10A73800D9390020F1380020994C9A4B2678029399
:10A74800994F002E00F06082B6B1DFF89492DFF8DE
:10A7580094B2DFF85482CA460025072D4046E9B274
:10A768007B6841F3D180984700B20135AE422BF89F
:10A77800020F0AF1040AF0D18C4B05931A46099985
:10A788008B4B12680392A3FB013E42F20103134074
:10A798004FEA9E1E079300F033828648864A874B0D
:10A7A80000788749069012781A70069B08702BB1BA
:10A7B800824B93F800B08BF001030693814A02990B
:10A7C800127838781090B1F82680088D91F822C058
:10A7D8000B92098B0B9A119194F829107A4B0E90D1
:10A7E80008461146A3FB01135B0803EB4303D31A86
:10A7F800DBB20D93039B2578744EDFF8ECB1DFF8DC
:10A80800EC91CDF810800F220CF1040C03F4805366
:10A8180084F828200A945FFA8CFC109C0F92AA46B0
:10A8280008930021804610972DB9A44599BFE246A8
:10A838006546A2462546A94280F29482069B002BD3
:10A8480000F04682624B049833F9112097B2874290
:10A858004FEA410303D30E98874240F2118259F818
:10A868002120964580F03E823BF90320079F002F68
:10A8780040F00E822BF8032001310636D4E794F815
:10A88800A790B9F1F90F00F2DB8109F101095FFA2C
:10A8980089F984F8A79084F8A610BCF1000F00F09D
:10A8A8008581B9F1140F7FF4DBAB5F2940F091810A
:10A8B800049E337813F0010300F04E870FF0E2FE98
:10A8C800337803F00103002B7FF4CAAB94F8A62079
:10A8D800572A00F0C786059B1B6813F0040302D0B3
:10A8E8005A2A00F0F2845D2A00F027875B2A00F0DC
:10A8F8002F875E2A00F0C484562A00F089872B78B7
:10A908002BB16F2A00F09F87324B00211960972ADC
:10A9180000F08D87A72A00F092840021BB2A1291AB
:10A9280000F0CD87B72A00F0AA87BE2A00F0CA87B0
:10A93800BD2A00F0C987792A00F0DF877A2A00F05B
:10A94800D5879E2A00F0CB879D2A00F0C087AE2AC3
:10A9580001F03D80AD2A7FF483ABFF21002016F083
:10A9680022FEFFF77DBB02211B48F9F71FFC0028D8
:10A978003FF414AC2580BA073FF521AC47F0020339
:10A98800BB4223803FF41BAC144B02201421FF224E
:10A9980018700F2059709A701AF0A8FE27880EE4D4
:10A9A800741E00204C4A0020CC8400207C4A0020E1
:10A9B800D34D6210B8300020B4010020B50100204A
:10A9C8006941002069320020ABAAAAAAA01E002073
:10A9D800781E002044380020303500200C4000202C
:10A9E800D0320020761E00203C8B00206C320020E4
:10A9F80008F10501687911F0FFFC00283FF42FAD3C
:10AA0800012E40F0FD8605F10D01A87A11F0F4FC45
:10AA1800002840F0F986C249E87B11F0EDFC0028D7
:10AA28003FF42EAD032E40F0DB86BE49287D11F0A1
:10AA3800E3FC002840F0D886BB49687E11F0DCFCB6
:10AA480000283FF42EAD052E40F0D286B749A87FE6
:10AA580011F0D2FC002840F0CF86B54995F82300C4
:10AA680011F0CAFC00283FF42EAD072E40F01384E5
:10AA7800B04995F8280011F0BFFC002840F0218467
:10AA8800AD4995F82D0011F0B7FC00283FF42EAD24
:10AA9800092E3FF42BAD4FF009094B46FEE3D4F8DD
:10AAA8008C30099AD31A002BFFF6E9A9A34A94F827
:10AAB8009030517CA24A029D32F811200C98A97D51
:10AAC800C4F88C00013303F00F0384F8903023445A
:10AAD80092B292FBF1F283F8942094F8940094F8DF
:10AAE800951094F8962094F8973001440A4494F805
:10AAF800980094F899101344184494F89A2094F8FC
:10AB08009B3001440A4494F89C0094F89D10134427
:10AB1800184494F89E2094F89F3001440A4494F80D
:10AB2800A00094F8A1101344184494F8A23094F8A3
:10AB3800A32001440B441A4442F30B12642AE97D12
:10AB4800A8BF642213B209B1C2F1640307EE903AB8
:10AB58009FED7C7AF8EEE77A06E525F040039BB294
:10AB6800AB4223803FF454AB774B02251421FF22DC
:10AB78000F201D7059709A701AF0B8FDFFF748BB86
:10AB8800238823F00405ADB2AB4225803FF436ABF1
:10AB98006D4B02251421FF220F201D7059709A70E9
:10ABA8001AF0A4FD2588FFF729BBE1460021674874
:10ABB800F9F7FCFAB8B1002384F8A8300FF0DEFBEF
:10ABC80094F8A730142B7FF44BAA2B78002B40F075
:10ABD8004787049B1B7803F0010374E6C3F53B63C6
:10ABE80008331BB2B1E4049B594A1B781060DF0795
:10ABF80000F11385B9F1140F3FF468AEFFF730BACE
:10AC0800544B1B780693D2E593F822303E780433F0
:10AC1800DBB2B3428EBF267023701E4694E594F8CB
:10AC2800A930002B3FF425AA049B1B7813F00103DD
:10AC380002BF012284F8A93084F8AA20FFF719BAC4
:10AC480084F8A630BCF1000FB0D0FFF709BA012193
:10AC580084F8A410FFF7B7B9012900F0238594F808
:10AC6800E0200123B34001361343042E84F8E0307A
:10AC780005F10C057FF4D4ACFFF764BA1A464B0013
:10AC88000EF5967749F82170079F002F3FF4F2AD33
:10AC98000D985F1807440A9800EB4707BA85B8F182
:10ACA800000F03D10B9802287FF6E4ADB6F80280B6
:10ACB8003288B78842441744274A3FB282FB0702CA
:10ACC8002648A2EBE772C75212B24FF00108D1E54D
:10ACD800049B002BD2D059F8212096454FEA410316
:10ACE800FFF4C2AD1E4A1E48D25CC718002A00F005
:10ACF8009281022A40F05B817A7802EB820202EBB1
:10AD0800820202F2EE2292B20329DFBF012000FA8A
:10AD180001F70F98B843CEBF12B212B20F90A5E553
:10AD2800E8390020ED390020F2390020F7390020F9
:10AD3800FC390020013A0020063A0020B4440020E3
:10AD4800D044002014AE23410C40002030350020B0
:10AD5800443800206941002056555555E81E00200A
:10AD6800043300200F990A9CB14B109F84F800A06F
:10AD78000F2942460CBF0122002284F8298084F85A
:10AD880028101A7006D11B21AA48F9F70FFA0028D3
:10AD980000F0C584A848A94B82681968A84BC1600F
:10ADA8008A1A012119704368A64E9A42029A317094
:10ADB80088BF002392F8226088BF80F82130089B62
:10ADC8003878B2F826C0B2F818E00436F6B2002B8C
:10ADD80000F0508186429C4A40F2C1819B4E174642
:10ADE80000210DB982460546A94218DA12F8113039
:10ADF80083B1022B0CD17B7803EB830303EB830332
:10AE080003F2EE239BB226F8023B01310237E8E752
:10AE18003388F8E7CBB2032BFAD87346F3E784F804
:10AE280000A00B9B8A4A01331370089BFFF71BB8DD
:10AE380012B901228AF80220864B04931D789AF8E9
:10AE4800218005F001031B20039311F0FFFAB8F1EC
:10AE5800010F079000F0D48105F0020306939AF8D9
:10AE680020207D4DDFF808927C4E744F052A00F2B1
:10AE78009580DFE802F08579032F3E51B8F1010F84
:10AE880004BF05238AF82030039B002B00F09C8028
:10AE9800029B3868B3F91810B9F80230002261F340
:10AEA8000F0263F31F42002361F30F0361F31F4393
:10AEB800DAF81410CBF804208842CBF8003040F2BE
:10AEC80021810323069347F230520323CAF81C203A
:10AED8008AF82030338843F0020333800FF0D2FB26
:10AEE8003A68DAF81C3013440422CAF818308AF891
:10AEF8002020B8F1010F40F024843B68DAF81820CC
:10AF08009A424BD2287818B911F0A0FA002845D1F6
:10AF1800338823F0020333803A68B9F80630642195
:10AF280001FB03234FF4806000228AF820208AF86E
:10AF38000320CAF810301AF0CFFC9AF8202095E7C1
:10AF480011F0B0FA012800F04184079B002B40F073
:10AF58005A81B8F1010F21D03B68DAF810209A42E3
:10AF680028D301238AF82030B8F1010FD4D099F8FA
:10AF78000830012B1ED013F031FB9AF8202075E71A
:10AF8800039B002BDCD1079B4FF48060002B00F063
:10AF9800AB801AF0B9FC0022CAF81020069B002BDF
:10AFA80040F0AC80059B1B680393FEF77BBF3BF822
:10AFB8000320A9E613F012FB032240F6B8338AF8FF
:10AFC8002020CAF81C3085E73B687CE745F004037D
:10AFD8009D4223800AD0224B02251421FF220F20F4
:10AFE8001D7059709A701AF081FB25881D4B1E4AF6
:10AFF800B3F904301D4982FB0302DB17C3EBA2033C
:10B008000B80FFF7FBB845F04003AB4223807FF489
:10B01800ABADFFF7FDB8CAB2022A40F2FB82032AA1
:10B02800C5D1119A0898049F002808BF3A466BE6D4
:10B03800E242002030350020844100203C450020B9
:10B04800B4010020B5010020043300203C8B00200F
:10B05800693200209B44002037020020A8410020CC
:10B068000C4000205C42002067666666BC1D00201C
:10B078000040002086421946B04A4BD8B0481746CF
:10B088000DB9B24635468D427FF7C9AE12F8113078
:10B0980083B1022B0CD17B7803EB830303EB83038F
:10B0A80003F2EE239BB220F8023B01310237E7E7B7
:10B0B8000388F8E7CBB2022B03D9032BF8D16346F8
:10B0C800F1E77346EFE727F001039BB2BB42238009
:10B0D8003FF451AC0F202E7085F8019085F802805E
:10B0E8001AF004FB278846E41AF0F6FB53E7082019
:10B0F8001AF0F2FBFFF719B90323069306981AF022
:10B10800F5FA4FE7B8F1010FF6D103239AF820209A
:10B118000693ABE68A4E17460DB982460546A94204
:10B12800BFF67DAE12F8113083B1022B0CD17B78BB
:10B1380003EB830303EB830303F2EE239BB226F8AE
:10B14800023B01310237E7E73388F8E7CBB2022B3D
:10B1580003D9032BF8D16346F1E77346EFE7784844
:10B16800174600210DB9B24635468D427FF757AED6
:10B1780012F8113083B1022B0CD17B7803EB8303D7
:10B1880003EB830303F2EE239BB220F8023B013169
:10B198000237E7E70388F8E7CBB2032BFAD8734600
:10B1A800F3E7C8398A423DDA94F8E0209B783241C7
:10B1B800D2073FF563AAC3F1000801201AF074FB17
:10B1C8007A1E162A00F2E780DFE812F0D801EC01B7
:10B1D800C101390100021102AE019B018601710112
:10B1E8005C01E500390149011102AE019B0125010D
:10B1F8001101FD00E800A300D2000126FEF75EBEA3
:10B20800002306932BE699F80430002B3FF4A1AEF7
:10B2180013F0E4F903224FF47A738AF82020CAF86D
:10B228001C3057E694F8E0300122B24023EA0203CA
:10B2380009F5FA7284F8E030AA60FFF71FBA4149AD
:10B24800059B0A781B6842F004020A7003F00403A5
:10B258003D4A0392FEF70ABF00213C48F8F7A6FFD3
:10B2680000287FF41FAA322384F8AB00A4F8AC307E
:10B27800FFF718BA9846002B0CBF012002209DE763
:10B28800334B02220320334D33492A700B601AF0E6
:10B298000BFBFEF7E5BE4FF007094B4603EB8303B4
:10B2A8001D4487F80090A97868781EF0B3FE049BC7
:10B2B8002A4A1B7801211170DA077FF51AA9FFF7CE
:10B2C80027B84FF008094B46E8E794F8A920002A68
:10B2D80040F0A78394F8AB2082F0010284F8AB20F9
:10B2E800002A40F099831E49096811F4003104D0FE
:10B2F8001C490979002940F0AE830A461A48855C42
:10B308000D2D02F10C0200F0498301311529F6D107
:10B318009EE7D4F8E400154B90F83B109A78414426
:10B32800FE29A8BFFE2121EAE17180F83B10002A1E
:10B3380040F0C2831DF0B4FB91E400BF0433002049
:10B348003C8B002038350020B47C002030350020AC
:10B35800048D00208E840020A4840020F41D002089
:10B36800E838002078410020B8300308858D002097
:10B37800D4F8E400B74B90F83A109A78414464291D
:10B38800A8BF642121EAE17180F83A10002AD1D0DF
:10B39800172011F0B9F8D4F8E400CBE7069AAD4BC2
:10B3A80051784144B1F5967FA8BF4FF4967121EAD0
:10B3B800E17151709B78002BEDD0152011F0A4F8A5
:10B3C800D4F8E400B6E7D4F8E4008178A14B41440E
:10B3D800C829A8BFC82121EAE17181709B78002B98
:10B3E800A8D0142011F090F8D4F8E400A2E7D4F81B
:10B3F800E4004178974B4144C829A8BFC82121EAF5
:10B40800E17141709B78002B94D0132011F07CF8E7
:10B41800D4F8E4008EE7D4F8E40001788D4B414479
:10B42800C829A8BFC82121EAE17101709B78002BC7
:10B4380080D0122011F068F8D4F8E4007AE7069872
:10B44800844B81799A7841446429A8BF642121EA10
:10B45800E1718171002A40F0F4820D2F9BD006988B
:10B468007C4B41799A7841446429A8BF642121EA38
:10B47800E1714171002A8ED00E2011F045F8D4F800
:10B48800E40057E7D4F8E400724B017A9A78414413
:10B49800C829A8BFC82121EAE1710172002A3FF436
:10B4A80049AF0B2011F030F8D4F8E40042E7D4F8A3
:10B4B800E400684BC1799A784144C829A8BFC821DB
:10B4C80021EAE171C171002A3FF434AF0A2011F07A
:10B4D8001BF8D4F8E4002DE7D4F8E4005D4B81793B
:10B4E8009A784144C829A8BFC82121EAE17181712D
:10B4F800002A3FF41FAF092011F006F8D4F8E40041
:10B5080018E7D4F8E400534B41799A784144C829A4
:10B51800A8BFC82121EAE1714171002A40F08B825D
:10B52800112F7FF452AF05E7D4F8E400494B0179B5
:10B538009A784144C829A8BFC82121EAE17101715C
:10B54800002A40F0B382102F7FF453AFF2E6069A38
:10B5580017794744642FA8BF642727EAE77717714C
:10B5680010F0ECFF3B4B9B78002B3FF414AF03200B
:10B57800394610F0C9FFD4F8E400DBE6069A354BEB
:10B5880011784144FA29A8BFFA2121EAE171117022
:10B598009B78002B3FF4FFAE012010F0B5FFD4F8E4
:10B5A800E400C7E6069A2B4B917841446429A8BF6A
:10B5B800642121EAE17191709B78002B3FF4EBAE96
:10B5C800022010F0A1FFD4F8E400B3E60698214B5E
:10B5D800C1799A78414481F30801C171002A3FF486
:10B5E800DAAE052010F090FFD4F8E400A2E6D4F813
:10B5F800E400184BC1789A784144C829A8BFC821EB
:10B6080021EAE171C170002A40F01F820F2F7FF4F8
:10B6180004AF8FE6119AFFF777BB0F4B1B78002B0F
:10B628003EF41EAD0D4BDB78002B7EF419AD94F87B
:10B63800A8300133DBB2032B84F8A8307EF610ADB6
:10B64800074B5B7813B9002E7EF40AAD0FF01AF899
:10B65800FFF7B6BA858D002069410020844100209B
:10B66800541E0020BA4ABB4B039210461A68BA49C6
:10B678004FF47A73B3FBF2F3C3EB431203EB820389
:10B688000268DB005507A1F8A83055BF059B059B4C
:10B698001B68B24A42BF1B680A21118003F00403E9
:10B6A800FEF7E4BC3BF912209978B2F5617F4FF4BC
:10B6B800966393FBF1F3C0F2818040F63301914227
:10B6C800A8BF11460C2FA1F5617191FBF3F800F0AA
:10B6D800BE80182F7FF4C3AA5FFA88F1C8290B46E9
:10B6E800A8BFC823D4F8E400C27DDFB297423FF474
:10B6F800B6AA9B1A9A4AC77548BF0733DB109278D7
:10B708005F1CFFB23AB9002F3FF4A9AA38461AF0D5
:10B71800CBF8FFF7A4BA182010F0F6FEF3E791492A
:10B72800914BCA681B688B609B1AC82B7FF679AB54
:10B73800012381F82130FFF774BB8C4B00220120D4
:10B74800A1E53968DAF81C200A44CAF8182025E46B
:10B75800874B0122022096E5864A1268960304D593
:10B76800854A1279002A40F03A81844819461A46D7
:10B77800465C0B2E01F10C0107D00132152AF7D1D6
:10B78800002284F8A720FFF79EB87D4ED6F800E087
:10B798005100BEF1000F07D08F1800EB87079EF805
:10B7A80001E07F787745EBD20A44764F764900EB83
:10B7B80082020020326038800860E1E70C2F5BD0FD
:10B7C800182F7FF44CAA00210B468BE73A68B9F88A
:10B7D8000630642101FB0323CAF81030FFF7B5BB1C
:10B7E8004FF003094B4659E54FF004094B4655E520
:10B7F8004FF005094B4651E54FF006094B464DE51C
:10B808004FF001094B4649E54FF002094B4645E523
:10B818000BF042FDF8F728F80BF026FDF7F746FE87
:10B8280001201AF041F894F8A620FFF768B8059BA4
:10B83800564A1B684FF4C8711180454A039203F0B9
:10B848000403FEF713BC0EF099FDFEF709BC5FFA7E
:10B8580088F74F4B5B78BB423FF401AA38460FF09C
:10B8680093FB3F4B9B7823B15FFA88F10C2010F0D3
:10B878004BFE0137FFB246E70027B846E9E70B461B
:10B888004FF6FE71434A32485589039090892B44FC
:10B898000144538191810BF0FFFCF7F7E5FF0BF0B2
:10B8A800E3FCF7F703FE012019F0FEFF059B1B6878
:10B8B800002203F0040384F8A720FEF7D7BB0B4649
:10B8C8000221DFE70223DDE74FF6FE73DAE7002106
:10B8D800FF2015F068FE94F8A620FFF738B801207D
:10B8E80015F061FE94F8A620FFF72EB82A4A137ABD
:10B8F80043F001031372FEF7B3BB274A137A23F010
:10B9080001031372FEF7ACBB029A515D9847032DF1
:10B918001BDC40F2EE2240F6CA0C00283EF425AFAC
:10B9280039F825E0BAF802104FF47A73A0EB0E004C
:10B9380003FB00F0A1EB0E0190FBF1F018449042DC
:10B94800B8BF10466045A8BF604600B2FEF70DBFFD
:10B95800B47C00204478002020700020249300202C
:10B96800858D0020844100203C450020708C0020FB
:10B97800BA8C0020E838002078410020B83003084D
:10B9880010250020A6250020A825002026930020A9
:10B998008E84002084340020C8420020494E376835
:10B9A8004A003FB1551800EB85057F786D78BD4298
:10B9B800BFF44EAC0A4400EB8202434F434D326061
:10B9C8000021434A398029600392FEF74FBB0121C9
:10B9D800002015F0E8FD94F8A620FEF7BBBF3D4A0D
:10B9E8001278002A7FF4C1AE19F064FE049B1B781C
:10B9F80003F00103C4E6002E3EF4B4AA94F8A5C0EF
:10BA0800BCF1000F3EF4E6AA19F054FE95F800C008
:10BA180084F8A570FEF7DEBA0C2019F067FEFEF771
:10BA28001FBB0122002184F8AA20294A84F8A91002
:10BA38000392FEF71BBB112010F066FDD4F8E4005A
:10BA48006EE50D2010F060FD07E50F2010F05CFD9D
:10BA5800D4F8E400DAE51F49097829B111464DE424
:10BA680094F8A610FEF721BF19F024FEFEF7F8BAE5
:10BA78003BB11949194A09684FF47A7000FB03135E
:10BA8800136094F8A530002B3EF4A4AA19F012FE16
:10BA9800002384F8A53095F800C0FEF79BBA0EF095
:10BAA800F1FD002384F8A530FEF792BA102010F0BB
:10BAB8002BFDD4F8E40046E5162010F025FDD4F857
:10BAC800E40037E410250020A6250020A825002042
:10BAD800B47C0020F68500203C450020403800203A
:10BAE800F8B55D4B1B78DB072DD55C4B5C4D1C789E
:10BAF8005C4E012C49D079D3022C1BD06B7A7BB1D8
:10BB0800EB886BB1584B1B7853B107F023FF002823
:10BB18007CD0AB7A83422CBF01230023337000E032
:10BB2800337852492A7A9C4238BF1C460C70002A46
:10BB380053D1F8BD4E494F4A098812889142DDD940
:10BB480001241C70DAE74A4B4B48454D1988EC78BC
:10BB5800B0F8E830A142A1EB030303F1020223D3BA
:10BB68002B788B4220D33D4B1C78032C51D03D4E73
:10BB7800424A1278022A04D13B4F414A3F78D78083
:10BB88009480012CA0F8E810B5D13A4A38491288B7
:10BB9800E87A0988121A914235DD3A4A12888A42AF
:10BBA800ACD200241C70A9E7B1EB440FDBDC2B4BB3
:10BBB8001C78032CDBD0042AD9D82A4EDFF8A8C079
:10BBC800DFF8C0E02B4F0022032434701C708CF87F
:10BBD8000020AEF800203A80CAE7012C36D0022CAB
:10BBE80010D10720BDE8F84019F080BD254A20494A
:10BBF8001288E87A0988121A91423FF77FAF012428
:10BC08001C707BE7F8BD02241C7077E702233370B1
:10BC180087E7042AABD82A7891FBF2F20132082A86
:10BC2800DFF844E06C78AE78164FA8BF08228EF88B
:10BC3800002092B216FB02F614FB02F20D4C3E8075
:10BC4800084E2280002434701C7091E70820BDE85B
:10BC5800F84019F04BBD00BF9B4400204C26002043
:10BC68007841002052260020F685002073410020EC
:10BC7800CC85002050260020741E0020FA360020B3
:10BC8800E44100204E2600202DE9F04FBC4B1E78E1
:10BC98008BB0002E40F0BC80BA4BBB4C1D78DFF84F
:10BCA80014A3DFF81493DFF8148305F00105A4F159
:10BCB8000A0B54F80A3CBBB1CC2707FB06B7184659
:10BCC800F6F7D2FE80B154F80A0CF6F7C5FE14F860
:10BCD800023C8BB9242831D0F5B154F80A3C1846F7
:10BCE800F6F7C2FE0028EED10136032E04F1CC048B
:10BCF800DFD10BB0BDE8F08F012B23D0022B2BD066
:10BD0800032B37D0042B67D0052B40D0062B4FD000
:10BD180054F80A2C1346D2E754F80A3C23281A464A
:10BD280000F08881994991F832108142C7D1984B27
:10BD3800CAF80090C3F80C801346C0E7012304F842
:10BD4800023CCAE74D2854F80A2C0CBF02230023F2
:10BD580004F8023C1346B2E700233C2804F8023CEE
:10BD680045D03E28D4D10122032304F8012C04F83D
:10BD7800023CB2E7C02814D80022042304F8050CBA
:10BD880004F8040C04F8062C04F8023CA5E714F89F
:10BD9800063C14F8052C9A422FD814F8043C834228
:10BDA80003D0002304F8023C97E7062304F8023C7A
:10BDB80014F801ECBEF1000F00F08C81BEF1010F08
:10BDC80000F0D08101360023032E04F8023C04F170
:10BDD800CC047FF46EAF8CE714F8043C04F8030C31
:10BDE8005840052304F8040C04F8023C75E70322C4
:10BDF80004F8013C04F8022C6FE714F8042CF91835
:10BE08004240013304F8042C04F8063C887264E7C5
:10BE1800604B186800283FF46CAFF7F7EFFA5E4BF9
:10BE28005E4D03F5947A5E4B1868F6F71DFE002800
:10BE38003FF45FAF5A4B1868F6F70EFE09281BD07F
:10BE48003F2819D02B68002B67D1042800F0AE8159
:10BE58000C2800F0E8807F28E5D0A0F12002D2B2BB
:10BE68005E2AE0D80BB92028DDD04E495A1CC854A8
:10BE78002A600FF037F9D6E72C68002C5BD12646EC
:10BE8800DFF8148100E0984608F10803002E08BF87
:10BE980046465345F7D3002E6DD03068D8F80020B9
:10BEA800075D135D9F42204402EB040140F07A8154
:10BEB8003C4F04F1FF3EBE4422460BB9FD2A7FD910
:10BEC8000EF8013F01322A6010F8013F11F801CF46
:10BED8009C45F2D00AB1B04512D033480FF00AF9A8
:10BEE800B04508D356F8080B0FF004F909200FF0F5
:10BEF800F9F84645F6D92D480FF0FCF82A680024D1
:10BF0800944290D22A4E264416F8010F0FF0EAF810
:10BF18002B6801349C42F7D385E70C2800F0838016
:10BF28000A2854D00D2852D07F2800F00881FF2B12
:10BF38003FF679AF91E7184FDFF868B04FF0000887
:10BF480007F59479464602E008374F450DD2224658
:10BF58003968584626F058FA0028F5D1B846002E18
:10BF6800F2D13E4608374F45F1D3002E95D1B8F1AE
:10BF7800000F3FF458AF0C480FF0BCF8B2E700BF11
:10BF8800E34100209B4400203E870020D86F00201A
:10BF980000ED00E0902E0020A82E0308942F00202A
:10BFA8008C2E0020942E0020F4540308FC5403081F
:10BFB800932E0020FC9F0020EFBEADDE0400FA05A2
:10BFC800511C2020B85429607B540A4683E77B4FD4
:10BFD8000FF0FDF83846232126F000FA002800F07B
:10BFE800E380C01B286078B1431EF95C202940F02B
:10BFF800E380FA1804E012F8011D202953D1034602
:10C00800581E002BF7D12B604FF4807200216B482B
:10C0180026F0AFF96A4B1B78002B3FF46AAE6948EB
:10C028000FF068F8FFE668480FF064F865480FF00D
:10C0380061F8F8E665496648C978664ADFF8C4E1F8
:10C04800C2F8EC30003118BF012101706249C2F812
:10C05800F0104021C2F8F43082F8F81082F8F95054
:10C068005E495F480B60F032CEF80020544A012345
:10C0780013700FF08DFD53480FF03CF8594A5A4998
:10C08800138891F8321043F080032329138005BFE9
:10C09800564A14F8023C14F8023CC2F80C8008BF57
:10C0A800CAF8009032E62B60514C444E002204F549
:10C0B8009479FA5402E008344C456FD2216830462E
:10C0C80009F016FD0028F6D04C4567D263689847FA
:10C0D800002398E7474BADF822E00FCB0DF1280C71
:10C0E80002AF87E80F004CF824ED14F8051C14F88B
:10C0F800033C069404EB010E624639464FF0010CEE
:10C1080006A8CDF81CE0ADF820308DF824C0F8F76B
:10C118002DFDE8B9019F002304F8023C002F3FF4ED
:10C12800E3AD54F80A0C18F04DFD013654F80A0C2A
:10C13800B847032E04F1CC047FF4BBADD9E5013B2D
:10C148001E4A2D482B600021D1540EF0D3FF6AE619
:10C15800029A2A4B03923946A4F10A00029307F087
:10C1680035FED7E714F8053C14F8032C069423444D
:10C1780007936E2A4FF0000308930993ADF8202027
:10C188007FF420AE631C06A80693F7F79FFD06A868
:10C19800F7F79CFD06A8F7F799FD13E618480EF087
:10C1A800A9FF95E7224695E628681CE7034808F0AA
:10C1B80099FF0BB0BDE8F08F034675E7942E002079
:10C1C800E3410020FC540308045503088E84002032
:10C1D800C0260020741E0020490500088C2E00206F
:10C1E80030550308A8410020D86F002000ED00E07A
:10C1F800A82E03088C2A03082C5503083093002026
:10C2080010550308902E00202DE9F04F2DED028BDC
:10C218008FB0064620F01EFC9C4B1F7827B10FB04C
:10C22800BDEC028BBDE8F08FDFF8C0B2DBF8003060
:10C238005905F4D5964B974D1B78002B40F05C813F
:10C24800954B1B78002B6BD0944C954AD4F86C31E5
:10C25800F31A934201F2478094F87481B8F1000F01
:10C2680031D1904F3868F6F7FFFBC0B201280ED9DC
:10C27800022841F0E6838C4B1A78002A41F0ED85BC
:10C28800D4F87821B21AB2F57A6F81F04C87D4F8D5
:10C298007C31002B44D094F87431BBB9834B1B68B4
:10C2A8009B7801211E3B00228B4284F8741184F88C
:10C2B800882141F2378638680221043020F0EBFAF1
:10C2C80094F880310FE0D4F87C314BB3D4F8843142
:10C2D80040F6B732F31A934222D994F88031002BF2
:10C2E80001F0E0826F4F013BDBB284F88031002B14
:10C2F80001F06B80D4F87C1194F8882111F801EBD7
:10C3080094F88931C4F87C1172440133386884F890
:10C318008821714684F88931F6F7AAFBC4F884614C
:10C32800634B2F681B7853B1DFF8C481D8F800003D
:10C3380028B1604B1B78013B012B41F255805E4BC5
:10C348001B7863B15D4F3B684BB1544CD5F80090F6
:10C35800D4F8C032A9EB0303632B00F22587584CAD
:10C368002378022B01F07F82DFF8888198F800306B
:10C37800032B01F01680534B1B7873B1524F3B6867
:10C388005BB1464CF6F720F9D4F8C832009044F671
:10C398001F62C31A934200F27F814C4B1B78002B1B
:10C3A8004BD14B4B1B7843B13C4CD4F8183403F5B4
:10C3B800C333A0339E4280F05787464B1B78002B2F
:10C3C8003FF42DAF354E444C444D06F239472068B2
:10C3D800F6F74AFB00283FF422AF2068F6F73CFB4B
:10C3E8002B7880465A1E33B120682A70F6F73CFB3A
:10C3F8000028F2D113E703223946781E25F09FFF63
:10C4080096F8383496F8392486F83B8483F47F43C9
:10C4180083F0FF039B1A1FFA88F89BB2B8EB132F1F
:10C42800D5D196F83A24DBB29A42D0D1781E20F0C2
:10C4380045F92B7818442870C9E7294C2278002A36
:10C4480040F0F286154CD4F8103403F5C333A0330A
:10C458009E42A6D3234A94F81434C4F81064D55CD9
:10C46800E90701F1EC83AA0701F1A8836B0701F141
:10C47800B4821D4A94F814341178013393FBF1F215
:10C4880001FB123384F814348BE700BFE34100202A
:10C49800648600203C4500206E860020B01F0020E6
:10C4A8003F0D030008860020250000200C86002090
:10C4B800708600207886002080860020186500207D
:10C4C8001A320020888600208C860020B48600203E
:10C4D800B586002092860020988600209C86002041
:10C4E8005C860020BC420020C14200207C4A00201B
:10C4F800E0850020350200205D4C2A68D4F85C31C4
:10C50800D31A7C2B7FF69CAE94F86031DFF88091CB
:10C518009FED588AC4F85C21013384F860314FF0EC
:10C528002408404620F05EFA534BF9EC016A1B8A56
:10C5380007EE103AF8EEE66AB8EEC77A08F1010895
:10C54800C6EE877A5FFA88F867EE887AFDEEE77AB2
:10C55800CDED007ABDF900A05FFA8AF020F01EFA4E
:10C56800CAF3072020F01AFAB8F1270FD9D13020E2
:10C5780020F038FAD4F86491DFF818815FFA89F06E
:10C5880020F00CFAC9F3072020F008FAD8F80000C8
:10C598005E21F6F76DFA94F860319A072DD1D4F838
:10C5A8005C2141F288339A4201F28E85142020F0F2
:10C5B80019FA324B324AB3F9043082FB03124FEABC
:10C5C800E379C9EBA2090FFA89F95FFA89F020F03B
:10C5D800E5F9C9F3072020F0E1F91C2020F002FA60
:10C5E800002020F0DBF9002020F0D8F95E21D8F8EF
:10C5F8000000F6F73DFA94F86031580701F09A8385
:10C60800282B7FF41DAE00271720D5F8009084F85A
:10C61800607120F0E7F9384620F0C0F9194B1A4C40
:10C62800A3FB09239B0BA4FB03125209C2EB0212C2
:10C63800A3EB8203D8B220F0B1F9182020F0D2F988
:10C64800124BA3FB09239B09A4FB03125209C2EB5B
:10C658000212A3EB8203D8B220F0A0F9384620F0EA
:10C668009DF9D8F800005E21F6F702FAE8E500BF68
:10C67800B01F002000007A44084200205C420020DD
:10C688006766666673B2E74589888888D34D621005
:10C698003C4200201086002094F8CE32002B41F056
:10C6A8007981E34B1A6802F00803002B48F603412E
:10C6B8004AF60B404BF60F4349F6074804BF0346BA
:10C6C800884612F0040F4FF0190118BF98469206D9
:10C6D80084F8CE1203D548F4804848F02008D54B9A
:10C6E8001A79C8F309010191002A41F05A855B794A
:10C6F800002B41F0D9869A4664204FF0FF330A4652
:10C708004FF00009CDF81880CDF81C800892ADF8DC
:10C7180026A0ADF828308DF83600ADF82490CDF875
:10C728002A90CDF82E90CDF832900DF1180CBCE877
:10C738000F00DFF810E384F85190AEE80F009CE892
:10C748000F00AEE807002EF8023B71464FF0010CCF
:10C758001B0C4FF0FE0E1F20C82201F81E3984F86A
:10C768004EE084F8522084F853C084F84F0094F8BF
:10C77800DE0284F8500080F0F10383EA0313DAB292
:10C78800130983F0E70343EA022383EAC2031BB2D7
:10C7980083EA0312D2B2C3F3072383EA121343EAEC
:10C7A800022383EAC2031BB283F0C80282EA0212A0
:10C7B800D2B2C3F3072383EA121343EA022383EABC
:10C7C800C2031BB283EA0C0E8EEA0E1E5FFA8EFEBF
:10C7D800C3F3072282EA1E1242EA0E22604482EA6A
:10C7E800CE0E84F8DE02A4F84CE001F11F0011F827
:10C7F800013B83EA0E0383EA0313DBB21A0982EAD8
:10C808001E2242EA032282EAC3031BB21FFA83FEF6
:10C818008142A4F84CE0EAD183F07C0383EA031355
:10C82800DBB21A0982EA1E2E8EEA032E8EEAC30EA6
:10C838000FFA8EFE1FFA8EF34FEA132A5FFA8EFE66
:10C84800A4F84C30DFF8009284F874A004F16E0369
:10C8580084F873E004F14E0C0193DCF80C30DCF83A
:10C868000000DCF80410DCF80820C846A8E80F002F
:10C87800019B0CF1100C9C45C146EED1DCF8000080
:10C88800C8F80000DFF8C4819CF8043089F8043047
:10C8980008F1270984F82DE384F82EA318F8011F5E
:10C8A8003868F6F7E5F8C145F8D194F8CF22002AA0
:10C8B80041F0758060492B6808780A2184F8CF1206
:10C8C800002801F07181DFF888C10128BCF8001048
:10C8D800059141F2C185BCF802100291022801F0CD
:10C8E8007C84BCF804100391032801F0F485BCF89B
:10C8F80006100191042801F0E8850528BCF8081005
:10C9080001F0DE850628BCF80AA001F0D5850728C5
:10C91800BCF80CE001F0B985BCF80E9094F8DE2262
:10C928000693104680F0300383EA0313DBB20490C9
:10C93800424A9DF810C0128884F850C0180980F047
:10C948007A0040EA032080EAC3033D48C2EB022292
:10C9580080FB02C01044D217C2EB602205988DF804
:10C968002D204FF0000860F30F0803984FF0000CDB
:10C9780060F30F0C00201BB261F30F0000216EF36F
:10C988000F0183EA031EC3F307230393029B63F398
:10C998001F48019BCDF81C8063F31F4C039BCDF807
:10C9A80020C05FFA8EFE6AF31F4069F31F4183EAD5
:10C9B8001E134FF0000A09900A918DF82CA043EA43
:10C9C8000E2C0DF11809B9E80F008CEACE0E0FFAFB
:10C9D8008EFE8EF0C808DFF86CC084F851A088EA93
:10C9E80008185FFA88F8CEF3072EACE80F008EEA35
:10C9F800181E4EEA082399E8030083EAC8080FFACC
:10CA080088F383F023024CF8040B82EA0210C0B2C8
:10CA1800C3F3072282EA1012049B2CF8141942EA85
:10CA28000022591C82EAC0004FF02308162211E0A8
:10CA3800B47C002078410020CC8400207041002084
:10CA48000308208004200020B8220020B7220020FC
:10CA58003C8B00204FF0FE0EC82384F8DE12A4F8A9
:10CA68004C000CEB020184F8538084F84EE084F803
:10CA78004F2084F852301CF8013B434083EA0313EB
:10CA8800DBB21A0982EA102242EA032282EAC303CD
:10CA98001BB298B28C45A4F84C00ECD183F0F40397
:10CAA80083EA0313DBB24FEA131E8EEA102E8EEAD6
:10CAB800032E8EEAC30EA0460FFA8EFE1FFA8EF9D9
:10CAC80058F84E0FDFF818C4A4F84C904FEA192A0A
:10CAD8005FFA8EFE84F86AE084F86BA0D8F8041038
:10CAE800D8F80820D8F80C30ACE80F00D8F81000B7
:10CAF800D8F81410D8F8182004F22539ACE8070043
:10CB080004F2073884F825A384F824E318F8011FF1
:10CB18003868F5F7ADFFC145F8D194F8D6E2BEF113
:10CB2800000F40F04687E64B94F8DEC2B3F90010D8
:10CB3800B3F90220B3F904309FEDE26A84F851E0BA
:10CB480007EE103A2B6806938CF06A0383EA031306
:10CB580006EE901AD9B20B0983F0D50343EA0123F4
:10CB680083EAC1031BB283EA03115242C9B207EE3A
:10CB7800902AC3F3072383EA111343EA0123F8EE4B
:10CB8800E77AF8EEE66AB8EEC77A83EAC1031BB221
:10CB980067EE867A66EE866A27EE067A002083F0CC
:10CBA800C805CDED087ACDED076A8DED097A0A90B2
:10CBB8000B900C9085EA05150DF11809EDB2C3F339
:10CBC8000728B9E80F0088EA151848EA052888EA0E
:10CBD800C505DFF810832DB2A8E80F0085F01E0EFA
:10CBE80099E807008EEA0E13DBB2C5F3072E8EEA2A
:10CBF800131E4EEA032E88E807008EEAC30EA8F13A
:10CC080010051C20C8214FF005091E234FF0FE080F
:10CC18000CF1010284F8521084F8D69284F853304B
:10CC280084F84E8084F84F00291884F850C0A4F87E
:10CC38004CE084F8DE2215F8013B83EA0E0383EA10
:10CC48000313DBB21A0982EA1E2242EA032282EAAD
:10CC5800C3031BB21FFA83FE8D42A4F84CE0EAD14D
:10CC680083F0270383EA0313DBB21A0982EA1E2E34
:10CC78008EEA032E8EEAC30E0FFA8EFE1FFA8EF38B
:10CC88004FEA13295FFA8EFEDFF85482A4F84C307D
:10CC980084F8719084F870E004F14E0C04F16E0A87
:10CCA800DCF80000DCF80410DCF80820DCF80C30B4
:10CCB80045460FC50CF1100CD445A846F0D1824D5D
:10CCC800BCF80030A8F8003005F1240884F82AE3FD
:10CCD80084F82B9315F8011F3868F5F7C9FE454508
:10CCE800F8D194F8D7320293002B40F05D86774B49
:10CCF8001B68052213F0140F84F8D72240F0B2867F
:10CD0800DFED737A94F8DE826D4B724AB3F9041042
:10CD1800B2F90620704D7148CDED087A88F02203EB
:10CD280083EA03135FFA83FE4FEA1E1383F0590365
:10CD3800B2F5FA6F43EA0E2383EACE03A8BF4FF495
:10CD4800FA621BB2B2F57A7F83EA031EB8BF4FF4CA
:10CD58007A725FFA8EFE4FF0640CA2F57A72C3F312
:10CD680007230CFB02F283EA1E1385FB025980FBA2
:10CD78000150D21743EA0E25C9174FF0000AC2EB3B
:10CD8800A912C1EBA00185EACE050DF1180CADF88A
:10CD98002A20ADF82810CDF818A0CDF81CA0CDF8A1
:10CDA80024A02DB285F0C80ECDF804C0BCE80F0051
:10CDB8008EEA0E1E5FFA8EFEC5F3072585EA1E155C
:10CDC800DFF82091DCF800C084F8508045EA0E2591
:10CDD800A9E80F0085EACE0212B282F04A0383EA7C
:10CDE8000313DBB2C2F3072282EA131249F810C90F
:10CDF80042EA03224A2082EAC3034FF0140E0025B8
:10CE080008F101084FF0FE0C84F85300C82084F89C
:10CE1800515084F8DE82A4F84C304A4609EB0E01E2
:10CE280084F84EC084F84FE084F852001D4612F88A
:10CE3800010B684080EA0010C0B2030983EA152399
:10CE480043EA002383EAC00000B285B28A42A4F80C
:10CE58004C50ECD180F0140080EA0010C0B24FEAC8
:10CE6800101E8EEA152E8EEA002E8EEAC00E25467A
:10CE78000FFA8EFE1FFA8EF855F84E0FDFF860C0D5
:10CE8800A4F84C804FEA182A5FFA8EFE84F869A04D
:10CE980084F868E06968EB68AA68ACE80F0028695C
:10CEA80069692B8BACE8030004F20735ACF8003055
:10CEB800A84684F823A384F822E304F2233A13E073
:10CEC8005C42002088C3E43AB7220020B47C0020EA
:10CED800000000003C8B0020D34D62106766666638
:10CEE800B82200200420002018F8011F3868F5F740
:10CEF800BFFDC245F8D1D14BD14A1B781278013B0E
:10CF080012F00100DBB214BFC0224022172B04D854
:10CF1800CC490B4493F824300293CB4B19888B07E8
:10CF28001ABF002342F01002012311F4027F18BF38
:10CF3800022311F0100F18BF062311F0200F18BF9D
:10CF48001023002841F07C80032194F8DEE2069348
:10CF58008EF0460383EA0313D8B2030983F09203E1
:10CF680043EA002383EAC0031BB283EA0310C0B27A
:10CF7800C3F3072888EA101848EA002888EAC00896
:10CF88000FFA88F888F0C80C9DF808008DF81C0086
:10CF98008CEA0C1C00235FFA8CFC8DF81E20032001
:10CFA800019A8DF81D30C8F307288DF81F108DF8E9
:10CFB800200088EA1C1807CA48EA0C2888EACC0C22
:10CFC8000FFA8CFC8CEA0C18A9E803005FFA88F8C1
:10CFD800CCF3072181EA181141EA082181EAC8083F
:10CFE80094F854C089F800200FFA88F28CEA020CF1
:10CFF8008CEA0C1C5FFA8CFCC2F3072282EA1C1232
:10D0080042EA0C2294F8550094F8561094F8579078
:10D0180094F8588084F8533082EACC0212B2504017
:10D0280080EA0010C0B2C2F3072282EA101242EA74
:10D03800002282EAC00212B2514081EA0111C9B24B
:10D04800C2F3072282EA111242EA012282EAC102ED
:10D0580012B289EA020989EA09195FFA89F9C2F361
:10D06800072282EA191242EA092282EAC90212B2A6
:10D0780088EA020888EA08185FFA88F8C2F30722E3
:10D0880082EA181242EA082294F859C094F85A0021
:10D0980094F85B1094F85C9084F8513082EAC802E6
:10D0A80012B28CEA020C8CEA0C1C5FFA8CFCC2F3FC
:10D0B800072282EA1C1242EA0C2282EACC0212B24D
:10D0C800504080EA0010C0B2C2F3072282EA101270
:10D0D80042EA002282EAC00212B2514081EA0111FA
:10D0E800C9B2C2F3072282EA111242EA012282EA95
:10D0F800C10213B289EA030282EA0212D2B2C3F36E
:10D10800072383EA121343EA022383EAC2031BB20A
:10D1180083F0320282EA0212D2B2C3F3072383EA0F
:10D12800121343EA022383EAC2031BB29AB24FF0F6
:10D13800FE0CDFF8288184F850E00920C8210EF1A0
:10D14800010EDBB284F84EC04FEA122C84F84F006F
:10D1580084F8521084F8DEE2A4F84C2084F85EC00B
:10D1680084F85D30D8F80000D8F80410D8F8082002
:10D17800B8F80CA008F2BA2EAEE8070008F2CA28E0
:10D188008EF80290AEF800A084F818C384F817331C
:10D1980015F8011F3868F5F76BFCA845F8D1009B16
:10D1A800C4F8C832FFF7F9B8DFF8B4A0DFF8B480E4
:10D1B80041201FF023FBBAF9023088FB0320DB175C
:10D1C800C3EBA00080B21FF0FFFABAF9003088FB69
:10D1D8000320DB17C3EBA00080B21FF0F5FABAF901
:10D1E800043088FB0320DB17C3EBA00080B21FF0DC
:10D1F800EBFA164B38681978F5F73AFC94F8C4320C
:10D2080013F0010800F03C84114AC4F8C0920133BD
:10D21800DBB2A2FB0312D20802EB8202A3EB4203A9
:10D2280084F8C432FFF79BB80A4B0B491868F5F726
:10D23800EFFB00232370FFF705B900BFF836002085
:10D248009B4400209C2A0308D84100208A650020BE
:10D25800CDCCCCCCB842002038860020FE1F002060
:10D268005C4200206766666694F81C34C74AC4F8B6
:10D27800186402EB8302D26B42B30EAD04F223436F
:10D28800C34E45F8203D002104F235433180079311
:10D2980080211523A52784F82234284684F82114F0
:10D2A80084F82074904728463188F6F74BFD069D90
:10D2B800B84804F584616D1A152DA8BF15252A46AE
:10D2C80022F0D6FDB44A94F81C341570B34A0133E1
:10D2D80082FB0312A2EBE37202EB42029B1A84F870
:10D2E8001C34FFF76AB8AE4BAE4AD4F87011286800
:10D2F800128893F80BE0AC4B401A4FF47A71D7B20E
:10D3080001FB0EF1120A9F771F7588424FF0000744
:10D31800DA775A759F701F7180F05183A34AA44928
:10D32800DFF89CC212680F688868DFF898E2C4F8D2
:10D338006C618CFB0281D217C2EB6112D4F86411C4
:10D348008CFB018C8EFB07988EFB009EC017C0EBF0
:10D35800AE0002F5FA724FEAE17E92B2CEEB6C1C97
:10D36800FF1701F5EA4EC7EBA8070EF1300E9A76C3
:10D37800120A0CF1780C4FEA2E2E3031DA764FEA89
:10D38800272802121F7783F81D8083F8200083F86E
:10D39800212083F824C083F823E083F82210FEF7C5
:10D3A8005BBF844F386803685B69984700283EF480
:10D3B800E2AF3868036801219B699847022200237D
:10D3C80088F800202370FEF7D6BF94F8881194F8E7
:10D3D800893138684A1C013384F8882184F88931F6
:10D3E800F5F746FBFEF79ABF734CDFF8DC914FF078
:10D3F800000A0BE01B2B00F049820D2B00F0128273
:10D408004FF0010389F80130D8F80000F5F72CFB3C
:10D41800002837D0D8F80000F5F71EFB83B27E2B22
:10D428002A6828D099F80120002AEDD194F88A11A9
:10D438000029DFD07D2B00F0098294F88EE1BEF13F
:10D44800000F04D080F02003DBB284F88E214A1C40
:10D45800D2B2092A635484F88A2100F0EB81082AA1
:10D46800D2D8B4F88C21134403EB132303F0FF0341
:10D47800A4F88C31C8E784F88AA184F88BA189F8CC
:10D4880001A0C1E794F88F312BB1637884F88F013C
:10D49800302B00F0658594F88B213C4BDFF82C91FC
:10D4A800DFF82CC1DFF82CA14FF0010E002A3EF462
:10D4B80046AF2968C91B012900F2AF8194F8A482FC
:10D4C800B8F1000F40F0F98194F8BC1233F811005C
:10D4D80010B984F8BCE2E9E70131B0F5826F84F84D
:10D4E800BC1200F0E0801ED9B0F5E26F00F0C180F8
:10D4F80034D9B0F5046F00F0CA80B0F5116F00F0B0
:10D508002581B0F5E46FD1D12C4AD76B118A6423F9
:10D5180003FB07F393FBF1F11FF0A3F9002384F851
:10D528008B31FEF70CBFB0F5007F00F0298153D88E
:10D53800B0F5807F00F04781B0F5887FB6D1D9F883
:10D5480000104907B2D5D4F864114FF488701FF061
:10D5580088F9002384F88B31FEF7F1BEB0F5C06F6F
:10D5680000F02181B0F5E06FA0D1144A506B118A08
:10D57800642303FB00F34FF4E06093FBF1F11FF029
:10D5880070F9002384F88B31FEF7D9BE9C2A030872
:10D59800C88500209C2F0020B12F002056555555D6
:10D5A800E8850020CC85002064420020E01D002092
:10D5B800D0850020B8320020B01F0020084200208B
:10D5C8001F85EB516766666625000020B47C002045
:10D5D80078410020F6850020B0F5047F00F0038133
:10D5E800B0F5806F7FF462AF94F8BD320133DBB2DF
:10D5F800032B00F2328142F2107184F8BD3201FB34
:10D6080003F1BE4B1B88002B40F025810131BC4B38
:10D618001B78D807BB4B1B8848BF0431DA0748BFC3
:10D628000A31980748BF14311A0648BF2831D8056F
:10D6380048BF28315A0748BF6431180748BFC83166
:10D648009A0548BF01F5C871980648BF01F57A7177
:10D65800DA0648BF01F5FA61580648BF01F57A6154
:10D668004FF480601FF0FDF8002384F88B31FEF73B
:10D6780066BEA54A976B118A642303FB07F393FBE5
:10D68800F1F11FF0EEF884F88B81FEF758BE9F4B3E
:10D69800B3F9041001EB810149001FF0E2F884F8A6
:10D6A8008B81FEF74CBED9F8001011F020087FF4EA
:10D6B800FDAEDBF80010090600F13C849449097BB3
:10D6C80000293FF4F3AE94F8BE12032900F2448611
:10D6D800DFE801F0322819028E4B1B6859799A79D4
:10D6E800DB7901F1407101EB022101EB03410023D9
:10D6F80084F8BE324FF482601FF0B3F8002384F838
:10D708008B31FEF71CBE844B1A68137A50799278D5
:10D718001B0403EB002313444A1C84F8BE2203EBCA
:10D728000161E7E77C4B1A68D379107952781B04BA
:10D7380003EB00231344EFE7774B1A689379D0780B
:10D7480012781B0403EB00231344E5E79CF804104C
:10D7580000293FF4ABAE9AF8001000293FF4A6AEBA
:10D768006E4B1B8803EB83035B004FF4116093FB44
:10D77800F1F11FF076F8002384F88B31FEF7DFBD56
:10D788009CF8051000293FF491AE654B65491B686C
:10D7980081FB0321DB17C3EBA1011FF062F884F8BA
:10D7A8008B81FEF7CCBD9CF8051000293FF47EAEB6
:10D7B8005B4B4FF4C06099681FF053F8002384F85E
:10D7C8008B31FEF7BCBDD9F8001048077FF56EAE67
:10D7D800554B4FF4807019681FF043F8002384F804
:10D7E8008B31FEF7ACBD9CF8041000293FF45EAE07
:10D7F8009AF8000000283FF459AE454B5B7B002B9C
:10D8080000F01A84454B198891FBF0F101EB810176
:10D8180049004FF404701FF024F8002384F88B317A
:10D82800FEF78DBD4FF0010284F88A212370A4F819
:10D838008C11E9E5B4F88C21C2F1FF0293427FF420
:10D84800DFAD4FF0010384F88F31D9E54FF00103C4
:10D8580084F88E31D8E50231D9E6012384F8BD3247
:10D8680042F21071CDE6F4F7AFFE304B1A6840F67D
:10D87800B833801A984200F2EB802D4F3B793A2B4F
:10D8880000F0F18200232370FEF775BDD8F8000080
:10D89800F5F7EAF800287FF4B3AD4FF0010384F8F8
:10D8A8008B31B1E5C4F87C3184F87431214F1FF015
:10D8B80021F894F88031FEF716BDD4F89432DFF8D9
:10D8C800789094F8BA224B4500F04A84511C94F899
:10D8D800BBE2D4F898C284F8BA1202F00F028DF8AD
:10D8E80018200DF11902ACEB0301002940F345851E
:10D8F80006A901910DF11E0723E000BFA8410020F1
:10D908009B440020D8410020084200205C420020AF
:10D91800E885002048380020A4840020CC85002019
:10D92800D085002067666666E01D00202032002052
:10D93800083200200886002044210020002840F3F7
:10D948009C800133C4F8943213F8011C02F8011BBF
:10D95800BA42ACEB030081EA0E0EEFD384F8BBE2C7
:10D9680000F00585501CB84282F800E005D20EABE5
:10D978009A1A1B3A002124F0FCFC019932201EF06F
:10D9880055FF4FF00008002384F8A48284F88B31F7
:10D99800FEF7D5BC013B84F8CE32FEF786BF013ACC
:10D9A80084F8CF22FFF7B9B8013B84F8D732FFF7E4
:10D9B800F6BB0EF1FF3E84F8D6E2FFF792B9C64AED
:10D9C80029681278C4F87011013A012A3FF6A6AC0A
:10D9D8001021022299701A71A0E4C04AC04B126843
:10D9E8000793A3F1240800202121D50003F8240C73
:10D9F80088F8021040F11483BA490327BA4B1B88F0
:10DA0800580500F10A83DA0700F1E48303F0020302
:10DA1800B64A002B1CBF03271146B54D3A46284687
:10DA280022F026FA7B190EA80133A91E40F8203DE2
:10DA380000225B1A7A5588F801301EF0E3FFFEF7E2
:10DA480018BD1EF049FFAB4B01221A70FEF71FBC30
:10DA5800A94AB2F8C63200210133A2F8C6322170B1
:10DA6800FEF789BCA54B9FEDA67AD3ED007AF8EEB8
:10DA7800E77A67EE877AFFF745B984F8BBE271E782
:10DA8800994B1B88DA0515D4D80600F1AE839906A0
:10DA980000F15E845A0600F19E84180700F1BD84E7
:10DAA800D90700F19C8413F0020F0CBF4FF0040853
:10DAB8004FF00C08934B944A1B78D27803F001037B
:10DAC8000AB143F00203532000931EF097FE8F4AD9
:10DAD800128802EB820202EB8202900080B21EF0F2
:10DAE80073FE00201EF070FE894A8A491288386841
:10DAF800C2EBC212520081FB023111444FEAE27AB2
:10DB0800CAEB612A5FFA8AFA5146F4F7B1FF824BF1
:10DB180038681A78009B48EA03087F4B8AEA020AA9
:10DB2800002183F800A0F4F7A3FF41463868F4F712
:10DB38009FFF794B784A1B78386888EA0303DBB281
:10DB480019461370F4F794FF94F8C432002B7FF44D
:10DB58005BAB4F201EF052FE16F0DEFF16F0DCFF26
:10DB680016F0DAFF01213868F4F782FF6B4A6A4B36
:10DB780092F800801B78684A386808F00108414626
:10DB880083F001031370F4F773FF634B38681B7855
:10DB980088EA0308604B414683F80080F4F768FF81
:10DBA80094F8C432FFF730BB86468246014601909E
:10DBB8000390029005908146FEF7B0BE484B53494A
:10DBC80007930EAFA3F1210047F8200D4FF0080E80
:10DBD8004FF000080A2003F822EC03F8230C03F89E
:10DBE800248C38460988F6F787F84D4B4D491B6851
:10DBF80081FB0321DB17C3EBA101384689B2F6F795
:10DC08007BF8494BB3F8069005F0A4FE069B5A1C16
:10DC1800069283F80080069B4FEA1922591C069148
:10DC28001A70069B5A1C069283F80090069B5A1C91
:10DC38000692187038461EF0E5FEFEF717BCDFF8AE
:10DC4800F0809FED3A8AB8F90230254A079207EE2C
:10DC5800903AF8EEE77A0EAF67EE887AA2F12403DD
:10DC6800FDEEE77AA2F12101002047F8201D02F815
:10DC7800240C0822CDED007A5A701E229A70BDF845
:10DC880000103846F6F738F8B8F9003007EE903A41
:10DC9800F8EEE77A384667EE887AFDEEE77ACDED5A
:10DCA800007ABDF80010F6F727F8B8F9043007EE47
:10DCB800903AF8EEE77A384667EE887AFDEEE77A2A
:10DCC800CDED007ABDF80010F6F716F838461EF0CC
:10DCD80099FEFEF7C8BB00BF734100203035002015
:10DCE8003886002040550308D841002050550308C5
:10DCF8001786002025000020B01F0020E01D00200E
:10DD08000AD7233C9B44002084410020CC85002076
:10DD180070410020030820808A65002038350020E3
:10DD2800D0850020676666667841002058A08B4140
:10DD38005C42002002201EF055FECD4BCD4ADB6927
:10DD4800323382FB0329DB17C3EB69195FFA89F0C9
:10DD58001EF024FEC9F307201EF020FE03201EF04B
:10DD680041FEC54B1B78D90740F172810EF09AFB32
:10DD7800C24B9FEDC37AD3ED037A67EE877AFCEE48
:10DD8800E77ACDED007ABDF80030002800F0D9829E
:10DD9800DFB24FEA132938461EF000FE48461EF04F
:10DDA800FDFDDFF8109399F80430002B40F0208235
:10DDB8000DF118094946B3481EF0B4FD13201EF0B2
:10DDC80011FEBDF91870F8B21EF0E8FDC7F3072080
:10DDD8001EF0E4FD1B201EF005FEBDF91A70F8B216
:10DDE8001EF0DCFDC7F307201EF0D8FD23201EF02F
:10DDF800F9FD4E201EF0D2FD00201EF0CFFD494651
:10DE0800A0481EF08FFD12201EF0ECFDBDF9187021
:10DE1800F8B21EF0C3FDC7F307201EF0BFFD1A209D
:10DE28001EF0E0FDBDF91A70F8B21EF0B7FDC7F399
:10DE380007201EF0B3FD22201EF0D4FD45201EF061
:10DE4800ADFD00201EF0AAFD5E21D8F80000F4F711
:10DE58000FFE94F86031FEF7D3BBC4F8786183F8FD
:10DE68000080FEF714BABB78DBB103F1FF3C5FFA20
:10DE78008CFC0CF1010CBC44BE4600221EF8013B90
:10DE8800534083EA0313DBB2120AD90042EA0322A1
:10DE9800F44581EA131382EA0302EFD1002A7FF4E2
:10DEA800F1AC794BDFF810C2D3F800E0774B784932
:10DEB8001B68DEF83080774ACCF83830764B098812
:10DEC800CCF81810CCF868001168B3F8C60292684C
:10DED800CCF82810CCF84820CCF85800B8F1000F3E
:10DEE80000F08F82D8F80430DEF840108B423BBF38
:10DEF800DEF80C205B1A5B1A9B18002B7EF434AA00
:10DF0800DEF80030DFF8B4819B697046022198473B
:10DF18000423F87888F8003009F062FD03232370A1
:10DF2800FEF724BA02213868F4F792FD94F880319C
:10DF3800FEF7D9B910230422184606A98DF81A80CD
:10DF48008DF81B808DF81C808DF81D808DF8183099
:10DF58008DF819201EF06AFC84F88B81FEF7EFB962
:10DF6800A3785A09012A40F0CA8103F00F0C13F074
:10DF7800100300F0D681DFF84881E37894F804E0D4
:10DF8800A4F8B20208EB03018EEA030084F890219A
:10DF98004346C4F8A882C4F8AC12A8F1070284F872
:10DFA800B802A4F8B0E294F8B802DFF818818646FF
:10DFB8000CE012F8011BC4F8A802424581EA0E0ED3
:10DFC800197007D2D4F8AC12D4F8A832994203F1E8
:10DFD8000100EED1424584F8B8E200F0618212787F
:10DFE80094F8B8329A4200F0CE812C4BC4F894329F
:10DFF80000220133B4F8B012C4F8983284F89021A2
:10E0080001234FF6F672A4F89C1284F8943184F830
:10E01800A432A4F89E22FFF73EBA03272049FCE465
:10E02800DBF800301F4A204903F48003834216BFFF
:10E03800114604270327E1E4154B1988FFF7E6BBCF
:10E048001A49C97800290CBF04210521FEF77DBFB4
:10E05800DFF86090164BB9F80670A3FB0737BF08C6
:10E06800F8B21EF09BFC380A1EF098FC9BE600BF35
:10E07800243400201F85EB519B440020F8850020A4
:10E08800CDCC4C3E80969800B8320020E01D002090
:10E09800CC850020D0850020B01F0020442100201E
:10E0A80044550308405503083855030884410020A7
:10E0B800CDCCCCCC78410020C40100203502002012
:10E0C800BC1F0020B81F0020DFF884A310201EF01A
:10E0D80089FCD54ADAF8003082FB0329DB17C3EB49
:10E0E80069195FFA89F01EF059FCC9F307201EF080
:10E0F80055FC21201EF076FCDAF80020CA4B83FB81
:10E10800023AD3176421C3EB6A1301FB1323002BD4
:10E11800D8BF5B421BB2D8B21EF040FC00201EF0F4
:10E128003DFCFEF743BA012238681A70F4F794FCF4
:10E1380080463868F4F790FC18F07F0F7EF4A7A8A3
:10E148008E287EF4A4A894F87431002B7EF4BBA822
:10E15800B64BC4F87C312D2384F88031FEF79EB885
:10E16800B4F99E12D4F898C294F89CE2501C02F0BC
:10E178000F0242F010020029B8BF42F020028DF8C9
:10E188001820ACEB090282EA0E0E5FFA8EFE8DF8BB
:10E19800192084F8BA0284F8BBE20DF11A02FFF7DD
:10E1A800A2BBA3495A790B8803EB830303EB8303D0
:10E1B8004FEA830A1FFA8AFA002A00F032819D4B3F
:10E1C8001B681BB2029305F0C5FB029B019A40B283
:10E1D800FEF796BA984904271FE4964692461146D8
:10E1E800019203929146FEF799BB4FF0340861E41F
:10E1F800DFF860A29AF80020002A3FF4D9ADB4F8FD
:10E2080068718B4B00921B883F016421BFB201FBF0
:10E2180003235100B3FBF1F347EA0327BFB2C3F36B
:10E2280003231F4306201EF0DDFBF8B21EF0B6FBE9
:10E23800380A1EF0B3FBB4F868317D4A7F49178865
:10E24800009A01339BB293FBF2F002FB1033487A39
:10E25800A4F86831012800F00E814B7B6E2202FB86
:10E2680007F7152297FBF2F7002B40F0FE803A20C3
:10E278001EF0B8FBBFB24FF0640AB7FBFAF293B2D4
:10E28800D8B2019200931EF089FB009B180A1EF079
:10E2980085FB3B201EF0A6FB019A0AFB127080B298
:10E2A8000A23053090FBF3F0C0B21EF077FB002084
:10E2B8001EF074FBDFF87CA128201EF093FB0A23D4
:10E2C800DAF8007097FBF3F7F8B21EF067FBC7F3B4
:10E2D80007201EF063FB04201EF084FBB9F806300B
:10E2E800002B40F08680DAF8087087F31007F8B240
:10E2F8001EF054FBC7F307201EF050FB58E5504BA7
:10E30800504AC4F89432591C012384F8900184F8C7
:10E318009401C4F89812C4F89C2284F8A432FFF738
:10E32800BAB894F89021002A3FF4B5A894F8B92215
:10E33800013202F00F02624555D084F89031FFF7A0
:10E34800AAB8DBF80020D2067FF522AD814622E587
:10E358004FF02408FFF7AEBB4B1CDBB2042B84F84C
:10E36800BE324FEA01617FF4C5A9FFF7C0B9019930
:10E3780032201EF05BFAFFF706BB06AB01930DF1E6
:10E388001E07FFF7EFBA304BD4F8A822C4F8AC2226
:10E398004FF0000E03F52272114603F5C479C4F854
:10E3A800982203F527707246C4F8A832C4F89CE294
:10E3B800C4F8949284F890E1F6F7D8FB013067D05E
:10E3C800D4F89432C4F898320123C4F8949284F8AB
:10E3D800A432FFF760B84FF01008FFF76BBB4FF09F
:10E3E8000808FFF767BBD4F8AC12D4F8A832174A6C
:10E3F800D9E505F0AFFA1EF0D1FA00201EF0CEFAEA
:10E40800D6E4DEF81C10DEF8203099423BBFDEF877
:10E418000C205218CB1AD31A6FE54FF02008FFF7DB
:10E4280049BB4FF0FF33CCE61F85EB516442002017
:10E43800CC850020D085002048550308E8850020B9
:10E44800442100200000F6FFBC1F0020B31F00205D
:10E45800E01D0020F685002096469246114601925E
:10E46800039202929146FEF759BABFB29AF8003069
:10E4780097FBF3F7FBE639201EF0B4FAF8B21EF06A
:10E488008DFA380A1EF08AFA14E79146FEF746BA62
:10E49800D4F894320222591CC4F894121A708FE7E7
:10E4A80084F8B9C2FEF7F7BF0E4B9246B3F90030B5
:10E4B80064200A46FEF724B996469146FEF72EBA1E
:10E4C800964692469146FEF729BA964692461146D6
:10E4D8009146FEF723BA9646924611460192914616
:10E4E800FEF71CBAD08500202DE9F04FDFF808B1FF
:10E4F8002DED0C8B9BF8003099B0012B039001F0A7
:10E508002C82DFF8F8A09AF80021002A41F0348222
:10E51800072B01F03B824FF00009344C636820461A
:10E52800984700286ED0B4F8A860002284F84920E3
:10E53800002E40F09182B4F92450E16AB4F9260023
:10E54800226BB4F92830691AA16329490091821A0B
:10E55800606BE2630D461B1A94F84A10236404F1B9
:10E5680038000BF0A3F92B6813F0005302F0C681B2
:10E57800D4ED0F5AD4ED0E7A1E4A9AED416ADAEDBF
:10E58800426A9AED437ADAF810311268B8EEE58AF1
:10E59800D4ED105AF8EEE77AF8EEE58A013377EE13
:10E5A800867A38EE268A78EE878A9342CAED417ACF
:10E5B8008AED428ACAED438ACAF8103101F0A4866E
:10E5C8009BF80060142E02F0AA870023DAF818518D
:10E5D8000193062D02F25482DFE815F0DB14C7140C
:10E5E800F21122171A16B1169E1500BF20700020CE
:10E5F8007C4A0020B87C0020FA360020EC2300205A
:10E60800DDF804909BF80080B8F1070F00F0DB827A
:10E618009AF828310593002B40F0E182CD4B5B79C5
:10E62800002B40F0148201239BF800208AF828313F
:10E63800072A02F07F8200230793C74BDAED4C9A32
:10E6480093ED007AC54AC64B1268C64FDAED4B8A7D
:10E65800DFF89493DFEDC4AA9FEDC49A9FEDC4BA86
:10E66800DFEDC4CA9FEDC4AADFEDC4BADFF87C832E
:10E67800C34E0493F7EE007A37EEE98A002428EEB9
:10E68800078A0292B4EEE78AF1EE10FA88BFB0EE7C
:10E69800678A019325460097BA4B2344D3ED007A45
:10E6A800B94BF5EE407A2344F1EE10FA93ED00CA27
:10E6B80017D0B64B234493ED007A7CEE476AB0EE50
:10E6C800E66AF4EEC67AF1EE10FA08D5F5EEC06AFD
:10E6D800F1EE10FACCBF37EE87CA37EE67CA83ED82
:10E6E80000CAAB4B1F88BB0700F08182022D04F0E3
:10E6F80028850299A74B91F8322007EE102A91F845
:10E7080031202344D3ED006A5342B8EEC77A07EEAE
:10E71800903A27EE267AF8EEE77AB4EEE77AF1EE49
:10E7280010FA0AD407EE902AF8EE677AF4EEC77A60
:10E73800F1EE10FA88BFF0EE477A974B0693974AA6
:10E7480003EB450332F91510B3F90A30C81A07EE7E
:10E75800100AB8EEC77AF807E7EE497A40F19882CE
:10E768008F4F97ED00CA27EE8CCA9AF86471E7B10B
:10E778008B4FDAF8680197ED007A8A4F5B1A07EE3B
:10E78800903A039B396827EE097AF8EEE77A1F1A60
:10E798008F4227EE87CA01F3AF81F7EE007AF4EED5
:10E7A800E79AF1EE10FA01F173817F4B2344D3ED20
:10E7B800007A019BD3ED01DA009B68EEA77A3CEE64
:10E7C8006DDA67EE8D7AC3ED007A784BD9ED006A81
:10E7D80093ED007A764BD6ED007A26EE877A2344BD
:10E7E80067EE086A93ED007A26EE877AF0EE676A9C
:10E7F800E7EE0D6AB0EE667A9AED4C6AF7EE006ABB
:10E80800B4EEE66AF1EE10FAACBF0123002343B17F
:10E81800F0EEE77AF0EEC76AF4EEE76AF1EE10FA86
:10E8280001D586ED007A022D04F08484614A624B9A
:10E8380052F825001B68B0EE6D0A98475F4A604B96
:10E8480052F825001B689847029B93F83A30632BCF
:10E8580004D84F4B1B88002B01F06081F0EE6C7AD6
:10E86800584B99ED007A37EEC00A2344D3ED007A6D
:10E8780083ED000A029B30EE670A93F8482080EE89
:10E8880007CADAB1F7EE007AF4EEE79AF1EE10FA79
:10E8980014DB4D4BD3ED007AB0EECC7AB4EEE77AC8
:10E8A800F1EE10FA0ADD494BD3ED007AB0EECDDA7D
:10E8B800B4EEE7DAF1EE10FA01F38E81444B9AF8E0
:10E8C80074212344D3ED007A68EEA77A27EE8CCA28
:10E8D80088ED00CA32B9009BC6ED00CAC3ED00CA74
:10E8E800C8ED00CA009B04330093019B0434043331
:10E8F8000C2C05F1010508F1040806F10406019342
:10E908007FF4CAAE9BF80030072B02F0CD80012BB4
:10E9180002F00081002304932E4B00931A460F4BFC
:10E9280012681B680192114693F82F2011F4805346
:10E93800069300F05182284B02931B7827480790D2
:10E9480013F0010F264B0393198B264B90ED037A96
:10E958004EE000BF0C700020607B0020A4840020E3
:10E9680044780020FC33002000009642CDCCCC3DFA
:10E97800AE47813F000000000000C8420000344359
:10E9880008340020547B0020202500202C2500205E
:10E99800D841002038250020843400205C42002023
:10E9A8003C7B0020647B0020107B00202800002096
:10E9B8001C7B00200C3A0020083A0020703A002006
:10E9C8006C3A002058250020747B0020707B0020C2
:10E9D800287B00207C4A00209B440020F8850020EA
:10E9E8004C4A0020E83F00200C7B00201434002013
:10E9F800DB8808BFAAF87C11C81A07EE900AF8EE5F
:10EA0800E77AB4EEE77AF1EE10FA42F26780CC18B2
:10EA180006EE904AF8EEE66AB4EEE67AF1EE10FAFF
:10EA280081F23B84BAF87C31984283F24681D54B17
:10EA3800D54993ED004AD1ED004AD44BCAED604A5E
:10EA48008AED614AD3ED006ADFEDD17AE0E1D14B7E
:10EA58001B78013BDBB2E7E5CF49D04B49780493FB
:10EA680000911B68CE4F9BF80080B7F906004FF461
:10EA78007A71B1FBF3F3C3EB431503EB8503DD00B8
:10EA8800ADB2AE4202F02F86E16FB4F924E0236EF6
:10EA98004A1C07EE90EA7344012AE2672366F8EEFF
:10EAA800E77A02F02A86D4ED1B5AD4ED1D6A07EEE8
:10EAB800102A37EEE56AB8EEC75A012E86EE057AB7
:10EAC80037EE257A77EEC77A84ED1C7AE6EE276A68
:10EAD80084ED1B7AF0EE667AC4ED1E6AC4ED1D6AF9
:10EAE80003F04A81D4F89010B4F926E0636E4A1C0A
:10EAF80007EE90EA7344012AC4F890206366F8EEA2
:10EB0800E77A02F01286D4ED205AD4ED226A07EE95
:10EB1800102A37EEE56AB8EEC75A012E86EE057A56
:10EB280037EE257A77EEC77A84ED217AE6EE276A02
:10EB380084ED207AF0EE667AC4ED236AC4ED226A89
:10EB480003F03C81D4F8A410B4F928E0A36E4A1C61
:10EB580007EE90EA7344012AC4F8A420A366F8EEED
:10EB6800E77A02F0FB85D4ED255AD4ED276A07EE43
:10EB7800102A37EEE56AB8EEC75A012E86EE057AF6
:10EB880037EE257A77EEC77A84ED267AE6EE276A9D
:10EB980084ED257AF0EE667AC4ED286AC4ED276A1A
:10EBA80003F02E81F880B4F8A8309BF80080013B70
:10EBB800A4F8A83004990023B8F1070F4B608B60C4
:10EBC800CB607FF425ADF3F7FFFC754F9AF8283139
:10EBD8000593A0EB09003880002B3FF41FAD013BE3
:10EBE8008AF8283119B0BDEC0C8BBDE8F08F9AF883
:10EBF800643163B1022D04F0A7826A4B06936A4A16
:10EC080003EB450332F91510B3F90A30B0E5674B49
:10EC1800234493ED000A019BD3ED01DA009B28EE13
:10EC2800800A3CEE6DDA022D20EE0D0A83ED000A13
:10EC38007FF4CBAD5E4A5F4B10681B6898475E4B0C
:10EC4800D9ED006A93ED007A5C4BD6ED007A1A781C
:10EC58005B4B83ED020A5B4B26EE877A234427EE53
:10EC6800087A93ED006A27EE067AF0EE676AE7EE17
:10EC78000D6A012AB0EE667A02D0192A7FF4BCAD7B
:10EC8800B4EEEADAF1EE10FACCBF01230023BEE5B8
:10EC9800DAED566A9AED577AB2F900E0B2F90270E5
:10ECA800B4EEE67AF1EE10FA8EEAEE7087EAE77CC7
:10ECB8004CBFB7EE007AF7EE006AA0EBEE70ACEB53
:10ECC800E77C4CBF77EE665A76EEC75A604540F34C
:10ECD8004587BEF1000FD6BFCEF1000007EE10EA5F
:10ECE80007EE100A384FB8EEC77A3F7827EE097A50
:10ECF800002F00F04387354F97ED005AB5EEC05A04
:10ED0800F1EE10FA41F35886314FD7ED004AF5EE8F
:10ED1800C04AF1EE10FA41F34F8634EEC77AB7EEE7
:10ED2800006AC7EE246A75EEC65AF4EEC66A65EE46
:10ED38008A5AF1EE10FA85EE857A88BFF0EE466AB7
:10ED4800F5EEC06AF1EE10FA37EE067AB8BFF0EECB
:10ED58006C6A66EE876AF4EEC66AF1EE10FA88BF4E
:10ED6800F0EE466AF5EEC06AF1EE10FAB8BFF0EEC2
:10ED78006C6A184F97ED007A67EE877AA7EEA6CAF5
:10ED8800F3E400BFE03F0020DC3F0020F83F002014
:10ED980000000000087B00200C7000204478002050
:10EDA800E4410020843400205C420020107B0020D5
:10EDB800D03E0020E43E002028000020047B0020F4
:10EDC800FC3300201C7B0020487B0020447B002073
:10EDD8004C7B0020407B0020E24B03935B8BE24995
:10EDE800079107EE903AE14B91ED037AE04993EDF4
:10EDF800004AE04BD1ED004AD3ED006ADE4B8AEDC4
:10EE0800614AF8EEE77A029377EE677ACAED604ACC
:10EE1800C7EEA62AD949DA4B91ED008AD949DFED28
:10EE2800DA6A91ED005AD9499FEDD96AD1ED005AB5
:10EE380093ED007AF7EE007AF4EEE72A38EE058AC9
:10EE4800F1EE10FA88BFF0EE672A38EE258AF4EE64
:10EE5800E62AF1EE10FA28EE066AB8BFF0EE662A46
:10EE6800F1EE476A34EEC43AB4EEE66AF1EE10FA0F
:10EE7800CAED622A8AED643A00F16B85B4EEC76A7E
:10EE8800F1EE10FA88BFB0EE476ABC4BDFEDC07AEE
:10EE9800D3ED018ABB4B93ED015ABC4B78EE858AC2
:10EEA800D3ED015A78EEA58A68EEA77AF4EEE76A00
:10EEB800F1EE10FA08DCB4EEE77AF1EE10FA8CBF46
:10EEC800F0EE676AF0EE476AAC4BDFEDB17A93ED8E
:10EED800029AAC4BD3ED025AAE4B39EE259A93ED1C
:10EEE800007A69EE277AF1EE475AF4EEE57AF1EE08
:10EEF80010FA08D4F4EEC77AF1EE10FA8CBFF0EEEF
:10EF0800475AF0EE675A002A41F08982F7EE007AF4
:10EF1800A14B5A789AF89431002AA04AFFEE003A99
:10EF2800B7EE007A127814BFB0EE472AB0EE632A23
:10EF3800002B14BFB0EE635AB0EE475A002A02F015
:10EF48005B84F4EEC77AF1EE10FA65EE825A944BC0
:10EF580041F3128393ED027A93ED011AD3ED031A6C
:10EF68009FED892A26EE877A67EE853AA6EE017A22
:10EF7800A5EEA17A27EE237AB4EEC27AF1EE10FA62
:10EF8800B4BFF0EE427AF0EE477A8DED0C7A88BF86
:10EF9800B0EE427A012A00F0BE8193ED065AD3ED15
:10EFA800051A93ED072A26EE855AA6EE215AA5EEF4
:10EFB800825A25EE235AB4EEC57AF1EE10FAF4EE31
:10EFC800C57A8CBFB0EE452AB0EE472AF1EE10FAAA
:10EFD80058BFB0EE427AB8BFF0EE457A022A8DEDFE
:10EFE8000D5A00F0988193ED0A5AD3ED091A93ED62
:10EFF8000B2A26EE855AA6EE215AA5EE825A25EE50
:10F00800235AB4EEC57AF1EE10FAF4EEC57A8CBF45
:10F01800B0EE452AB0EE472AF1EE10FA58BFB0EE2E
:10F02800427AB8BFF0EE457A032A8DED0E5A00F009
:10F03800728193ED0E5AD3ED0D1A93ED0F2A26EE39
:10F04800855AA6EE215AA5EE825A25EE235AB4EE29
:10F05800C57AF1EE10FAF4EEC57A8CBFB0EE452A07
:10F06800B0EE472AF1EE10FA58BFB0EE427AB8BFB8
:10F07800F0EE457A042A8DED0F5A00F04C8193ED9D
:10F08800125AD3ED111A93ED132A26EE855AA6EEDD
:10F09800215AA5EE825A25EE235AB4EEC57AF1EE2E
:10F0A80010FAF4EEC57A8CBFB0EE452AB0EE472AC6
:10F0B800F1EE10FA58BFB0EE427AB8BFF0EE457ADA
:10F0C800052A8DED105A00F0268193ED165AD3EDDE
:10F0D800151A93ED172A26EE855AA6EE215AA5EEA3
:10F0E800825A25EE235AB4EEC57AF1EE10FAF4EE00
:10F0F800C57A8CBFB0EE452AB0EE472AF1EE10FA79
:10F1080058BFB0EE427AB8BFF0EE457A062A8DEDC8
:10F11800115A00F0008193ED1A5AD3ED191A93EDA4
:10F128001B2A26EE855AA6EE215AA5EE825A25EE0E
:10F13800235AB4EEC57AF1EE10FAF4EEC57A8CBF14
:10F14800B0EE452AB0EE472AF1EE10FA58BFB0EEFD
:10F15800427AB8BFF0EE457A072A8DED125A00F0D0
:10F16800DA801FE04C4A0020F8850020483500204E
:10F17800DC3F0020F03F00209B440020FC330020AF
:10F18800787B0020083400200000000014340020A0
:10F198006F12833A7C7B0020F83600202034002050
:10F1A8001C3F002093ED1E5AD3ED1D1A93ED1F2A24
:10F1B80026EE855AA6EE215AA5EE825A25EE235A46
:10F1C800B4EEC57AF1EE10FAF4EEC57A8CBFB0EE63
:10F1D800452AB0EE472AF1EE10FA58BFB0EE427A4F
:10F1E800B8BFF0EE457A082A8DED135A00F09380E7
:10F1F80093ED225AD3ED211A93ED232A26EE855A50
:10F20800A6EE215AA5EE825A25EE235AB4EEC57A07
:10F21800F1EE10FAF4EEC57A8CBFB0EE452AB0EEE6
:10F22800472AF1EE10FA58BFB0EE427AB8BFF0EEB6
:10F23800457A092A8DED145A6DD093ED265AD3EDEF
:10F24800251A93ED272A26EE855AA6EE215AA5EE11
:10F25800825A25EE235AB4EEC57AF1EE10FAF4EE8E
:10F26800C57A8CBFB0EE452AB0EE472AF1EE10FA07
:10F2780058BFB0EE427AB8BFF0EE457A0A2A8DED53
:10F28800155A48D093ED2A5AD3ED291A93ED2B2A13
:10F2980026EE855AA6EE215AA5EE825A25EE235A65
:10F2A800B4EEC57AF1EE10FAF4EEC57A8CBFB0EE82
:10F2B800452AB0EE472AF1EE10FA8DED165A58BFDE
:10F2C800B0EE427AA8BFB0EE675A0B2A02F0F1847A
:10F2D800D3ED2E7AD3ED2D1A93ED2F2A66EEA77A69
:10F2E800E1EE867AE2EE257A67EEA37AF4EEC77A43
:10F2F800F1EE10FAF4EEC57A8CBFF0EE476AF0EE44
:10F30800676AF1EE10FACDED177A98BFB0EE667A1B
:10F31800B8BFF0EE457A77EEC77AF7EE006AF4EEFA
:10F32800E67AF1EE10FACAED4C7A42F3B28486EE30
:10F33800A77A012ADDED0C7A67EE877ACDED0C7A93
:10F3480055D0DDED0D7A67EE877A022ACDED0D7A7C
:10F358004DD0DDED0E7A67EE877A032ACDED0E7A71
:10F3680045D0DDED0F7A67EE877A042ACDED0F7A66
:10F378003DD0DDED107A67EE877A052ACDED107A5B
:10F3880035D0DDED117A67EE877A062ACDED117A50
:10F398002DD0DDED127A67EE877A072ACDED127A45
:10F3A80025D0DDED137A67EE877A082ACDED137A3A
:10F3B8001DD0DDED147A67EE877A092ACDED147A2F
:10F3C80015D0DDED157A67EE877A0A2ACDED157A24
:10F3D8000DD0DDED167A67EE877A0B2ACDED167A19
:10F3E80005D0DDED177A27EE877A8DED177AE14B98
:10F3F800196811F0805100F0AC834FF07C53CAF8C3
:10F408008831002A02F0F281029BDB4E1F78DB4C28
:10F41800DB48DC4DD6ED005A9AF88C31039EE4782F
:10F428000078B5F90650DAED626A768B07F0010CC0
:10F43800019F07F0100E07F48007002B40F0AB8205
:10F44800BEF1000F00F0AE85BCF1000F42F07E83E4
:10F45800002C42F05A84CC4BDDED0C7A93ED007A07
:10F46800CA48E7EE267ABDEEE47A17EE101AB0EE37
:10F47800447AA3EE277A0D46F0EE477AFDEEE77A56
:10F48800BDEEC47A17EE906A17EE104AB142A8BFD3
:10F498003546B442C8BF254607EE905AF8EEE77ADB
:10F4A800012AC0ED007A00F04D8193ED047ADDED7C
:10F4B8000D7AE7EE267AB0EE447AA3EE277AFDEECF
:10F4C800C77A17EE906A17EE905A8E42A8BF0D467B
:10F4D800A642B8BF254607EE905AF8EEE77A022A08
:10F4E800C0ED017A00F02E8193ED087ADDED0E7AF9
:10F4F800E7EE267AB0EE447AA3EE277AFDEEC77AD5
:10F5080017EE906A17EE905A8E42A8BF0D46A64293
:10F51800B8BF254607EE905AF8EEE77A032AC0ED01
:10F52800027A00F00F8193ED0C7ADDED0F7AE7EEA9
:10F53800267AB0EE447AA3EE277AFDEEC77A17EE64
:10F54800906A17EE905A8E42A8BF0D46A642B8BFE1
:10F55800254607EE905AF8EEE77A042AC0ED037ABA
:10F5680000F0F08093ED107ADDED107AE7EE267A60
:10F57800B0EE447AA3EE277AFDEEC77A17EE906ACA
:10F5880017EE905A8E42A8BF0D46A642B8BF254630
:10F5980007EE905AF8EEE77A052AC0ED047A00F0F3
:10F5A800D18093ED147ADDED117AE7EE267AB0EE8C
:10F5B800447AA3EE277AFDEEC77A17EE906A17EE23
:10F5C800905A8E42A8BF0D46A642B8BF254607EE00
:10F5D800905AF8EEE77A062AC0ED057A00F0B28074
:10F5E80093ED187ADDED127AE7EE267AB0EE447ADA
:10F5F800A3EE277AFDEEC77A17EE906A17EE905AB7
:10F608008E42A8BF0D46A642B8BF254607EE905ABF
:10F61800F8EEE77A072AC0ED067A00F0938093EDBA
:10F628001C7ADDED137AE7EE267AB0EE447AA3EE83
:10F63800277AFDEEC77A17EE906A17EE905A8E4237
:10F64800A8BF0D46A642B8BF254607EE905AF8EE69
:10F65800E77A082AC0ED077A74D093ED207ADDEDB9
:10F66800147AE7EE267AB0EE447AA3EE277AFDEE16
:10F67800C77A17EE906A17EE905A8E42A8BF0D46C9
:10F68800A642B8BF254607EE905AF8EEE77A092A4F
:10F69800C0ED087A56D093ED247ADDED157AE7EEC1
:10F6A800267AB0EE447AA3EE277AFDEEC77A17EEF3
:10F6B800906A17EE905A8E42A8BF0D46A642B8BF70
:10F6C800254607EE905AF8EEE77A0A2AC0ED097A3D
:10F6D80038D093ED287ADDED167AE7EE267AB0EE8B
:10F6E800447AA3EE277AFDEEC77A17EE906A17EEF2
:10F6F800905A8E42A8BF0D46A642B8BF254607EECF
:10F70800905AF8EEE77A0B2AC0ED0A7A1AD093EDF0
:10F718002C7ADDED177AE6EE877AA3EE274AFDEE1E
:10F72800C47A17EE903A9942A8BF19469C42D8BFAE
:10F738000C4607EE904AF8EEE77AC0ED0B7A002AFD
:10F7480000F0F98392001249104820F091FB114B08
:10F758001B68002B00F0F4830F4B1B78192B22D861
:10F7680001220E4902FA03F31940002942F054839A
:10F7780016E000BF30350020E83E0020844100201C
:10F78800744500203C8B00201C3F0020543400208E
:10F79800EC3E0020007B0020047B00203241300337
:10F7A8001E0301F1AE86AD4DAD4E019B9C061BD5E7
:10F7B800F37AFF2B04D0AB4A12789A4201F29C8666
:10F7C800B6F90870F37D2F80FF2B04D0A54A127874
:10F7D8009A4201F28C86B6F914406C8008200CF02D
:10F7E80035FE002841F0A083B6F90600B5F900E01F
:10F7F800B5F90270B6F91210B6F91E20B5F9044031
:10F80800B6F90430B5F906C07045A8BF7046B942CC
:10F81800A8BF3946A242A8BF22469E45A8BF0346B4
:10F828002B80B6F91030B5F90800BB42C8BF19469D
:10F83800B6F92A306980B6F91C10B6F934706345F8
:10F84800A8BF6346A142CCBF0C461446B6F9362081
:10F85800AC80B6F92840B5F90A108242A8BF024622
:10F86800A445ACBF9C46A446B6F94230B5F90C4055
:10F87800A5F806C08B42A8BF0B468742CCBF3846C6
:10F888001046B6F94E202881B6F94000B5F90E7039
:10F89800A242A8BF22468842C8BF0346B6F95A000A
:10F8A800B6F94C106B81B842B6F958306E4EA8BF05
:10F8B80038469F42A8BF0346A142D8BF1146A98136
:10F8C800EB81B38923B3694FDFF8B891DFF89081F2
:10F8D80007F11004B7F9023000EE103A4846B8EEC6
:10F8E800C00AF0F78DFF20F037FCB8F90430B8F9FA
:10F8F800062000B2984209F12C0908F10C0803DB34
:10F9080082421346A8BF034627F8023FA742E1D127
:10F91800574B1B78013B182B00F2C485DFE813F026
:10F92800B005C205C205F00AC205C205C2051F0E10
:10F93800C205C205C205C205C2055F0EC205C205E1
:10F94800C205C2050E0EF00A500EC205C2055F0EB2
:10F95800B005B0EE666AFFF798BA464BDFF828A103
:10F968001968454A454F9AF80031C96912883980A3
:10F978007A80002B3EF4CFADF7F70EFC00238AF80F
:10F9880000319BF80030072B7EF4C5ADF2F71CFE62
:10F998008146FEF7C2BDBEF1000F00F04B81BCF1FD
:10F9A800000F42F02181002841F03A82FDEEC47A2E
:10F9B8000DF1300E17EE906AFDEEE47A0EEB82033D
:10F9C80017EE907AFDEEE57A2D48DFF8C090CDF875
:10F9D80024A017EE905AB1EE436A84F001084FFA5A
:10F9E80084FC08929A46034693ED007AFEEC017A6D
:10F9F800E7EE267A3A461030B0EE647AA6EE277A19
:10FA0800FDEEC77A17EE903A9F42A8BF1A469D426C
:10FA1800CCBF002104F00101002914BF114629467A
:10FA28009E42CCBF002308F0010307EE901A002B7A
:10FA380014BF13463346B8EEE77A07EE903AF8EE6D
:10FA4800E77ABCF1000F18BFF0EE477AD645E9EC2B
:10FA5800017AC8D1089ADDF824A070E64434002061
:10FA6800E47B0020CC840020608200204234002007
:10FA7800047B0020B88600209A2F0020E441002053
:10FA88001C3F0020BC780020EC23002054340020C8
:10FA9800069BB2F90070B3F90A305A49F81A096896
:10FAA80080EAE073A3EBE0738B42BEF67EAEB2F958
:10FAB8000230069AB2F90C209A1A82EAE273A3EB92
:10FAC800E27399427EF771AE04994F4BD1ED017AFA
:10FAD80093ED007AF0EEE77AF4EEC77AF1EE10FAD9
:10FAE8007EF563AED1ED027AF0EEE77AB4EEE77A0E
:10FAF800F1EE10FA7EF759AE444B1A8800238AF8C3
:10FB08006431002A40F0EA83414A424B1178186870
:10FB180081F00101F3F72AFAFEF747BE3E4B3F4A50
:10FB28002344D3ED006A92ED007A3D4B26EE877AA6
:10FB3800F7EE006AB4EEE67AD3ED007AF1EE10FA49
:10FB480088BFB0EE667A27EE277A67EE0C7AFEF762
:10FB580087BE019B5F023FF550AC52E4002FD6BF31
:10FB6800784207EE107A07EE100A2E4FB8EEC77AE1
:10FB78003F7827EE097A002F7FF4BDA82A4FD7EDEA
:10FB8800006AF4EECB6AF1EE10FA40F1BE87B7EEE8
:10FB9800005A35EE665A9FED256A254F3BEEC77A27
:10FBA80025EE065A97ED006AE7EE056A26EE867A94
:10FBB800B5EEC07AF1EE10FA40F2FE86CAEE076A98
:10FBC800B7EE006A35EEC67AF0EE465AE7EE265AE8
:10FBD800F0EE656AFFF7BFB801230399CAF8681108
:10FBE800022A8AF864317EF469AE084A1288002A2B
:10FBF80043F0E181064A074B11781868F3F7B6F924
:10FC0800FEF75CBE687B00206C7B0020144500205A
:10FC1800164500201845002044250020387B002088
:10FC2800347B0020487B0020507B0020610BB63BD2
:10FC3800447B0020D44BDDED0C7A93ED007A00284C
:10FC480040F09887E7EE267AD048B1EE436AB0EEE6
:10FC5800647AA6EE277AF0EE477ABDEEE47A002CB5
:10FC680042F0F282FDEEE77A17EE104A17EE906A3C
:10FC7800FDEEC47AB44217EE901A17EE105AA8BFD8
:10FC88003546B142C8BF0D4607EE905AF8EEE77AFE
:10FC9800012AC0ED007A00F04A8193ED047ADDED87
:10FCA8000D7AE7EE267AB0EE647AA6EE277AFDEEB4
:10FCB800C77A17EE906A17EE905AA642A8BF254653
:10FCC8008E42B8BF0D4607EE905AF8EEE77A022A40
:10FCD800C0ED017A00F02B8193ED087ADDED0E7A04
:10FCE800E7EE267AB0EE647AA6EE277AFDEEC77ABA
:10FCF80017EE906A17EE905AA642A8BF25468E4284
:10FD0800B8BF0D4607EE905AF8EEE77A032AC0ED21
:10FD1800027A00F00C8193ED0C7ADDED0F7AE7EEB4
:10FD2800267AB0EE647AA6EE277AFDEEC77A17EE49
:10FD3800906A17EE905AA642A8BF25468E42B8BFD1
:10FD48000D4607EE905AF8EEE77A042AC0ED037ADA
:10FD580000F0ED8093ED107ADDED107AE7EE267A6B
:10FD6800B0EE647AA6EE277AFDEEC77A17EE906AAF
:10FD780017EE905AA642A8BF25468E42B8BF0D4638
:10FD880007EE905AF8EEE77A052AC0ED047A00F0FB
:10FD9800CE8093ED147ADDED117AE7EE267AB0EE97
:10FDA800647AA6EE277AFDEEC77A17EE906A17EE08
:10FDB800905AA642A8BF25468E42B8BF0D4607EE08
:10FDC800905AF8EEE77A062AC0ED057A00F0AF807F
:10FDD80093ED187ADDED127AE7EE267AB0EE647AC2
:10FDE800A6EE277AFDEEC77A17EE906A17EE905ABC
:10FDF800A642A8BF25468E42B8BF0D4607EE905AC8
:10FE0800F8EEE77A072AC0ED067A00F0908093EDC5
:10FE18001C7ADDED137AE7EE267AB0EE647AA6EE68
:10FE2800277AFDEEC77A17EE906A17EE905AA64227
:10FE3800A8BF25468E42B8BF0D4607EE905AF8EE89
:10FE4800E77A082AC0ED077A71D093ED207ADDEDC4
:10FE5800147AE7EE267AB0EE647AA6EE277AFDEEFB
:10FE6800C77A17EE906A17EE905AA642A8BF2546A1
:10FE78008E42B8BF0D4607EE905AF8EEE77A092A87
:10FE8800C0ED087A53D093ED247ADDED157AE7EECC
:10FE9800267AB0EE647AA6EE277AFDEEC77A17EED8
:10FEA800906A17EE905AA642A8BF25468E42B8BF60
:10FEB8000D4607EE905AF8EEE77A0A2AC0ED097A5D
:10FEC80035D093ED287ADDED167AE7EE267AB0EE96
:10FED800647AA6EE277AFDEEC77A17EE906A17EED7
:10FEE800905AA642A8BF25468E42B8BF0D4607EED7
:10FEF800905AF8EEE77A0B2AC0ED0A7A17D093EDFC
:10FF08002C7ADDED177AE6EE877AE6EE274AFDEEE3
:10FF1800E47A17EE903A9C42A8BF1C469942D8BF93
:10FF2800214607EE901AF8EEE77AC0ED0B7ABCF19D
:10FF3800000F3FF404AC164B1B68002B7FF40CAC8D
:10FF4800144B1B7893B1144B187860B10F4D134EB6
:10FF58000024E0B23368B5EC010A98470E4B1878D4
:10FF680001348442F5DB0E4B1B6898479BF8003040
:10FF7800072B00F0AB8501238AF8003119B0BDECDE
:10FF88000C8BBDE8F08F00BF1C3F002054340020CC
:10FF9800007B0020DC490020203400206845002038
:10FFA80070450020D24BDDED0C7A93ED007A002CE1
:10FFB80041F05484E7EE267ACE48BDEEE47A17EE97
:10FFC800101AB0EE447AA3EE277A0D46F0EE477A7F
:10FFD800FDEEE77ABDEEC47A17EE906A17EE104A86
:10FFE800B142A8BF3546B442C8BF254607EE905A6D
:08FFF800F8EEE77A012AC0EDE2
:020000040801F1
:10000000007A98D093ED047ADDED0D7AE7EE267A4A
:10001000B0EE447AA3EE277AFDEEC77A17EE906A27
:1000200017EE905A8E42A8BF0D46A642B8BF25468D
:1000300007EE905AF8EEE77A022AC0ED017A3FF413
:100040007AAF93ED087ADDED0E7AE7EE267AB0EE20
:10005000447AA3EE277AFDEEC77A17EE906A17EE80
:10006000905A8E42A8BF0D46A642B8BF254607EE5D
:10007000905AF8EEE77A032AC0ED027A3FF45BAFBC
:1000800093ED0C7ADDED0F7AE7EE267AB0EE447A46
:10009000A3EE277AFDEEC77A17EE906A17EE905A14
:1000A0008E42A8BF0D46A642B8BF254607EE905A1D
:1000B000F8EEE77A042AC0ED037A3FF43CAF93ED03
:1000C000107ADDED107AE7EE267AB0EE447AA3EEF0
:1000D000277AFDEEC77A17EE906A17EE905A8E4295
:1000E000A8BF0D46A642B8BF254607EE905AF8EEC7
:1000F000E77A052AC0ED047A3FF41DAF93ED147A38
:10010000DDED117AE7EE267AB0EE447AA3EE277A97
:10011000FDEEC77A17EE906A17EE905A8E42A8BF8E
:100120000D46A642B8BF254607EE905AF8EEE77A8C
:10013000062AC0ED057A3FF4FEAE93ED187ADDEDA8
:10014000127AE7EE267AB0EE447AA3EE277AFDEE35
:10015000C77A17EE906A17EE905A8E42A8BF0D46E6
:10016000A642B8BF254607EE905AF8EEE77A072A6E
:10017000C0ED067A3FF4DFAE93ED1C7ADDED137A25
:10018000E7EE267AB0EE447AA3EE277AFDEEC77A40
:1001900017EE906A17EE905A8E42A8BF0D46A642FF
:1001A000B8BF254607EE905AF8EEE77A082AC0ED68
:1001B000077A3FF4C0AE93ED207ADDED147AE7EED6
:1001C000267AB0EE447AA3EE277AFDEEC77A17EED0
:1001D000906A17EE905A8E42A8BF0D46A642B8BF4D
:1001E000254607EE905AF8EEE77A092AC0ED087A1C
:1001F0003FF4A1AE93ED247ADDED157AE7EE267A91
:10020000B0EE447AA3EE277AFDEEC77A17EE906A35
:1002100017EE905A8E42A8BF0D46A642B8BF25469B
:1002200007EE905AF8EEE77A0A2AC0ED097A3FF411
:1002300082AE93ED287ADDED167AE7EE267AB0EEFF
:10024000447AA3EE277AFDEEC77A17EE906A17EE8E
:10025000905A8E42A8BF0D46A642B8BF254607EE6B
:10026000905AF8EEE77A0B2AC0ED0A7A3FF463AEB3
:1002700093ED2C7ADDED177AE6EE877AA3EE274A26
:10028000FDEEC47A17EE903A9942A8BF19469C42F7
:10029000D8BF0C4607EE904AF8EEE77AC0ED0B7A2D
:1002A00049E607EE901AF8EEE77A1548154C90EDFE
:1002B000004AD4ED004A1448CAED604A06EE903A6E
:1002C00077EE677ABCEEC77AF8EEE66A17EE103A78
:1002D00077EEE67A8AED614AAAF87C31D0ED006AC1
:1002E000FEF79ABD09494A69002A3EF462AA0A68E3
:1002F00013604B74FEF75DBA1C3F0020543400209D
:10030000E03F0020DC3F0020F83F00201C4500209B
:1003100007EE103A9BF800308E4FCAF81061B8EE25
:10032000C77AF7EE006A132B86EE879AB7F90400B6
:10033000BAF8145194ED080A01F06481864B874A9B
:1003400093ED001A93ED093A93ED162A93ED1F6A87
:10035000D3ED0B1A93ED144AD3ED015AD3ED0A3ABB
:1003600093ED0C7A93ED155AD3ED172AD3ED206A4D
:10037000D3ED044AD3ED030A69EE277A69EE288AA1
:1003800029EE088AA7EE813A02EB85060021A2EE4B
:10039000286ACAF80411CAF80811A8EE214AE7EE43
:1003A000A53AA8EE075A93ED1A7AD3ED0F5A93EDBA
:1003B000021AD3ED0E1A86ED003AE2EEA86A64EE58
:1003C000C34A27EE467A93ED0D2AD3ED192A86ED1E
:1003D000204AE3EE603A65EEC45A93ED183AC3ED55
:1003E000093AE7EE814AF0EE477AA4EE615AE8EE68
:1003F000025AE2EEC66AE3EE287AC3ED0A4A83EDBA
:10040000145AC3ED155A86ED406AC3ED1F6AC3ED59
:10041000207ACAF80C116B1C03F01F03AAF81431E0
:10042000B880FEF7D1B84E4B1A79002A3EF472AD6F
:100430004C4A1278002A3EF46DAD1B789FED4A2A93
:1004400007EE103A494B07EE902A1B88F8EEE77A40
:1004500005EE103AB8EE477AB8EE455A27EE277AFD
:10046000F7EE003AC7EE057AF4EEC27AF1EE10FA32
:1004700088BFF0EE427AF4EEE37AF1EE10FAB8BFFC
:10048000F0EE637AFEF748BDB37B002B42F06B843D
:10049000029B1B7813F0010342F06584344A126812
:1004A000002A02F02186136001230593009B1B683C
:1004B000980633D42F4A1278052A2FD0D9027FF517
:1004C00043ADF57B112D3FF63FAD2B4BDDF814808E
:1004D0001C4633F9153000EE103A4046B8EEC00A1B
:1004E0006F1C05F10E060AF0E5FC4346FFB25D1BEA
:1004F000F6B2A04600E027467C1C7819122FE4B221
:10050000C0B23FF421AD38F9173000EE103AB8EE22
:10051000C00A0AF0CFFCB442EDD115E5059A1346A6
:100520000233541CDBB21046E4B20593B5F9003037
:1005300000EE103AB8EEC00A0AF0BCFCB5F9023081
:1005400000EE103A2046B8EEC00A0AF0B3FC009B59
:100550001B68B3E7E4410020787F0020DC7C0020AA
:1005600078410020F6850020713DAA3FCC8500200F
:1005700070820020047B00203C8B002000000000E3
:1005800093ED027A93ED012AD3ED037A5FED053AFC
:1005900026EE877AA6EE027AA5EEA77A27EE057AEE
:1005A000B4EEE37AF1EE10FAB4BFF0EE637AF0EE57
:1005B000477A8DED0C7A88BFB0EE637A012A3EF45B
:1005C000AEAED3ED063AD3ED051A93ED072A66EEEB
:1005D000A33AE6EE213AE5EE823A63EE853AB4EECE
:1005E000E37AF1EE10FAF4EEE37A8CBFB0EE632A10
:1005F000B0EE472AF1EE10FA58BFB0EE427AB8BF1B
:10060000F0EE637A022ACDED0D3A3EF488AED3EDDA
:100610000A3AD3ED091A93ED0B2A66EEA33AE6EEF9
:10062000213AE5EE823A63EE853AB4EEE37AF1EEF2
:1006300010FAF4EEE37A8CBFB0EE632AB0EE472AEC
:10064000F1EE10FA58BFB0EE427AB8BFF0EE637A1E
:10065000032ACDED0E3A3EF462AED3ED0E3AD3ED61
:100660000D1A93ED0F2A66EEA33AE6EE213AE5EE77
:10067000823A63EE853AB4EEE37AF1EE10FAF4EEE4
:10068000E37A8CBFB0EE632AB0EE472AF1EE10FA9F
:1006900058BFB0EE427AB8BFF0EE637A042ACDEDCF
:1006A0000F3A3EF43CAED3ED123AD3ED111A93ED6E
:1006B000132A66EEA33AE6EE213AE5EE823A63EEBD
:1006C000853AB4EEE37AF1EE10FAF4EEE37A8CBFF9
:1006D000B0EE632AB0EE472AF1EE10FA58BFB0EE42
:1006E000427AB8BFF0EE637A052ACDED103A3EF4B7
:1006F00016AED3ED163AD3ED151A93ED172A66EE22
:10070000A33AE6EE213AE5EE823A63EE853AB4EE9C
:10071000E37AF1EE10FAF4EEE37A8CBFB0EE632ADE
:10072000B0EE472AF1EE10FA58BFB0EE427AB8BFE9
:10073000F0EE637A062ACDED113A3EF4F0ADD3ED3A
:100740001A3AD3ED191A93ED1B2A66EEA33AE6EE98
:10075000213AE5EE823A63EE853AB4EEE37AF1EEC1
:1007600010FAF4EEE37A8CBFB0EE632AB0EE472ABB
:10077000F1EE10FA58BFB0EE427AB8BFF0EE637AED
:10078000072ACDED123A3EF4CAADD3ED1E3AD3EDB1
:100790001D1A93ED1F2A66EEA33AE6EE213AE5EE26
:1007A000823A63EE853AB4EEE37AF1EE10FAF4EEB3
:1007B000E37A8CBFB0EE632AB0EE472AF1EE10FA6E
:1007C00058BFB0EE427AB8BFF0EE637A082ACDED9A
:1007D000133A3EF4A4ADD3ED223AD3ED211A93EDB2
:1007E000232A66EEA33AE6EE213AE5EE823A63EE7C
:1007F000853AB4EEE37AF1EE10FAF4EEE37A8CBFC8
:10080000B0EE632AB0EE472AF1EE10FA58BFB0EE10
:10081000427AB8BFF0EE637A092ACDED143A3EF47D
:100820007EADD3ED263AD3ED251A93ED272A66EE59
:10083000A33AE6EE213AE5EE823A63EE853AB4EE6B
:10084000E37AF1EE10FAF4EEE37A8CBFB0EE632AAD
:10085000B0EE472AF1EE10FA58BFB0EE427AB8BFB8
:10086000F0EE637A0A2ACDED153A3EF458AD93EDD9
:100870002A2AD3ED291AD3ED2B3A26EE822AA6EEA8
:10088000212AA5EEA32A22EE052AB4EEC27AF1EEC1
:1008900010FAF4EEC27A8CBFF0EE423AF0EE473A2C
:1008A000F1EE10FA8DED162A58BFB0EE637AA8BFAC
:1008B000B0EE672A0B2A02F03A83D3ED2E7AD3EDFD
:1008C0002D1AD3ED2F3A66EEA77AE6EE217AE3EE03
:1008D000A57A67EE857AF4EEC77AF1EE10FAF4EEB7
:1008E000C27A8CBFF0EE476AF0EE676AF1EE10FA5A
:1008F000CDED177A98BFB0EE667AB8BFF0EE427AC7
:10090000FEF70DBD904A04920025904E904FDDF801
:100910001080CDF80490A946B6EC018AD4ED087A8F
:10092000B8EEC88A28EE278AB9F1000F02F0EB83EF
:100930007BBB9BF80030082B3BD005F5D260B0EEB6
:10094000480A2044D4F88C36984705F5E360D4F87B
:100950001437204498479BF80030032BB0EE408AB0
:1009600022D0D4F8AC30D6F84406B0EE480A984706
:1009700008EB890309F10109B9F1030F05F12C0511
:1009800083ED010A3DF440AE009B1B6803F0005369
:10099000C2E705F5F460B0EE480A2044D4F89C376D
:1009A0009847B0EE408AC4E71FF0DAFB27F8190039
:1009B000D7E7B0EE480A1FF0D3FB27F81900BCE7D1
:1009C000DFED646AFEF7D9B9DFF8A881DAED017AC4
:1009D0009AED006AB8F80000D8F8143077EEA77ADC
:1009E000F0EE006AB0EE677AA6EE267A01380AEBDE
:1009F000C002D6EE267A083A1033F6EE003A27EE19
:100A0000237A67EEA37A8AED207ACAED217ADFF89D
:100A100068A157460AF1800192ED027A92ED036ACD
:100A2000D7ED036AD7ED027A53ED014A13ED025A6E
:100A300037EE674A76EEC65A77EE277AE4EE845AA6
:100A40000138A2F10802E5EE047A07F1080703F184
:100A5000080336EE267A01F10801E4EE877AE5EE26
:100A6000475A67EEA37A25EEA37AC1ED007A81EDAD
:100A7000017AD1D1142E07D1F1F7AAFD019B344F91
:100A8000C01A7880DAF818512F4B0493324A009B31
:100A9000013582FB05125119EA17C2EBA1021B684E
:100AA000C2EBC202AD1ACAF8185103F000532BE78B
:100AB000F1F78EFD9BF80030079A254F801A012B25
:100AC00078802CD0072B7DF429AFF1F781FD0490BD
:100AD000FDF726BFF1F77CFD049A1D4B801AD880E4
:100AE000FFF74DBA1D491E481E4B91ED004AD0ED4F
:100AF000004A1D491B78CAED604A8AED614AD1ED72
:100B0000006A13B101238AF88C31DAED627AFEF7BC
:100B100083B9164F97ED007AFFF74EB80C4FF1F7F7
:100B200057FD134ADAF8783112680490C31A9A1AFA
:100B3000CAF87801BB80FA80FDF7F2BEF1F748FDF4
:100B40000790FDF77EBD00BF44780020587000205C
:100B5000E441002000000000932449924835002021
:100B6000E43F002074450020F43F0020447B002037
:100B7000E0360020C47C0020EC230020E7EE267A3B
:100B8000DF48B1EE436AB0EE647AA6EE277AF0EE63
:100B9000477ABDEEE47A002C41F09686FDEEE77AC6
:100BA00017EE104A17EE906AFDEEC47AB44217EEC3
:100BB000901A17EE105AA8BF3546B142C8BF0D466D
:100BC00007EE905AF8EEE77A012AC0ED007A3FF47A
:100BD000B2A993ED047ADDED0D7AE7EE267AB0EE58
:100BE000647AA6EE277AFDEEC77A17EE906A17EEC2
:100BF000905AA642A8BF25468E42B8BF0D4607EEC2
:100C0000905AF8EEE77A022AC0ED017A3FF493A9F0
:100C100093ED087ADDED0E7AE7EE267AB0EE647A8F
:100C2000A6EE277AFDEEC77A17EE906A17EE905A75
:100C3000A642A8BF25468E42B8BF0D4607EE905A81
:100C4000F8EEE77A032AC0ED027A3FF474A993ED37
:100C50000C7ADDED0F7AE7EE267AB0EE647AA7EE35
:100C6000C37AFDEEC77A17EE906A17EE905AA64245
:100C7000A8BF25468E42B8BF0D4607EE905AF8EE43
:100C8000E77A042AC0ED037A3FF455A993ED107A70
:100C9000DDED107AE7EE267AB0EE647AA7EEC37A3D
:100CA000FDEEC77A17EE906A17EE905AA642A8BFDB
:100CB00025468E42B8BF0D4607EE905AF8EEE77A09
:100CC000052AC0ED047A3FF436A993ED147ADDEDE0
:100CD000117AE7EE267AB0EE647AA7EEC37AFDEEDB
:100CE000C77A17EE906A17EE905AA642A8BF25461B
:100CF0008E42B8BF0D4607EE905AF8EEE77A062A04
:100D0000C0ED057A3FF417A993ED187ADDED127A5C
:100D1000E7EE267AB0EE647AA7EEC37AFDEEC77AE4
:100D200017EE906A17EE905AA642A8BF25468E424B
:100D3000B8BF0D4607EE905AF8EEE77A072AC0EDE5
:100D4000067A3FF4F8A893ED1C7ADDED137AE6EE0F
:100D5000877A2546B0EE647AA6EE277AFDEEC77A4A
:100D600017EE906AB442A8BF3546B142C8BF0D46DF
:100D700007EE905AF8EEE77A082AC0ED077A3FF4BA
:100D8000DAA893ED207ADDED147AE6EE877A25462F
:100D9000B0EE647AA6EE277AFDEEC77A17EE906A77
:100DA000B442A8BF3546B142C8BF0D4607EE905ABF
:100DB000F8EEE77A092AC0ED087A3FF4BCA893ED73
:100DC000247ADDED157AE6EE877A2546B0EE647A70
:100DD000A6EE277AFDEEC77A17EE906AB442A8BF56
:100DE0003546B142C8BF0D4607EE905AF8EEE77A95
:100DF0000A2AC0ED097A3FF49EA893ED287ADDED2A
:100E0000167AE7EE267A2546B0EE647AA7EEC37A24
:100E1000FDEEC77A17EE906AB442A8BF3546B142DC
:100E2000C8BF0D46FFF767B8FDEEC47A0CA817EEF1
:100E3000906AFDEEE47A00EB820317EE907AFDEE05
:100E4000E57ADFF8C090DFF8B8E0089217EE905A24
:100E5000B1EE436A84F001084FFA84FC1946CDF8DC
:100E600024A04B4693ED007AF0EC017AE7EE267A67
:100E700004F0010309F11009B0EE647AA6EE277AB6
:100E8000B4EEC74AF1EE10FAD8BF0023002BF0EE03
:100E9000477A18BFB0EE657ABDEEC77AFDEEE77A05
:100EA00017EE102A17EE90AABA4217EE103AA8BF12
:100EB0003B469542CCBF002204F00102002A08BF45
:100EC0002B46574507EE103A3A46A8BF52465645BC
:100ED000CCBF002308F00103002B08BF324607EE09
:100EE000902AB8EEC77AF8EEE77ABCF1000F18BF87
:100EF000F0EE477A8842EEEC017AB2D1FEF7AEBD51
:100F0000543400201C3F0020B84BB5F908101A6873
:100F100002B111609B69B5F90A2003B11A60009B08
:100F20001B689A0601F1A58602220592FFF7C6BA50
:100F30009AF8B831012B01F02287AD4B96F91600D3
:100F40005A8896F90AE01B88AA4910FB03F31EFB96
:100F500002F281FB020C81FB0301D217DB17C2EB0B
:100F60002C12C3EB21133A441C442A806C80FEF7F8
:100F70003FBCDFF8A082A048D8F80820B8F80C10D1
:100F80001DF09EFF9BF80060142E02F05880DAF8E6
:100F900018510135CAF8185118E5DFF87882B8F809
:100FA0000060D8F804E04FEA560C4FEA8C020AEBD6
:100FB0008607F6080AEB020300F09F801032013624
:100FC0008E4803EB06163A4410330EF1100507F174
:100FD000100151ED032A51ED043A10ED043A10EDE1
:100FE000032A51ED026A11ED016A10ED020A10EDBB
:100FF000018A12ED044A12ED035A53ED044A53EDEF
:10100000035A13ED027A53ED017A52ED020A12ED02
:10101000011A73EE238A72EE221A40ED048A40ED23
:10102000031A70EE268A78EE061A40ED028A40ED29
:10103000011A74EE848A75EE851A43ED048A43ED35
:10104000031A77EE208A77EE811A43ED028A43ED88
:10105000011A73EE633A75EE655A15ED035A32EED6
:10106000623A74EE644A65EE631A15ED044A23EEA3
:10107000052A64EE652AE3EE041A1033B34224EE27
:10108000843AA3EE842A00F1100005F11005A5EEC4
:10109000853A01F1100102F11002E4EE852A41EDDA
:1010A000071A01ED082A02ED073A42ED082A55ED2C
:1010B000055A15ED065A70EE666A38EE466A30EE4D
:1010C000C77A71EE677A26EE253A65EEE63A25EEA6
:1010D000674A67EE054AE6EE053AA6EE853AA7EEC0
:1010E000254AE7EEA54A01ED063A41ED053A02ED43
:1010F000064A42ED054A7FF46CAF1FFA8CF5724642
:1011000029463D4815F0D6FC2946D8F80420384633
:1011100015F0D0FC9BF80030142B7FF4B3ACABE49B
:10112000374BDAF81CC10493BAF81481C8F12003D4
:10113000D8B2344B08EB4C1703EB8707830801F058
:10114000798701331B0130492C4A029307EB030EC8
:1011500007F1100313ED024A13ED035A13ED016A70
:1011600013ED047A51ED024A51ED035A51ED016A33
:1011700051ED047A64EE244A65EE255A66EE266A3D
:1011800067EE277A1033734542ED024A42ED035A67
:1011900042ED016A42ED047A01F1100102F1100200
:1011A000D8D1029B1949A3F11002174401EB020E9A
:1011B000524410F0030309D0B7EC017AFEEC017A37
:1011C00067EE277A013BE2EC017AF5D1B8F1000F26
:1011D00041F05585142E7FF459ACF1F7F9F9019BD4
:1011E0000B4FDAF81851C01A78804FE47082002053
:1011F0005C4200201F85EB51EC230020FC230020E3
:1012000044780020DC7C00206C7E00205C7E002086
:10121000E4410020C47C0020D94B1A78DAF81CE1A4
:10122000D8489FEDD97A4FEACE07C31983ED007AEB
:10123000002A7AD0D549B0EE476AF0EE476A00231B
:10124000F1EC017A013367EEA77A05EE903AB4EE3D
:10125000E77AF1EE10FAF8EEE55AB8BFB0EE677A29
:10126000934276EEA76AA7EEA56AE9D1F5EEC06AC9
:10127000C319F1EE10FA83ED007A56DDC6EE265A58
:10128000C34BC44A1288F7EE007A75EEE75AD3EDE5
:10129000007A65EEA77AFDEEE77A17EE903A812B99
:1012A00041F309839342A8BF134607EE903AF8EE44
:1012B000E77AB94B2C2101FB0E3393ED097AD3ED7C
:1012C000003A93ED0A6A93ED014AD3ED046AD3ED37
:1012D000034A93ED025AA3EEA77AA4EE276A66EEBC
:1012E000C76AA7EE646ABDEEC77AE5EE276A17EE15
:1012F000101A812983ED096AC3ED0A6A41F3D88285
:101300008A42A8BF0A4607EE902AF8EEE77AFCEE7A
:10131000E77ACDED027ABDF80830C2199380BEF1AC
:10132000000F02D1132E01F05986152E7FF4A2ABC7
:1013300038449A4F838827F81E30994BDAF81851B1
:101340000493FFF7A3BBDAF81C81954A8D4B0492F6
:1013500003EBC803126802929DED027A9B88DFEDD1
:10136000917A914AF8EE478A09EE103A643BC82B0D
:10137000A8BFC82368EEA78AF8EE497A782BB8BFD1
:10138000782368EEA78A07EE903A2C27B0EE680A19
:1013900007FB0827B8EEE78A1EF02EFFB8EEC99AC1
:1013A000F0EE409AB0EE680A1EF088FE38EE097A38
:1013B00079EE487A28EE098A67EE877AB7EE006AF6
:1013C00088EE277A142EF8EE007A77EE076A60EE40
:1013D000277A89EEA67A77EE065A36EE477AC6EE77
:1013E000256A67EEA67A27EE267AC7ED006A87EDB2
:1013F000047AC7ED026AC7ED017AC7ED037A01F0FE
:1014000036866A4B9BF8006008F1010883FB083CB4
:10141000ACEBE87C0CEB4C0C0135A8EB0C0CCAF8DF
:101420001851CAF81CC17FE6DFF8548198F80020F3
:10143000970801F03B86DFF88CC1781C40010CEB6B
:10144000000E0CF12003ACF1700113ED076A53EDAF
:10145000056A13ED037A53ED017A53ED025A13ED49
:10146000084A53ED064A13ED045A26EE066A66EE64
:10147000A66A27EE077A67EEA77AA4EE046A2033FD
:101480007345E4EEA46A01F11001A5EE057AE5EEDC
:10149000A57AF1EEC65AB1EEE66AF1EEC76AB1EE90
:1014A000E77A41ED085A01ED076A41ED066A01ED60
:1014B000057ACAD1203884440AEB071712F00303D7
:1014C00018BF0CF1080C0FD05CED017A1CED027A0C
:1014D00067EEA77A013BE7EE077A0CF1080CB1EE54
:1014E000E77AA7EC017AEFD1142E01F0B28501352D
:1014F000CAF8185192E62E4A32F91340FEF771B934
:101500002B4A32F91370FEF761B9294B294D1A683D
:1015100059682A609A68DB68EB606960264EAA60A9
:10152000019BFEF747B9F1F753F89BF80060019073
:10153000142E05BF194FDAF81851DAF818513D800A
:10154000FDF74BB81D4F002437F9023F00EE103A6B
:10155000E0B2B8EEC00A013409F0ACFC082CF3D1BB
:101560000594FEF7A3BF164BB5F906101A6802B131
:1015700011609B69B5F90820002B7FF4CFACCEE455
:10158000BE7C0020DC7E002000000000EC23002058
:10159000C07C0020BC7C0020F47E0020E4410020C0
:1015A0004478002027D4D236C077002056555555B0
:1015B0003C8B002044340020E47B00204234002097
:1015C000708200206C2400209A4F002437F9023BDF
:1015D00000EE103AE0B2B8EEC00A013409F06AFC3D
:1015E000042CF3D1BCE7944F002437F9023F00EEFE
:1015F000103AE0B2B8EEC00A013409F05BFC062CE8
:10160000F3D1ADE78D4EDFF8588296ED004A96EDA6
:10161000097AD6ED014A96ED0A6AD6ED046A96ED8E
:10162000035AD6ED025A69EE277A08EB8503A7EE36
:10163000847AA7EEA46A66EEC76AA7EE456AE7EE6B
:10164000A56A20EE070A86ED096AC6ED0A6A83EDEF
:10165000007A29EE088A1EF083FD69EE288AD6ED0D
:10166000145AD6ED1F6A96ED0B1AD6ED161A96EDA2
:10167000155A96ED207A96ED0C2AD6ED172A96ED9E
:101680000F6AD6ED1A7A96ED0E3AD6ED0D3A96ED32
:10169000194AD6ED184AE8EE015A002208EB8503F4
:1016A000E8EEA16A00B2CAF80421A8EE025ACAF80C
:1016B0000821CAF80C21A8EEA27A26EE656A67EE28
:1016C000E67AA5EEC35AA8EE236AA6EEC47AE8EE3F
:1016D000A47A86ED145AC3ED205A86ED156AC3ED3F
:1016E000406A86ED1F7AC6ED207AFEF794BEB4F903
:1016F0002430E26207EE903A0122F8EEE77A2366A0
:10170000E2670023012EC4ED1C7AC4ED1B7A6367E7
:1017100001F05184AE427DF4E9A9B4F92630636644
:1017200007EE903A00220123F8EEE77A2263C4F82C
:1017300090300023012EC4ED217AC4ED207AC4F844
:10174000883001F03484AE427DF400AAB4F9283028
:10175000A36607EE903A00220123F8EEE77A62636F
:10176000C4F8A4300023012EC4ED267AC4ED257AF6
:10177000C4F89C307DF41AAA9FED318AB8F1030FAA
:1017800001F0E783009B4BB107EE903AF8EEE77A61
:10179000F4EEC87AF1EE10FA01F18D84294AA36EB5
:1017A00012689AF82011F88003EB550393FBF5F5C6
:1017B0000023656393621363D36221B1224B1B88BC
:1017C000002B7DF4F4A9214B1B6813F4003304D0E3
:1017D0001F4B1B79002B41F063841E491A46C85CDD
:1017E000012803F10C0301F02C820132152AF6D1F5
:1017F000FDF7DDB9029B1F7807F0010CFEF79BBBDC
:10180000154BDFED167A1968CAED4C7A11F080514C
:1018100000F07082B7EE007A77EE677AF4EEE27A43
:10182000F1EE10FA88BFF0EE627ACAED627AFDF747
:10183000ECBD00BF4A34002046340020787F0020F1
:1018400000000000B8860020A8410020E8380020F1
:1018500078410020B83003083035002000000080B7
:10186000DC7C0020002840F05086E7EE267ADE4837
:10187000BDEEE47A17EE105AB0EE447AA3EE277A62
:101880002C46F0EE477AFDEEE77ABDEEE57A17EEEC
:10189000906A17EE101AB542A8BF3446B142C8BFCD
:1018A0000C4607EE904AF8EEE77A012AC0ED007A7E
:1018B0003EF441AB93ED047ADDED0D7AE7EE267A46
:1018C000B0EE447AA3EE277AFDEEC77A17EE906A5F
:1018D00017EE904AAE42A8BF2C468E42B8BF0C46C7
:1018E00007EE904AF8EEE77A022AC0ED017A3EF45C
:1018F00022AB93ED087ADDED0E7AE7EE267AB0EEB4
:10190000447AA3EE277AFDEEC77A17EE906A17EEB7
:10191000904AAE42A8BF2C468E42B8BF0C4607EE96
:10192000904AF8EEE77A032AC0ED027A3EF403AB60
:1019300093ED0C7ADDED0F7AE7EE267AB0EE447A7D
:10194000A3EE277AFDEEC77A17EE906A17EE904A5B
:10195000AE42A8BF2C468E42B8BF0C4607EE904A56
:10196000F8EEE77A042AC0ED037A3EF4E4AA93ED98
:10197000107ADDED107AE7EE267AB0EE447AA3EE27
:10198000277AFDEEC77A17EE906A17EE904AAE42BC
:10199000A8BF2C468E42B8BF0C4607EE904AF8EE20
:1019A000E77A052AC0ED047A3EF4C5AA93ED147ACD
:1019B000DDED117AE7EE267AB0EE447AA3EE277ACF
:1019C000FDEEC77A17EE906A17EE904AAE42A8BFB6
:1019D0002C468E42B8BF0C4607EE904AF8EEE77AE6
:1019E000062AC0ED057A3EF4A6AA93ED187ADDED3D
:1019F000127AE7EE267AB0EE447AA3EE277AFDEE6D
:101A0000C77A17EE906A17EE904AAE42A8BF2C46EE
:101A10008E42B8BF0C4607EE904AF8EEE77A072AE6
:101A2000C0ED067A3EF487AA93ED1C7ADDED137AB9
:101A3000E7EE267AB0EE447AA3EE277AFDEEC77A77
:101A400017EE906A17EE904AAE42A8BF2C468E421F
:101A5000B8BF0C4607EE904AF8EEE77A082AC0EDC8
:101A6000077A3EF468AA93ED207ADDED147AE7EE6A
:101A7000267AB0EE447AA3EE277AFDEEC77A17EE07
:101A8000906A17EE904AAE42A8BF2C468E42B8BF6D
:101A90000C4607EE904AF8EEE77A092AC0ED087A7C
:101AA0003EF449AA93ED247ADDED157AE7EE267A25
:101AB000B0EE447AA3EE277AFDEEC77A17EE906A6D
:101AC00017EE904AAE42A8BF2C468E42B8BF0C46D5
:101AD00007EE904AF8EEE77A0A2AC0ED097A3EF45A
:101AE0002AAA93ED287ADDED167AE7EE267AB0EE93
:101AF000447AA3EE277AFDEEC77A17EE906A17EEC6
:101B0000904AAE42A8BF2C468E42B8BF0C4607EEA4
:101B1000904AF8EEE77A0B2AC0ED0A7A3EF40BAA57
:101B200093ED2C7ADDED177AE6EE877AA3EE274A5D
:101B3000FDEEC47A17EE903A9D42A8BF1D46994229
:101B4000D8BF294607EE901AF8EEE77AC0ED0B7A77
:101B5000FEF7F1B9069B002B01F03281FDEEE57A2C
:101B60000CA917EE90EAFDEEE47A204D1E4E17EE1A
:101B7000903AFDEEC47A01EB820217EE907A14E0FF
:101B8000FDEEC77A17EE908AB84503DB9845C44648
:101B9000A8BF9C4607EE90CAF8EEE77A9142E6ECC1
:101BA000017A05F110053EF4CAA995ED007AF1EC31
:101BB000017AE7EE267ABC46B0EE447AA3EE277AA5
:101BC000F0EE477A002CDBD030B1B4EE474AF1EEAC
:101BD00010FAC8BFF0EE657AFDEEE77AF44617EE2C
:101BE000908AC645D2DDD5E7543400201C3F002042
:101BF000069B002B01F04081FDEEC47A0CAB17EE82
